:020000040800F2
:100000000020001031B90208614002087D03010898
:100010005D400208594002085540020800000000F7
:100020000000000000000000000000005140020835
:100030004D4002080000000049400208EDB80008E9
:1000400099B9020899B9020899B9020899B9020840
:1000500099B9020899B90208A11C0008CD1D000831
:10006000911D0008551D0008191D0008592F000892
:10007000492F0008392F0008292F0008192F0008E0
:10008000052F0008F12E000899B9020899B9020855
:10009000F140020899B9020899B90208DD1C00086C
:1000A00065B0000895B0000855B00008A5B000087C
:1000B00085B0000875B0000899B9020899B902081E
:1000C00099B9020899B9020899B9020899B90208C0
:1000D00099B9020871BA0008F5B9000879B90008A1
:1000E000651C000899B902083940020899B902084C
:1000F00099B9020899B9020899B9020899B9020890
:1001000000000000000000000000000099B9020893
:1001100099B9020899B90208C5630108A9630108E1
:10012000DD2E0008C92E0008B52E0008A12E0008FB
:100130008D2E000899B902080000000000000000A0
:1001400099B9020899B9020899B90208000000009B
:10015000000000000000000000000000000000009F
:10016000000000000000000099B9020899B90208D7
:1001700099B9020800000000000000000000000023
:080180000000000099B902081B
:100188000023037043708370C37070472D2343703E
:100198002E2303712F23C371704700BF2DE9F0414F
:1001A800846814B12568A4882C8541F080014468CE
:1001B80040F2E93501E0002D51D02689013D16F0C5
:1001C800020FADB2F7D0217304F10C0640F2E93109
:1001D80001E000294DD02589013915F0010F89B2B8
:1001E800F7D031784468A1894FF0000C4FF47A7148
:1001F8004FF6FF764FF0FF0E634502D127E0B1427C
:100208001CD025890139AF0789B2F8D584F80CE0EC
:1002180004F10C084FF47A7102E0B9B2B1420DD082
:100228002589ED0701F1FF37F7D598F80050EDB2B1
:100238000AB1157001320CF1010CDDE7124B9C423A
:1002480005D1124A538B01339BB25383538B836876
:1002580013B11A689B8893610120BDE8F0810A49AF
:100268008C42C0D1094D698B013189B26983698B90
:10027800B9E705498C42B5D1044C618B013189B28B
:100288006183618B4468AEE70038004084720020C7
:1002980030B4836813B11C689B882385436840F297
:1002A800E93401E0002C3FD01D89013C15F0020F14
:1002B800A4B2F7D0197303F10C0540F2E93101E05B
:1002C80000293BD01C89013914F0010F89B2F7D0FD
:1002D8002B78436840F2E93100E0D9B11C89013933
:1002E80014F0020F89B2F8D01A7303F10C0440F22B
:1002F800E93200E072B11989013A11F0010F92B2A6
:10030800F8D02378836813B11A689B889361012019
:1003180030BC70470F4A9342F4D10F4A538B0133D4
:100328009BB25383538BEDE70A498B42D2D10A4CD7
:10033800618B013189B26183618BCBE705498B42BF
:10034800C7D105494B8B01339BB24B834B8B436819
:10035800C0E700BF0038004084720020002870B554
:100368001EDB0928044620DD012303EB83035B0021
:10037800B0FBF3F2092AF8D87BB10E4EB4FBF3F0C8
:100388000928CCBF57223022A6FB03E5024403FB11
:100398001044EB0801F8012BF0D100230B7070BD5D
:1003A8002D230B7040420131DBE7303001F8010B9F
:1003B800F3E700BFCDCCCCCC884230B44FF0010479
:1003C8002ED301FB04F4B0FBF4F58D42F9D284B1CD
:1003D800AAB901E0B0FBF4F5092DCCBF57223022B1
:1003E8002A4404FB150003F8012BB4FBF1F4002C9C
:1003F800F0D100221A7030BC7047B0FBF4F5092D1B
:10040800CCBF372230222A4404FB150003F8012B05
:10041800B4FBF1F4002CF0D100221A7030BC704704
:100428000546002AEBD1D7E703685A1C0260197009
:10043800704700BF2DE9F047089C2578002B8046BF
:1004480089460CBF4FF0200A4FF0300A661C35B3BE
:10045800002A29DD334601E0024698B113F8011B52
:10046800501E0029F8D1971E60B13D46013D514606
:100478004046C8476B1C002BF8DC257827EAE77054
:10048800013055B1041B29464046C847301916F8B3
:10049800015B002DF7D1BDE8F087BDE8F087002AA1
:1004A80004DC2846BDE8F0870020EBE7571EDCE7B0
:1004B80083684268D0ED037A00EB830101339342ED
:1004C80081ED040A836004BF0023836000EB83038B
:1004D80093ED047A036870EE277A9A42C0ED037AA6
:1004E80077EEC77AC0ED037A0CDA013307EE103ADB
:1004F800F8EEC76AB7EE007A87EEA60A036030EE18
:10050800070A704707EE102AB8EEC77A87EE870AFF
:10051800704700BF90ED057A90ED004AD0ED066A6D
:10052800D0ED014AD0ED047A90ED035AD0ED025A8D
:10053800A4EE007AB0EE406AB0EE470AB0EE667AF2
:10054800A6EE247A67EEC07AA0EE457AE6EE257A22
:1005580080ED057AC0ED067A704700BFD0ED057AC8
:1005680090ED013AD0ED003AD0ED064A90ED024AFE
:1005780090ED077A90ED035A90ED086AD0ED045A91
:10058800C0ED067AF0EE406A27EE830AC0ED056AF0
:10059800A3EEA60A80ED087AA4EE240AA5EE470A7F
:1005A800A5EEC60A80ED070A704700BFD0ED007AB5
:1005B80090ED017A30EE670AE7EE007AB0EE670A4E
:1005C800C0ED007A704700BF704700BF0A449142EF
:1005D80014D030B40139551E41F2210211F8014FEF
:1005E800082380EA042004044CBF82EA400040004B
:1005F800013B80B2F7D18D42F0D130BC704700BFCB
:100608002A4B1B7813B12A4B1B7803B970472DE985
:10061800F04328490B7803F0FF0E002B44D1264DF8
:100628002B68C31A002B3FDB244B254E1A786C68C5
:10063800244BDFF8A49013F80480013A570007EB25
:10064800020C06EB4C0C3A44BCF8043006EB4206AC
:10065800A9FB03C372880134DB086C600E2C03FB12
:1006680008F310440C7888BFC5F804E003442B60F5
:1006780034B1154803680A780133002AFBD10360B6
:10068800124A1348134B126800681C8A012500237C
:100698000D705460436203889BB22B430380136838
:1006A8002B431360BDE8F083BDE8F083F8350020E4
:1006B800F9350020305A0020A01D0020345A0020AF
:1006C8007CE50208CCE10208285D0020C023002058
:1006D800C4230020405A0020CDCCCCCC70B40F4CA1
:1006E8000F4E054607CC0023AA603446286069608F
:1006F800042200E0A27912F0200F04F1140404D1BE
:1007080001330A2BF6D170BC704703EB830306EB69
:1007180083031B79EB7270BC704700BFDCE10208F1
:100728003C05030810B40268047B11680223A34047
:10073800194209D00649406800240C7001684FF638
:10074800FE742140016053605DF8044B704700BFA0
:10075800305A00204FF480538382704750F8043C8D
:10076800012280F84520103803B11847704700BFB0
:1007780070B5044682B00830656A06236A463B2194
:10078800A847A8B19DF804009DF800609DF80110E5
:100798009DF802509DF803209DF8053041EA062196
:1007A80043EA002342EA0522E1822283638301208F
:1007B80002B070BD70B40468037B2268022101FA9C
:1007C80003F31A4213D042690A49582000FB021267
:1007D8004FF6FE7650685289C5680068296831402E
:1007E8002960C168D24392B20A40C260636070BC9B
:1007F800704700BFB453002030B4094B1C7864B173
:10080800084B002503EBC4041A6899885562D06820
:1008180008330143A342D160F6D130BC704700BF12
:10082800745600207856002010B40268047B1168C2
:100838000223A340194209D00649406800240C70DD
:1008480001684FF6FE742140016053605DF8044B67
:10085800704700BFC73800202DE9F34105690646F7
:100868000F467DBBD0F80080C8F30A0323B30023EA
:10087800D6F80080019321F0A7FE042819D1224C54
:10088800236943F001032361BBB2A8F8003021F0CB
:100898009BFE04282ED108F102030193019B3F0C13
:1008A8001F8021F091FE2369042823F001032361AE
:1008B80025D06FF0010505E021F086FE042805D05B
:1008C8004FF0FF35284602B0BDE8F0810E4C236991
:1008D80043F002032361C4F81480236943F0400302
:1008E800236121F071FE2369042823F002032361A8
:1008F800BDD0E5E7236923F001032361D9E7336815
:1009080004333360DEE700BF00200240F8B5044638
:100918000D468E180027B54201D12069F8BDE3685D
:10092800591CE160234415F8012B1A720429F2D1ED
:10093800A1682046FFF790FFE7602061EBE700BF62
:1009480070B582B004466946143029F0A9FAB0B1EE
:100958009DF805009DF801609DF802109DF8035070
:100968009DF804209DF8063041EA062143EA002359
:1009780042EA0522A187E287A4F84030012002B0AC
:1009880070BD00BF10B490E80600047B40690223E4
:10099800A3404B6013685DF8044B4FF6FE710B40A3
:1009A80013600BF09FB800BF03689B69184700BF2E
:1009B80003685B69184700BF0368DB68184700BF16
:1009C80003689B68184700BF03685B68184700BF47
:1009D80003682DE9F041DF691FB13B46BDE8F041EE
:1009E8001847002A164611DD04460D460E4400E05D
:1009F80023689B68204698470028F9D0236815F893
:100A0800011B1B6820469847AE42F1D1BDE8F08132
:100A180003681B68184700BF014B1868F8E700BF58
:100A2800A86D0020054B53F8203033B11A689B8815
:100A3800918A0B4218BF1B0493617047A06F002076
:100A480003682DE9F04F03F13845644EAD0A0124DF
:100A5800755D05F01F066D09022D04FA06F400F015
:100A6800A280032D00F0A480012D52D08088B0FA16
:100A780080F4C4F11F04A4B2E50803EB850504F073
:100A880007042E6AA4000F27A74026EA07062E624D
:100A98002E6A01F0030702FA04F47A1E3443012A8D
:100AA800C1F3810CC1F300182C62C1F3411135D98F
:100AB800C60700F19780850700F1A380440700F17D
:100AC800B180020700F1BF80C60600F1CD8085061F
:100AD80000F1DB80440600F1E980020600F1F780AE
:100AE800C60500F10581850500F11381440500F173
:100AF8002181020500F12F81C60400F13D818504A2
:100B080000F14B81440400F15981020455D4BDE839
:100B1800F08F334D6E6934436C61A7E70024224699
:100B28004FF0010E4FF0030904E00132102A04F1DE
:100B38000204ECD00EFA02F636EA0005F5D1D3F835
:100B480008A009FA04F5ED430AEA050AC3F808A063
:100B5800D3F808B00CFA04FA4AEA0B0AC3F808A05A
:100B6800B3F804A01FFA8AFA2AEA06069E80B3F8A8
:100B780004A008FA02F646EA0A06B6B29E801E6883
:100B88002E401E60D3F800A007FA04F646EA0A06CB
:100B98001E60D3F80CA001FA04F605EA0A0A46EA30
:100BA8000A05DD60C1E70E4DAE693443AC615DE70F
:100BB8000B4DEE693443EC6158E71A6822F0404265
:100BC8001A601A6842EA87771F60DA6822F04042A2
:100BD80042EA8171D960BDE8F08F00BF340503088F
:100BE800001002401A6822F003021A601A683A4399
:100BF8001A60DA6822F003020A438507DA607FF593
:100C08005DAF1A6822F00C021A601A6842EA87027D
:100C18001A60DA6822F00C0242EA81024407DA60BC
:100C28007FF54FAF1A6822F030021A601A6842EA5C
:100C380007121A60DA6822F0300242EA0112DA601A
:100C480002077FF541AF1A6822F0C0021A601A68DD
:100C580042EA87121A60DA6822F0C00242EA811278
:100C6800C606DA607FF533AF1A6822F440721A605C
:100C78001A6842EA07221A60DA6822F4407242EAE5
:100C880001228506DA607FF525AF1A6822F44062F2
:100C98001A601A6842EA87221A60DA6822F4406207
:100CA80042EA81224406DA607FF517AF1A6822F417
:100CB80040521A601A6842EA07321A60DA6822F467
:100CC800405242EA0132DA6002067FF509AF1A683B
:100CD80022F440421A601A6842EA87321A60DA68D7
:100CE80022F4404242EA8132C605DA607FF5FBAE63
:100CF8001A6822F440321A601A6842EA07421A60F7
:100D0800DA6822F4403242EA01428505DA607FF56A
:100D1800EDAE1A6822F440221A601A6842EA874245
:100D28001A60DA6822F4402242EA81424405DA6015
:100D38007FF5DFAE1A6822F440121A601A6842EA98
:100D480007521A60DA6822F4401242EA0152DA6065
:100D580002057FF5D1AE1A6822F440021A601A68BB
:100D680042EA87521A60DA6822F4400242EA815263
:100D7800C604DA607FF5C3AE1A6822F040721A60C2
:100D88001A6842EA07621A60DA6822F0407242EA98
:100D980001628504DA607FF5B5AE1A6822F0406218
:100DA8001A601A6842EA87621A60DA6822F04062BA
:100DB80042EA81624404DA607FF5A7AE1A6822F03D
:100DC80040521A601A6842EA07721A60DA6822F01A
:100DD800405242EA0172DA6097E600BF036803F105
:100DE80038422DE9F04F920A584DAA5C02F01F05CF
:100DF80052090124022A04FA05F400F08C80032A1F
:100E080000F08E80012A3CD001F003077A1E012AE7
:100E1800C1F3810CC1F300188088C1F3411135D9A1
:100E2800C60700F19780850700F1A380440700F109
:100E3800B180020700F1BF80C60600F1CD808506AB
:100E480000F1DB80440600F1E980020600F1F7803A
:100E5800C60500F10581850500F11381440500F1FF
:100E68002181020500F12F81C60400F13D8185042E
:100E780000F14B81440400F15981020455D4BDE8C6
:100E8800F08F334A55692C435461BDE7002422464C
:100E98004FF0010E4FF0030904E00132102A04F16B
:100EA8000204ECD00EFA02F636EA0005F5D1D3F8C2
:100EB80008A009FA04F5ED430AEA050AC3F808A0F0
:100EC800D3F808B00CFA04FA4AEA0B0AC3F808A0E7
:100ED800B3F804A01FFA8AFA2AEA06069E80B3F835
:100EE80004A008FA02F646EA0A06B6B29E801E6810
:100EF8002E401E60D3F800A007FA04F646EA0A0658
:100F08001E60D3F80CA001FA04F605EA0A0A46EABC
:100F18000A05DD60C1E70E4A95692C43946173E7C1
:100F28000B4AD5692C43D4616EE71A6822F0404217
:100F38001A601A6842EA87771F60DA6822F040422E
:100F480042EA8171D960BDE8F08F00BF340503081B
:100F5800001002401A6822F003021A601A683A4325
:100F68001A60DA6822F003020A438507DA607FF51F
:100F78005DAF1A6822F00C021A601A6842EA87020A
:100F88001A60DA6822F00C0242EA81024407DA6049
:100F98007FF54FAF1A6822F030021A601A6842EAE9
:100FA80007121A60DA6822F0300242EA0112DA60A7
:100FB80002077FF541AF1A6822F0C0021A601A686A
:100FC80042EA87121A60DA6822F0C00242EA811205
:100FD800C606DA607FF533AF1A6822F440721A60E9
:100FE8001A6842EA07221A60DA6822F4407242EA72
:100FF80001228506DA607FF525AF1A6822F440627F
:101008001A601A6842EA87221A60DA6822F4406293
:1010180042EA81224406DA607FF517AF1A6822F4A3
:1010280040521A601A6842EA07321A60DA6822F4F3
:10103800405242EA0132DA6002067FF509AF1A68C7
:1010480022F440421A601A6842EA87321A60DA6863
:1010580022F4404242EA8132C605DA607FF5FBAEEF
:101068001A6822F440321A601A6842EA07421A6083
:10107800DA6822F4403242EA01428505DA607FF5F7
:10108800EDAE1A6822F440221A601A6842EA8742D2
:101098001A60DA6822F4402242EA81424405DA60A2
:1010A8007FF5DFAE1A6822F440121A601A6842EA25
:1010B80007521A60DA6822F4401242EA0152DA60F2
:1010C80002057FF5D1AE1A6822F440021A601A6848
:1010D80042EA87521A60DA6822F4400242EA8152F0
:1010E800C604DA607FF5C3AE1A6822F040721A604F
:1010F8001A6842EA07621A60DA6822F0407242EA25
:1011080001628504DA607FF5B5AE1A6822F04062A4
:101118001A601A6842EA87621A60DA6822F0406246
:1011280042EA81624404DA607FF5A7AE1A6822F0C9
:1011380040521A601A6842EA07721A60DA6822F0A6
:10114800405242EA0172DA6097E600BF10B504091E
:10115800013C052C17D80D4B33F8142000F00F0074
:1011680042FA00F313F001030DD0012303FA00F053
:10117800013810402AF0C4FB054A064B125D1044A2
:1011880003EBC00010BD002010BD00BFECFE02083C
:10119800F8FE0208FC5E00202DE9F04F4A484B4B50
:1011A8004B4C4FF090414FF0010A4FF002094FF0BD
:1011B80004084FF0080C4FF0100E20274026802519
:1011C80030F8022B12F0010F03D01960A3F804A025
:1011D800083312F0020F03D01960A3F80490083303
:1011E80012F0040F03D01960A3F80480083312F03A
:1011F800080F03D01960A3F804C0083312F0100FC9
:1012080003D01960A3F804E0083312F0200F02D0CD
:1012180019609F80083312F0400F02D019609E8039
:10122800083312F0800F02D019609D80083312F441
:10123800807F05D04FF4807B1960A3F804B0083391
:1012480012F4007F05D04FF4007B1960A3F804B0B6
:10125800083312F4806F05D04FF4806B1960A3F83F
:1012680004B0083312F4006F05D04FF4006B196016
:10127800A3F804B0083312F4805F05D04FF4805B04
:101288001960A3F804B0083312F4005F05D04FF4D6
:10129800005B1960A3F804B0083312F4804F05D03E
:1012A8004FF4804B1960A3F804B00833D20B04D074
:1012B8004FF4004219609A80083301F58061A14219
:1012C8007FF47EAFBDE8F08FECFE0208FC5E0020E4
:1012D80000180048002867D003682DE9F04F03F193
:1012E80038445C4EA40A0125345D04F01F066409E5
:1012F800022C05FA06F558D0032C00F0A580012C25
:1013080058D08088B0FA80F4C4F11F04A4B2E5086C
:1013180003EB850504F007042E6AA4000F27A740F5
:1013280026EA07062E622E6A01F00307A2407C1EF9
:101338003243012CC1F3810CC1F300182A62C1F3B6
:1013480041113CD9C60700F18980850700F19580D5
:10135800440700F1A380020700F1B180C60600F13E
:10136800BF80850600F1CD80440600F1DB800206CF
:1013780000F1E980C60500F1F780850500F10581D7
:10138800440500F11381020500F12181C60400F132
:101398002F81850400F13D81440400F14B81020452
:1013A80000F15981BDE8F08F70472B4CA669354391
:1013B800A561A6E7284C666935436561A1E7002465
:1013C80022464FF0010E4FF0030904E00132102AC3
:1013D80004F10204E6D00EFA02F636EA0005F5D169
:1013E800D3F808A009FA04F5ED430AEA050AC3F898
:1013F80008A0D3F808B00CFA04FA4AEA0B0AC3F8B2
:1014080008A0B3F804A01FFA8AFA2AEA06069E8002
:10141800B3F804A008FA02F646EA0A06B6B29E80B5
:101428001E682E401E60D3F800A007FA04F646EAAC
:101438000A061E60D3F80CA001FA04F605EA0A0AA7
:1014480046EA0A05DD60C1E7034CE6693543E56114
:1014580057E700BF34050308001002401A6822F05D
:1014680003021A601A683A431A60DA6822F0030223
:101478000A438507DA607FF56BAF1A6822F00C0221
:101488001A601A6842EA87021A60DA6822F00C02C7
:1014980042EA81024407DA607FF55DAF1A6822F0FC
:1014A80030021A601A6842EA07121A60DA6822F0F3
:1014B800300242EA0112DA6002077FF54FAF1A687C
:1014C80022F0C0021A601A6842EA87121A60DA68C3
:1014D80022F0C00242EA8112C606DA607FF541AF07
:1014E8001A6822F440721A601A6842EA07221A60DF
:1014F800DA6822F4407242EA01228506DA607FF552
:1015080033AF1A6822F440621A601A6842EA8722E6
:101518001A60DA6822F4406242EA81224406DA60FC
:101528007FF525AF1A6822F440521A601A6842EA19
:1015380007321A60DA6822F4405242EA0132DA606D
:1015480002067FF517AF1A6822F440421A601A683B
:1015580042EA87321A60DA6822F4404242EA81326B
:10156800C605DA607FF509AF1A6822F440321A60BE
:101578001A6842EA07421A60DA6822F4403242EAFC
:1015880001428505DA607FF5FBAE1A6822F4402235
:101598001A601A6842EA87421A60DA6822F440221E
:1015A80042EA81424405DA607FF5EDAE1A6822F41A
:1015B80040121A601A6842EA07521A60DA6822F47E
:1015C800401242EA0152DA6002057FF5DFAE1A687E
:1015D80022F440021A601A6842EA87521A60DA68EE
:1015E80022F4400242EA8152C604DA607FF5D1AEA5
:1015F8001A6822F040721A601A6842EA07621A6092
:10160800DA6822F0407242EA01628504DA607FF506
:10161800C3AE1A6822F040621A601A6842EA87620A
:101628001A60DA6822F0406242EA81624404DA60B1
:101638007FF5B5AE1A6822F040521A601A6842EA7D
:1016480007721A60DA6822F0405242EA0172DA60E0
:1016580002047FF5A7AE1A6822F040421A601A68A1
:1016680042EA87771F60DA6822F0404242EA8171D5
:10167800D960BDE8F08F00BF002852D0036803F19D
:1016880038422DE9F04F920A504DAA5C02F01F052E
:1016980052090124022A04FA05F443D0032A00F06F
:1016A8009080012A43D001F003077A1E012AC1F372
:1016B800810CC1F300188088C1F341113CD9C607D9
:1016C80000F18880850700F19480440700F1A2802A
:1016D800020700F1B080C60600F1BE80850600F161
:1016E800CC80440600F1DA80020600F1E880C605E5
:1016F80000F1F680850500F10481440500F11281AE
:10170800020500F12081C60400F12E81850400F154
:101718003C81440400F14A81020400F15881BDE88B
:10172800F08F70472A4A95692C439461BBE7284A91
:1017380055692C435461B6E7002422464FF0010E48
:101748004FF0030904E00132102A04F10204E6D044
:101758000EFA02F636EA0005F5D1D3F808A009FA20
:1017680004F5ED430AEA050AC3F808A0D3F808B05F
:101778000CFA04FA4AEA0B0AC3F808A0B3F804A062
:101788001FFA8AFA2AEA06069E80B3F804A008FA25
:1017980002F646EA0A06B6B29E801E682E401E6011
:1017A800D3F800A007FA04F646EA0A061E60D3F842
:1017B8000CA001FA04F605EA0A0A46EA0A05DD6001
:1017C800C1E7034AD5692C43D4616CE734050308A3
:1017D800001002401A6822F003021A601A683A439D
:1017E8001A60DA6822F003020A438507DA607FF597
:1017F8006CAF1A6822F00C021A601A6842EA870273
:101808001A60DA6822F00C0242EA81024407DA60C0
:101818007FF55EAF1A6822F030021A601A6842EA51
:1018280007121A60DA6822F0300242EA0112DA601E
:1018380002077FF550AF1A6822F0C0021A601A68D2
:1018480042EA87121A60DA6822F0C00242EA81127C
:10185800C606DA607FF542AF1A6822F440721A6051
:101868001A6842EA07221A60DA6822F4407242EAE9
:1018780001228506DA607FF534AF1A6822F44062E7
:101888001A601A6842EA87221A60DA6822F440620B
:1018980042EA81224406DA607FF526AF1A6822F40C
:1018A80040521A601A6842EA07321A60DA6822F46B
:1018B800405242EA0132DA6002067FF518AF1A6830
:1018C80022F440421A601A6842EA87321A60DA68DB
:1018D80022F4404242EA8132C605DA607FF50AAF57
:1018E8001A6822F440321A601A6842EA07421A60FB
:1018F800DA6822F4403242EA01428505DA607FF56F
:10190800FCAE1A6822F440221A601A6842EA87423A
:101918001A60DA6822F4402242EA81424405DA6019
:101928007FF5EEAE1A6822F440121A601A6842EA8D
:1019380007521A60DA6822F4401242EA0152DA6069
:1019480002057FF5E0AE1A6822F440021A601A68B0
:1019580042EA87521A60DA6822F4400242EA815267
:10196800C604DA607FF5D2AE1A6822F040721A60B7
:101978001A6842EA07621A60DA6822F0407242EA9C
:1019880001628504DA607FF5C4AE1A6822F040620D
:101998001A601A6842EA87621A60DA6822F04062BE
:1019A80042EA81624404DA607FF5B6AE1A6822F032
:1019B80040521A601A6842EA07721A60DA6822F01E
:1019C800405242EA0172DA6002047FF5A8AE1A6852
:1019D80022F040421A601A6842EA87771F60DA6884
:1019E80022F0404242EA8171D960BDE8F08F00BF21
:1019F800F0B5044690F8590083B0002840F0C28042
:101A0800764E377A002F4FD004F11405A06929F0DB
:101A1800BFF894F852201A212846FEF739FC012015
:101A280009F068FEA269E66D138823F040031B04E1
:101A38001B0C1380138823F038031B041B0C138022
:101A480013889BB243F040031380284606236A4656
:101A58004321B047D8B19DF802609DF803309DF846
:101A680000509DF801109DF804009DF8052043EAF8
:101A780006231BB2E3875BB241EA052142EA002252
:101A88000133A187A4F8402006D003B0F0BDB4F913
:101A98003E305BB20133F8D194F93C300133F4D1D4
:101AA800062008F02DFDF0E704F11405A06929F0DF
:101AB8006FF880226B212846FEF7EAFB962009F092
:101AC80073FE032268212846FEF7E2FB962009F000
:101AD8006BFE03226B212846FEF7DAFB0F2009F084
:101AE80009FE10226A212846FEF7D2FB0F2009F0D2
:101AF80001FE3A466C212846FEF7CAFB0F2009F082
:101B0800F9FD94F8542019212846FEF7C1FB0F204F
:101B180009F0F0FD18221B212846FEF7B9FB0F201B
:101B280009F0E8FD10221C212846FEF7B1FB0F2022
:101B380009F0E0FD102237212846FEF7A9FB0F2007
:101B480009F0D8FD012238212846FEF7A1FB0F2015
:101B580009F0D0FDA269138823F040031B041B0C75
:101B68001380138823F038031B041B0C138013887D
:101B78009BB243F040031380012009F0BBFD012311
:101B8800337243E7FFF7E2FA0546D8B12023002174
:101B98008371C171FFF770FD2146114B41F8103F69
:101BA800284628F01DF9AB88B3FA83F3C3F11F0365
:101BB8005A1C3FF425AF01229A400A490B68134387
:101BC8000B601DE70146FFF757FD2146044B41F81E
:101BD800103F284628F004F90122EEE7A01D002056
:101BE800650700080004014010B1036882881A855F
:101BF800704700BF10B1036882889A61704700BFC0
:101C080038B100298388026814BF002110218B4055
:101C18009361704710B40A4B0A4A1C780123834029
:101C2800234052F8200029B9B3FA83F149095DF835
:101C3800044BE5E7191C18BF01215DF8044BDFE7E9
:101C48009F6F0020A06F002030B1036882881B8A34
:101C58001A4214BF01200020704700BF2DE9F0414F
:101C68000B4E346873691C400FD0DFF828800127B9
:101C7800B4FA84F3C3F11F0307FA03F558F82300F5
:101C880003689847AC437561F2D1BDE8F08100BFA5
:101C980000040140586F00202DE9F0410B4E3468D4
:101CA80073691C400FD0DFF828800127B4FA84F349
:101CB800C3F11F0307FA03F558F823000368984790
:101CC800AC437561F2D1BDE8F08100BF000401406A
:101CD800586F00202DE9F0410B4E346873691C40A1
:101CE8000FD0DFF828800127B4FA84F3C3F11F036B
:101CF80007FA03F558F8230003689847AC43756161
:101D0800F2D1BDE8F08100BF00040140586F002007
:101D18002DE9F0410B4E346873691C400FD0DFF891
:101D280028800127B4FA84F3C3F11F0307FA03F5E7
:101D380058F8230003689847AC437561F2D1BDE8B1
:101D4800F08100BF00040140586F00202DE9F041E8
:101D58000B4E346873691C400FD0DFF828800127C8
:101D6800B4FA84F3C3F11F0307FA03F558F8230004
:101D780003689847AC437561F2D1BDE8F08100BFB4
:101D880000040140586F00202DE9F0410B4E3468E3
:101D980073691C400FD0DFF828800127B4FA84F358
:101DA800C3F11F0307FA03F558F82300036898479F
:101DB800AC437561F2D1BDE8F08100BF0004014079
:101DC800586F00202DE9F0410B4E346873691C40B0
:101DD8000FD0DFF828800127B4FA84F3C3F11F037A
:101DE80007FA03F558F8230003689847AC43756170
:101DF800F2D1BDE8F08100BF00040140586F002017
:101E0800084A094808B5936943F001039361002122
:101E180040222CF022F9054B4FF0FF321A60C3F82C
:101E2800032008BD00100240586F0020986F002062
:101E38002DE9F041044618460D461646984629F005
:101E4800B5F82768E6722844A07229467D6943469A
:101E580032462046AC46BDE8F0416047036810B5FD
:101E680004461B689847236820469B689847A37BCD
:101E78000133A37310BD00BF427A02B9704710B591
:101E880004460368406804F10A0198470023637216
:101E980010BD00BF437A5A1C0344D2B242729972F1
:101EA800037A934200D802B9704710B50446036814
:101EB800406804F10A0198470023637210BD00BF0F
:101EC80030B40B4D002305F11C0101E0272B0BD08A
:101ED80011F8132082424FEA430403F10103F5D1BC
:101EE8002C44607F30BC7047002030BC704700BF76
:101EF800CCE1020870B5448806460D46C4F30B04CD
:101F08002246002128462CF0A8F83369094A934252
:101F180009D3094A934206D2224628461946BDE803
:101F2800704029F01BBE23B121462846BDE8704009
:101F3800184770BD703B03085B3C0308064B074914
:101F48008B4202D30023184670471A88C2F30B024B
:101F58009042F8D01433F3E760370308703B030866
:101F6800024A136823EA000010607047E84C00201A
:101F7800F8B5174D2B78A42B28D16B78BE2B25D11B
:101F8800022229464FF6FF70FEF720FB114FAC1CCA
:101F980022884AB1A618BE4218D2052A16D9214667
:101FA800FEF714FB3446F3E721460222FEF70EFB48
:101FB8000222A118FEF70AFB0634074B641B1C809B
:101FC80041F60F53C31A58425841F8BD0020F8BDD6
:101FD80000F00308000004082C3600202DE9F04F1B
:101FE800DFF864914F4F8BB00326A7EB090718223F
:101FF800002104A82CF031F84B4BCDF81090059730
:102008001A69120604D5494A5A6002F188325A60A0
:1020180001228DF824203422DA60454B454C1B8878
:10202800ADF800300222694604A8FEF76FFC0222D0
:1020380069464FF6FF70FEF7C9FADFF810A180462F
:102048004FF0000B544536D30AAC002524F8245D24
:102058000222214604A8FEF759FC022221464046E6
:10206800FEF7B4FA40BAC043ADF80800022202A94C
:1020780004A8FEF74BFC079860B106ABC0F1040258
:10208800294618442BF0E9FF069904A8FEF7E4FB5B
:10209800079508909DF82430089A23B122490B69C6
:1020A80043F080030B61013E2DD0002A9FD1FFF73A
:1020B8005FFF50B332E065888DF80DB0C5F30B05AE
:1020C800AB1DADF808302388C3F30B02ADF80A2026
:1020D8001B0B062202A904A88DF80C30FEF716FC8B
:1020E800062202A94046FEF771FA616880462A4630
:1020F80004A8FEF70BFC616840462A46FEF766FA1C
:10210800143480469EE7002AD1D0052023F09AFA9D
:10211800094B0A4A1A600A4B0A4ADA600BB0BDE852
:10212800F08F00BF0000040800200240230167452B
:1021380036E2020860370308FC9F0020EFBEADDEE0
:1021480000ED00E00400FA0500F00308703B030806
:102158000378202B024600F10100F9D0092BF7D0B3
:102168002D2B2CD02B2B03BF5378B7EE000A024639
:10217800B7EE000AA3F13001C8B209289FED467AEC
:1021880010D8F2EE046A07EE901AF8EEE77A12F821
:10219800013FE7EE267AA3F13001C8B20928B0EE74
:1021A800677AF0D92E2B4CD003F0DF03452B0BD0E8
:1021B800F7EE007A67EE276A20EE260A7047537812
:1021C800BFEE000A0246D5E710B451782D2959D040
:1021D8002B290ABF9178501C901C0024A1F13003D0
:1021E800092B53D8002303EB830301EB430310F8B7
:1021F800011FA1F13002092AA3F13003F3D9B3F585
:102208009A7F28BF4FF49A73072B42D9DFED236AD0
:102218001A46F7EE007A083A072A67EEA67AFAD83D
:1022280003F007032BB1F2EE046A013B67EEA67ACE
:10223800FBD124B3C7EE276A5DF8044B20EE260ACB
:1022480070475378A3F13001C8B2092802F101029E
:10225800AAD8F2EE046AF0EE665A07EE901AF8EE83
:10226800E77A12F8013F87EEA66AA3F13001C8B2F7
:10227800092866EEA56A37EE067AEED994E767EE86
:10228800276AD9E7901C91780124A7E7F7EE007A2E
:10229800CFE7F7EE007AC5E70000000020BCBE4C8F
:1022A800B5EEC00ADFED317AF1EE10FACCBF30EEB0
:1022B800270A30EE670ADFED2E7A20EE270A30B5BE
:1022C800FDEEC07A87B017EE904A054684EAE470BE
:1022D800002303A9A0EBE47001930093029324F078
:1022E80025FD002CACBF20232D2303A88DF800303A
:1022F80028F05CFE012803A924D002282DD0032849
:1023080005BF3023684668468DF801302BF0CBFEB8
:10231800684628F04BFE0338C4B222466946284670
:102328002BF01FFF00232B55284628F03FFE2E22B6
:10233800431C2A540DEB0401E8182BF0D1FE284663
:1023480007B030BD302368468DF801308DF8023073
:102358008DF803302BF0A7FEDAE7302368468DF8B6
:1023680001308DF802302BF09EFED1E76F12033A50
:1023780000007A442DE9F041064615460846B6FBAA
:10238800F2F43CB905FB1464124B1B5D00F8013BE9
:10239800BDE8F081B4FBF2F767B90E4B05FB1747B0
:1023A80005FB1464DA5D00F8012B1B5D00F8013BA6
:1023B800BDE8F081B7FBF2F8B8F1000F02D0404653
:1023C800FFF7D8FF05FB1878024B13F8082000F830
:1023D800012BE3E70406030830B402681146531CD6
:1023E800036011F8024B0160D31C517803609378A5
:1023F800151D05601B0443EA0123D078234343EAF3
:10240800006030BC704700BF0368591C1A46016061
:1024180012F8021B0260587841EA0020704700BF9A
:1024280003685A1C02601878704700BF38B5044624
:102438000068154629F092FB22682A44226038BDBC
:10244800036810B40A0A5C1C04601A7003685A1CFA
:10245800026019705DF8044B704700BF03685A1C8E
:10246800026010B4197003680A0A5C1C04601A70D0
:1024780003680A0C5C1C04601A700368090E5A1C75
:10248800026019705DF8044B704700BF03685A1C5E
:10249800026019700368090A5A1C026019707047B3
:1024A8002DE9F047002488B080460F461E46A14615
:1024B80005AD531C0393117839B3252933D1931CE7
:1024C800CDF810900393507830284ED04FF0000A82
:1024D800A0F13003DBB2092B42D96C2819D064284B
:1024E80000F0938024D825281CD063D9582876D0AA
:1024F80063281BD131784046B847039A531C03938D
:102508001178043601340029D7D1204608B0BDE837
:10251800F087039B5A1C03921B78642B7CD02AD823
:10252800252B54D1252140460134B847039AC0E7EA
:10253800732833D044D975284FD106F1040E30687A
:102548002B4600220A217646FDF736FF049A0095AD
:10255800534639464046FDF76DFF039A0444A8E701
:1025680004AA03A924F0BEFBB7E7D31C0393907811
:102578004FF0010AACE7732B10D05BD9752B3AD01A
:10258800782B96D1A3F15802B2FA82F23068520938
:102598002B4610210436FDF70FFFD7E73368049A5E
:1025A8000093394600234046FDF744FF04360444AF
:1025B800039A7EE70028B9D1204608B0BDE8F08725
:1025C8006E28B3D1039A336804361C6071E72AD9A0
:1025D800582BD7D0632B8DD06BE77828A6D1A0F1E4
:1025E8005802B2FA82F2306852092B461021FDF7E0
:1025F800E3FE0436AAE706F1040E30682B460022F3
:102608000A217646FDF7D8FEA0E7331D3068294633
:102618001E46FDF7A3FE99E7331D306829461E467E
:10262800FDF79CFE92E7002B7FF443AF204608B0ED
:10263800BDE8F0876E2BC6D03BE700BF0EB400B5EF
:1026480084B005AB019053F8042B0649039301A805
:10265800FFF726FF019B00221A7004B05DF804EB17
:1026680003B07047310400080FB430B583B006AB2F
:102678000A490B4853F8042B096800680193FFF7CF
:102688000FFF084C05462068FEF792F90028FAD09B
:10269800284603B0BDE8304004B07047AC35002090
:1026A800B0350020A86D0020DFED2B7AB4EEE70AE4
:1026B800F1EE10FA4ADDDFED296A9FED297A01E093
:1026C800B0EE670AB4EEC70AF1EE10FA70EE667A59
:1026D800F6DC9FED247AF4EEC77AF1EE10FA38D5DD
:1026E800DFED1E6A9FED207A01E0F0EE407AF4EE0D
:1026F800C77AF1EE10FA37EEA60AF6D4DFED1B7AA8
:10270800B4EEE70AF1EE10FA14DDDFED137A37EED6
:10271800C00A60EE006A9FED166A9FED167ADFED3B
:10272800167AA6EE867A20EE266AE6EE877AA6EE76
:10273800270A7047DFED117AB4EEE70AF1EE10FAD6
:1027480044BFDFED087A37EEC00AE2E7F0EE407AE0
:10275800BFE7B0EE670AD1E7DB0F4940DB0FC9409E
:10276800E4CB1641DB0F49C0E4CB16C1DB0FC93FF0
:1027780092E741B99730083C15A82ABEDB0FC9BFBC
:1027880009B909E0194690FBF1F301FB1303084668
:10279800002BF7D1084670470146FBE710B507EE56
:1027A800901A2DED028BB8EE678ADFED217A28EEBC
:1027B800008A044628EE278AB0EE480A29F08EFBE4
:1027C800F0EE408AB0EE480A29F0EAFAF7EE007A0D
:1027D8009FED187AF0EE675AE8EE875A0023A36156
:1027E800B0EE676AC7EEA56A63612362E361A8EE8B
:1027F800C76ABDEC028B77EEC07AB6EE007AF8EEC7
:10280800005A27EE877A20EE250A27EE267A26EE4A
:10281800266A67EEA67A20EE260A84ED046AC4EDDD
:10282800017A84ED007A84ED027A84ED030A10BD02
:1028380027D4D236F304353F10B44C09012250F89E
:10284800243001F01F0102FA01F10B4340F8243053
:102858005DF8044B704700BF4B0901F01F0150F8A9
:102868002320012303FA01F1114214BF1846002066
:10287800704700BFF0B55B4B5B4A97B0196891424F
:1028880000AF00F0A3805949594A00234FF4700063
:10289800C1F888003B607B60136843F480331360A1
:1028A80003E03B68B3F5A04F09D0136803F4003385
:1028B8007B603B6801333B607B68002BF1D04C4B5D
:1028C8001B6813F4003318BF01237B607B68012B5E
:1028D80052D0464C464B474AE260474A596A116013
:1028E8005A6A42F080725A625A6942F4FC025A618A
:1028F8000025032207F10801012341F6FF764FF076
:102908009040FD60BE603A73BB7322F0C1FB4FF686
:10291800FF7307F108013948BB6022F0B9FB07F1E2
:1029280008013748374E22F0B3FB07F10801364853
:1029380022F0AEFB07F10801344822F0A9FB07F1A9
:102948000801334822F0A4FB07F1080022F0FAFB43
:10295800BB683049304AA1FB031330499B0CF02077
:102968004FF0070E5C370B60566084F823009560C3
:10297800C2F800E0BD46F0BD294A1D4B1221116086
:102988005A685A605A685A605A6842F480625A60B3
:102998005A6822F47C125A605A6842F4E8125A6063
:1029A8001A6842F080721A601A689201FCD5596858
:1029B8000F4A21F003015960596841F0020159603A
:1029C800536803F00C03082BFAD182E700221A603F
:1029D80062B6144B1B6883F30888134B1B6898472F
:1029E800FEE700BFFC9F0020EFBEADDE00ED00E07B
:1029F800001002400005FA05D860002000040048D5
:102A0800000800483F190100000C00480010004869
:102A18000014004883DE1B4310E000E0D86F00205C
:102A28000020024000D8FF1F04D8FF1F70B50F4CCC
:102A38000F4DC0EBC00004EB800468692669304381
:102A4800686182B09209667BA1600025012101A816
:102A580063618DF804608DF805208DF806508DF8B7
:102A6800071022F009FA02B070BD00BF7C1A0020DE
:102A780000100240074BC0EBC00030B403EB8000ED
:102A8800054C056963692B4363610176427630BC66
:102A9800704700BF7C1A0020001002402DE9F04169
:102AA800854BDD7A94B045B11B78022B0BD0032BF4
:102AB80000F0EA80012B00F0D480804B00221A70CD
:102AC80014B0BDE8F0817E4C7E4BC4F8E432002699
:102AD8004FF41B7318224AF29E37626004F1140007
:102AE80031461A46A760267023612BF0B6FA2846AD
:102AF80027F07CFF744FC36802683A600646002BD3
:102B080000F0A9802846FEF721FB704B186018B129
:102B1800292200238271C371327A4E21FEF7DAFB33
:102B280000222921307CFFF7A5FF0023C022684935
:102B3800307CFFF77BFF386808F020FC27F0EAFCC0
:102B4800A188644A644B386802FB01F29A4240F358
:102B5800AB80002314A9002521F84C3D5E4AADF84E
:102B68000C500133B2FBF3F3A268B3FBF2F3C3F3E7
:102B78004E029BB2A2810293ADF80650ADF80E50FA
:102B880027F0E2FEADF816500695ADF81C50ADF8EA
:102B98001E50ADF82050ADF82250F379ADF814501E
:102BA800602204925A077BD401214FF48072ADF859
:102BB8001410ADF82020002503F00203ADF81C30F6
:102BC800069504AA71793868DFF8248108F044F87A
:102BD8007179386827F098FE3A68F068536CC8F83D
:102BE800000043F40043536403684FF6FE72134039
:102BF800036022F0B9F909A822F088F93B687279D4
:102C08002169ADF83010343313440993102280231E
:102C180009A90B920E934FF480724FF40053D8F821
:102C280000002E4C13950D95109511950F92129347
:102C38000A9422F079F972793B680C2A9CBF2849DA
:102C480031F81250D968D8F800200D43DD601368B8
:102C580043F002031360194B01221A7022F03AFF65
:102C68002EE7174C1F4923701F4EC4F8E4124FF487
:102C78003473182704F114001A4600216760A6600F
:102C880023612BF0EAF932E70D4C184BC4F8E43213
:102C9800C823122749F2704604F114001A46ECE7DB
:102CA8000422ADF8162086E703EB5203B3FBF2F3D8
:102CB800013B9BB24EE700BF345A0020F835002094
:102CC800405A002038E20208C4230020C82300200C
:102CD8002D07000840420F0000A24A04545A002061
:102CE80078FD02083CE20208CE07070040E202082D
:102CF800C02300202DE9F04F5E4C54F8204083B0EB
:102D0800002C71D0666D984691465B4B7268E26400
:102D1800A160236004F15A014FF4807304F5AD7289
:102D28006161A261E36023610746307E27F0F2FB10
:102D3800F068A8B1514B00215A68904203F11C0376
:102D480000F0928001310C29F6D100207A1CD2B211
:102D58000C21FFF78FFEE36CF26822632433A3642F
:102D6800B068D8B1454B00215A68904203F11C0362
:102D780078D001310C29F7D100257A1CD2B20B2169
:102D88002846FFF777FE2346F27E3D492846FFF79F
:102D98004DFEE36CB26862632833636494F85900AB
:102DA800FEF7D4F9054694F85800FEF7CFF918F065
:102DB800080F824696F819B01AD0CDB118F0110F45
:102DC8004FF00B0307F1010714BF4E213E21EF71AD
:102DD8005A46AB712846FEF77DFA18F0010F45D028
:102DE800236B5BB3636B4BB3204603B0BDE8F08F36
:102DF80018F0010F0CBF4FF02E084FF04E0819F0D5
:102E0800020F09D045B10B227B1CAA71EB71284631
:102E18005A464146FEF75EFA19F0010FE0D0BAF1C2
:102E2800000FDDD001370C238AF807705A46414657
:102E38008AF806305046FEF74DFAD1E7337FB27E66
:102E48008DF804209B090021012201A88DF8053086
:102E58008DF806108DF8072022F00EF8204603B0F2
:102E6800BDE8F08FCDB288E7C8B26FE72846FEF715
:102E7800BBFEB5E7B835002044E202087C1A002002
:102E88008D0900080348D0F83C3113B100F59A7059
:102E9800184770477C1A00200348D0F8203113B136
:102EA80000F58C70184770477C1A00200348D0F84A
:102EB80004310BB1FC301847704700BF7C1A002062
:102EC8000348D0F8E8300BB1E0301847704700BF2E
:102ED8007C1A00200348D0F8CC300BB1C430184716
:102EE800704700BF7C1A00200348D0F8B0300BB1FF
:102EF800A8301847704700BF7C1A00200348D0F854
:102F080094300BB18C301847704700BF7C1A0020F2
:102F18000248836F0BB17030184770477C1A002045
:102F28000248C36D0BB15430184770477C1A002013
:102F38000248036C0BB13830184770477C1A0020E0
:102F48000248436A0BB11C30184770477C1A0020AE
:102F58000248836803B11847704700BF7C1A0020F5
:102F68001749184B184A194810B4D1F8884044F446
:102F78007004C1F888401C6844F001041C605C6857
:102F880022405A601A6822F0847222F480321A6051
:102F98001A6822F480221A605A6822F4FE025A60E3
:102FA800DA6A22F00F02DA621A6B002410404FF03E
:102FB800006218639C608A605DF8044B704700BF2C
:102FC80000ED00E0001002400CC07FF8CCFC00FFD0
:102FD8002DE9F04F2DED028B93B0834615F0E4FEFA
:102FE800B44B1D7825B113B0BDEC028BBDE8F08F52
:102FF800B14B1B685C05F6D5B04FB14E3B68002B52
:1030080056D0B04C3168D4F810218A1A7C2A4FD98E
:1030180094F81421DFF800839FEDAB8AC4F81011EF
:10302800013284F814214FF0240A5E209847504654
:103038003B689847A54BF8EC016A9B8A07EE103A63
:10304800F8EEE66AB8EEC77A0AF1010AC6EE877AA0
:103058005FFA8AFA67EE887AFDEEE77ACDED027AB2
:10306800BDF908905FFA89F01BF0E6F9C9F307206B
:103078001BF0E2F9BAF1270F3B68D6D15E209847DA
:103088003B683020984700201BF0D6F900201BF041
:10309800D3F93B685E20984794F8143113F003087D
:1030A80000F07481580700F0E987282B01F02B8382
:1030B800874B1B78002B6ED0824C864AD4F8183187
:1030C800ABEB0303934200F27E87DFF850A29AF835
:1030D8000090B9F1000F34D1DFF80882D8F8000069
:1030E800FDF772FCC0B201280FD902287A4F41F0CF
:1030F800BD833B78002B41F0CD85D4F82031ABEB74
:103108000303B3F57A6F81F0278774480268002AB1
:1031180041D09AF80030BBB9714BD8F800001B6851
:103128009B781E3B012B4FF0020141F28986043047
:103138001BF0F4F8012200238AF8002084F82C31CF
:1031480027E06648026832B3D4F8283140F6B73130
:10315800ABEB03038B421ED994F82431002B01F00A
:103168008183013BDBB284F82431002B01F0C38258
:1031780012F8011B94F82C71026094F82D3159480B
:10318800CA190133006884F82C2184F82D31FDF721
:103198003FFCC4F828B1544BD6F800801B7843B1E3
:1031A800524F386828B1524B1B78013B012B41F232
:1031B8001280504B1B7863B14F4F3B684BB1414C69
:1031C800D6F80090D4F84431A9EB0303632B00F23E
:1031D8005B86DFF84C8198F80030022B01F05F82A3
:1031E8003D4F97F87430032B00F03287434B1B7820
:1031F80073B1434D2B685BB1324C08F02FFAD4F809
:103208005031029044F61F62C31A934200F21281B1
:103218003C4B1B78002B40F085803B4B1B7843B11F
:10322800284CD4F8A03203F5C333A0339B4580F073
:103238008B86364B1B78002B3FF4D5AE214E344C91
:10324800344D06F2C1272068FDF7BEFB00283FF485
:10325800CAAE2068FDF7B0FB2B7880465A1E33B102
:1032680020682A70FDF7B0FB0028F2D1BBE60322E4
:103278003946781E2AF0D7FE96F8C03296F8C12251
:1032880086F8C38283F47F4383F0FF039B1A1FFAF7
:1032980088F89BB2B8EB132FD5D196F8C222DBB2CF
:1032A8009A42D0D1781E1AF0B5FD2B7818442870B0
:1032B800C9E700BFBD6E00208C510020884800205F
:1032C800D46F0020E41D002000007A44842A0020E6
:1032D800B63900203F0D0300000000208048002080
:1032E8007C48002078480020B8390020F8450020A4
:1032F800C0390020C83900206C690020D03900206E
:10330800D4390020143A0020393A0020DA39002054
:10331800E0390020E4390020BC2A0020844800203D
:10332800BA580020394C2278002A40F0ED85384EF2
:103338003478002C5DD1374D2878002841F0388446
:10334800354C364DD4F898122A78354B93FBF2F366
:103358000B449B45FFF461AF324A94F89C32C4F8A1
:1033680098B2D65CF70701F15886B10701F11286C9
:10337800720701F1AD8594F89C322978013393FBEB
:10338800F1F201FB123384F89C3246E7D4F810219D
:1033980041F288339A4201F239823B685E209847AD
:1033A8003B6814209847204B204AB3F9043082FB2D
:1033B80003124FEAE378C8EBA2080FFA88F85FFA1D
:1033C80088F01BF039F8C8F307201BF035F83B6884
:1033D8005E2098473B681C20984700201BF02CF87B
:1033E80000201BF029F83B685E20984794F81431B8
:1033F80058E60F4D286E002841F0D5818046064BCF
:1034080086F80080C3F898B207E700BFA839002003
:103418001D3A00201C3A0020E41D0020383A002004
:10342800A0860100243A00206C4300206766666687
:10343800403A002094F85631002B41F0AA81DB4B2A
:103448001A6802F00803002B48F603414AF60B40BD
:103458004BF60F4349F6074704BF03460F4612F0E1
:10346800040F4FF0190118BF1F46920684F8561131
:1034780003D547F4804747F02007CD4B5A79C7F367
:103488000909002A41F01B869B79002B41F0108620
:10349800984664204FF0FF3A4FF0000C0A970B97BC
:1034A800ADF834C0CDF83AC0CDF83EC0CDF842C032
:1034B800CDF83090ADF83680ADF838A08DF84600DC
:1034C8000AAF0FCFDFF800E384F805C0AEE80F00BD
:1034D80097E80F00AEE807002EF8023B71464FF060
:1034E800010C1B0CFE271F20C82201F81E39A770EB
:1034F800A27184F807C0E07094F86601207180F02A
:10350800F10383EA0313DAB2130983F0E70343EA0A
:10351800022383EAC2031BB283EA0312D2B2C3F3C3
:10352800072383EA121343EA022383EAC2031BB286
:1035380083F0C80282EA0212D2B2C3F3072383EAF5
:10354800121343EA022383EAC2031BB283EA0C077D
:1035580087EA0717FFB2C3F3072282EA171242EA83
:10356800072200EB0C0382EAC7070EEB0C0084F875
:103578006631278011F8013B7B4083EA0313DBB2F5
:103588001A0982EA172242EA032282EAC3031BB21B
:103598009FB281422780EDD183F07C0383EA031335
:1035A800DBB24FEA131E8EEA172E8EEA032E8EEA3E
:1035B800C30E0FFA8EFE1FFA8EFADFF810C2A4F8B7
:1035C80000A05FFA8EFE4FEA1A2A84F828A084F831
:1035D80027E00CF5C77804F12209DCF80000DCF8D4
:1035E8000410DCF80820DCF80C3047460FC70CF153
:1035F800100CCC45B846F0D1DCF8000038606D4FAF
:103608009CF8043088F8043007F1270884F8B5E1FD
:1036180084F8B6A117F8011F2868FDF7F9F9B8452D
:10362800F8D194F85731002B41F0B88062493268DC
:1036380009780A2084F85701002901F0D8815F4FE2
:1036480001293888069041F25D860229B7F802E020
:1036580001F04F85B8880590032901F04C86F88859
:103668000490042901F063860529388901F05A86F7
:103678000629B7F80A9001F051860729B7F80C8097
:1036880001F04986FB89039394F866110A920B4668
:1036980083F0300282EA0212D2B21709484907932E
:1036A80087F07A0747EA02270988237187EAC20266
:1036B800444FC1EB012187FB013A069B4FF0000CF8
:1036C80063F30F0C059B6EF31F4C4FF0000E63F372
:1036D8000F0E049BCDF82CC012B28A440027C917DC
:1036E80063F31F4EC1EB6A2A039BCDF830E082EAF0
:1036F800021160F30F070020C9B268F30F00C2F38C
:10370800072269F31F4782EA111263F31F404FF043
:1037180000090D978DF83DA00E908DF83C9042EA77
:1037280001220DF1280C82EAC107BCE80F003FB264
:1037380087F0C80888EA0818DFF88CE084F8059054
:103748005FFA88F8C7F30727AEE80F0087EA18176B
:1037580047EA08239CE8030083EAC8031BB283F006
:1037680023024EF8040B82EA0212D2B2C3F30723F3
:10377800079F83EA1213704643EA022383EAC202D0
:1037880007F1010C20F814194FF023081621FE2721
:10379800C82384F866C1228084F807800EF1020EDF
:1037A800A770E170A371114612E000BF203A002013
:1037B800283A0020731F0020203E0020EC3800200B
:1037C8001439002003082080EC1D0020E61D00208D
:1037D80010F8013B4B4083EA0313DBB21A0982EA73
:1037E800112242EA032282EAC3031BB299B270454E
:1037F8002180EDD183F0F40383EA0313DBB24FEAAF
:10380800131E8EEA112E8EEA032E8EEAC30E0FFACD
:103818008EFE1FFA8EF8E64FA4F800804FEA182CA7
:103828005FFA8EFE84F81EE084F81FC07968BA68D3
:103838003868FB6807F5C778A8E80F003869796920
:10384800BA6904F28F17A8E8070004F2AD1884F8E3
:10385800ADC184F8ACE117F8011F2868FDF7D8F866
:10386800B845F8D194F85EC1BCF1000F40F08B87E1
:10387800D04B94F86671B3F90010B3F90220B3F98C
:1038880004309FEDCD6ADFF840E384F805C007EE09
:10389800103A33680A9387F06A0383EA031306EE43
:1038A800901AD9B20B0983F0D50343EA012383EABE
:1038B800C1031BB283EA03115242C9B207EE902A30
:1038C800C3F3072383EA111343EA0123F8EEE77AE7
:1038D800F8EEE66AB8EEC77A83EAC1031BB267EE70
:1038E800867A66EE866A27EE067A002083F0C80894
:1038F800CDED0C7ACDED0B6A8DED0D7A0E900F9013
:10390800109088EA08160DF12809F6B2C3F30728C3
:10391800B9E80F0088EA161848EA062888EAC608AF
:103928000FFA88F8AEE80F0088F01E0699E807003D
:1039380086EA0616F6B2C8F3072383EA161343EAA3
:1039480006238EE8070083EAC6061C20C8214FF02C
:1039580005084FF01E0CFE237A1CE070A17184F854
:103968005E8184F807C0A370AEF1100127710EF1D3
:103978000C00268084F8662111F8013B734083EA25
:103988000313DBB21A0982EA162242EA032282EA08
:10399800C3031BB29EB281422680EDD183F0270378
:1039A80083EA0313DBB24FEA131E8EEA162E8EEA61
:1039B800032E8EEAC30E0FFA8EFE1FFA8EFC7C4F82
:1039C800A4F800C05FFA8EFE4FEA1C2C84F825C0CC
:1039D80084F824E007F5C77804F122093868796883
:1039E800BA68FB6846460FC610374F45B046F5D152
:1039F800724E3B88A8F8003006F1240784F8B2E13B
:103A080084F8B3C116F8011F2868FDF701F8B7421A
:103A1800F8D194F85FA1BAF1000F40F0AE8694F89F
:103A28006681644B664AB3F90410B2F90620654E04
:103A3800DFF898E1644F84F805A088F0220080EA56
:103A48000010C0B2030983F0590343EA002383EA54
:103A5800C0031BB2B2F5FA6F83EA0310C0B2A8BF65
:103A68004FF4FA62C3F30723B2F57A7F83EA10139F
:103A780043EA0023B8BF4FF47A7283EAC000A2F584
:103A88007A72642303FB02F28EFB023ED31786FB95
:103A98000162C9174FF0000CC3EBAE13C1EBA201D2
:103AA800CDF828C006B2CDF82CC0CDF830C0CDF87E
:103AB80034C0ADF83A30ADF838100DF1280CBCE838
:103AC8000F0086F0C80E8EEA0E1E5FFA8EFEC6F351
:103AD800072686EA1E1646EA0E260FC786EACE068F
:103AE80036B286F04A0383EA0313DBB2C6F3072132
:103AF80081EA13113A46DCF800E042F810E941EA9D
:103B0800032108F1010681EAC30305204A214FF089
:103B1800FE0C84F866614FF0C80E142684F85F0125
:103B280084F8048023800437E17184F802C0E670C9
:103B380084F806E0184612F8011B414081EA011199
:103B4800C9B20B0983EA102343EA012383EAC101BE
:103B580009B288B2BA422080EDD181F0140181EA1D
:103B68000111C9B24FEA111E8EEA102E8EEA012EFB
:103B78008EEAC10E0FFA8EFE1FFA8EF60C4F2680C3
:103B88004FEA16295FFA8EFE84F81D9084F81CE02F
:103B980079683868BA68FB68B7F8188007F5C77C91
:103BA800ACE80F0038697969ACE8030010E000BFA1
:103BB800E61D00206C43002088C3E43A731F0020F0
:103BC800EC38002067666666EC1D0020D34D621055
:103BD80004F28F16ACF8008084F8AB91B04684F8F4
:103BE800AAE104F2AB1918F8011F2868FCF710FFC6
:103BF800C145F8D1C94BCA4A1B781278013B12F06B
:103C08000100DBB214BFC0214021172B03D8C54ADD
:103C1800134493F830A0C44B1A8893071ABF0023A3
:103C280041F01001012312F4027F18BF022312F0A1
:103C3800100F18BF062312F0200F18BF10230028FA
:103C480041F07C814FF0030C94F866910A9389F057
:103C5800460383EA0313DAB2130983F0920343EAB3
:103C6800022383EAC2031BB283EA0310C0B2C3F380
:103C7800072282EA101242EA002282EAC00212B245
:103C880082F0C80E8EEA0E1E5FFA8EFEC2F307227D
:103C9800002382EA1E1203208DF82CA08DF82FC075
:103CA8008DF82D3042EA0E2C8DF82E108DF830004C
:103CB8000AAA07CA8CEACE0E0FFA8EFEDFF87CA29B
:103CC800E3718EEA0E1CAAE803005FFA8CFCCEF3BF
:103CD800072E8EEA1C1E4EEA0C2181EACC0C94F8C1
:103CE80008E08AF800200FFA8CFC8EEA0C0E8EEAA7
:103CF8000E1E5FFA8EFECCF3072282EA1E1242EAFB
:103D08000E22607AA17A94F80BC0637182EACE021F
:103D180012B2504080EA001E5FFA8EFEC2F30720FE
:103D280080EA1E1040EA0E2080EACE0000B2414030
:103D380081EA0111C9B2C0F3072282EA111242EAEC
:103D4800012282EAC10212B28CEA020C8CEA0C1C33
:103D58005FFA8CFCC2F3072282EA1C1242EA0C22A8
:103D680094F80CE0607BA17B94F8108084F80490B0
:103D780082EACC0212B28EEA020E8EEA0E1E5FFAB8
:103D88008EFEC2F3072282EA1E1242EA0E2282EA5D
:103D9800CE0212B2504080EA0010C0B2C2F307222D
:103DA80082EA101242EA002282EAC00212B25140AC
:103DB80081EA0111C9B2C2F3072282EA111242EA6A
:103DC800012282EAC102E17B13B281EA030282EA9C
:103DD8000212D2B2C3F3072383EA121343EA02237F
:103DE80083EAC2031BB288EA030282EA0212D2B251
:103DF800C3F3072383EA121343EA022383EAC203C5
:103E08001BB283F0320282EA0212D2B2C3F3072352
:103E180083EA121343EA022383EAC2031BB29AB26B
:103E28004FF0FE0C4FF0090EC82009F10101DBB27A
:103E380084F802C084F803E04FEA122CA07184F8D9
:103E48006611228084F812C0637438687968BA6889
:103E5800B7F80C900AF5C07EAEE807000AF5C87AF4
:103E68008EF80280AEF8009084F8A0C184F89F31E3
:103E780016F8011F2868FCF7CBFDB245F8D1029B64
:103E8800C4F85031FFF7C4B9DFF8B4A0DFF8B48044
:103E980041201AF0F3F9BAF9023088FB0320DB1746
:103EA800C3EBA00080B21AF0CFF9BAF9003088FB52
:103EB8000320DB17C3EBA00080B21AF0C5F9BAF9EA
:103EC800043088FB0320DB17C3EBA00080B21AF094
:103ED800BBF9164B38681978FCF79AFD94F8483105
:103EE80013F0010800F0F084114AC4F8449101333A
:103EF800DBB2A2FB0312D20802EB8202A3EB42035D
:103F080084F84831FFF765B90A4B0B491868FCF784
:103F18005FFD00232370FFF70ABA00BFF42C0020CE
:103F28002E5A00206CE2020816390020A46D0020E9
:103F3800CDCCCCCC183A002068390020EC1D0020EC
:103F48006C4300206766666694F8A432C94AC4F8D0
:103F5800A0B202EB8302926C42B312AD04F2AB231F
:103F6800C54E45F8203D002104F2BD2331800B9356
:103F780080211523A52784F8AA32284684F8A91297
:103F880084F8A872904728463188FEF77FFA0A9D80
:103F9800BA4804F52A716D1A152DA8BF15252A46A9
:103FA80027F0DCFDB64A94F8A4321570B54A0133FF
:103FB80082FB0312A2EBE37202EB42029B1A84F823
:103FC800A432FFF736B9B04AB04B92F80BE031682B
:103FD800D4F81C211B88AE48891A4FF47A72DFB2D4
:103FE80002FB0EF21B0A8777077591424FF0000714
:103FF800C37743758770077180F0F983A54BA6498D
:104008001A689B68C4F818B181FB02E7D21781FBD4
:1040180003E1C2EBA702DB17C3EBA10311124FEABE
:10402800232C4FF0F40E02770127417780F82030D7
:1040380030217522782380F821C080F81AE0C776ED
:1040480080F8221080F8232080F82430FFF73DB84C
:10405800DFF86092D9F80000FCF7AAFC00283FF4CA
:10406800C5A8D9F800000121FCF79EFC0222002314
:1040780087F8742088F80030FFF7B8B83B685E20EE
:1040880098473B6802209847844B834AB3F95030DD
:1040980082FB03124FEAE378C8EBA2080FFA88F80C
:1040A8005FFA88F01AF0C8F9C8F307201AF0C4F9C3
:1040B8003B685E2098473B6803209847784B1B78FD
:1040C800D90740F1BD8316F00DF8764B9FED767A4F
:1040D800D3ED037A67EE877AFCEEE77ACDED027AC4
:1040E800BDF80830002800F0C586D8B24FEA13287A
:1040F8001AF0A2F940461AF09FF9DFF8BC8198F847
:104108000530002B40F086840AA968481AF058F94F
:104118003B685E2098473B6813209847BDF9288084
:104128005FFA88F01AF088F9C8F307201AF084F9C2
:104138003B685E2098473B681B209847BDF92A805A
:104148005FFA88F01AF078F9C8F307201AF074F9C2
:104158003B685E2098473B68232098474E201AF01A
:104168006BF900201AF068F90AA950481AF028F9E2
:104178003B685E2098473B6812209847BDF9288025
:104188005FFA88F01AF058F9C8F307201AF054F9C2
:104198003B685E2098473B681A209847BDF92A80FB
:1041A8005FFA88F01AF048F9C8F307201AF044F9C2
:1041B8003B685E2098473B682220984745201AF0C4
:1041C8003BF900201AF038F93B685E20984794F8CC
:1041D8001431FEF76ABF364CDFF8E0904FF0000A62
:1041E8000AE01B2B00F071820D2B00F036824FF095
:1041F800010389F801303868FCF7E6FB00285FD036
:104208003868FCF7D9FB83B27E2B32682AD099F83C
:1042180001100029EFD194F82E21002AE1D07D2B3E
:1042280000F0308294F83CE1BEF1000F04D080F039
:104238002003DBB284F83C11511CC9B2224409297D
:1042480084F82E1182F8303100F010820829D2D873
:10425800B4F83A21134403EB132303F0FF03A4F843
:104268003A31C8E784F82EA184F82FA189F801A073
:10427800C1E700BF6CE2020824390020C43C0020DA
:10428800D93C002056555555AC4600200C46002018
:10429800E839002000460020676666660070002046
:1042A8002E5A0020BC460020CDCC4C3E809698006B
:1042B800E41D002040590020283A0020000000207A
:1042C80094F83D3133B194F8313184F83D01302B05
:1042D80000F0D88594F82F21C04BDFF834C3DFF8FD
:1042E80034E3DFF834A30127104600283EF461AF19
:1042F8003268A2EB0802012A00F2AA8194F83E91E2
:10430800B9F1000F40F0EC8194F83F1133F8112017
:1043180012B984F83F71E8E70131B2F5826F84F889
:104328003F1100F0F9801FD9B2F5E26F00F09A80D2
:1043380034D9B2F5046F00F0A480B2F5116F00F023
:10434800AD80B2F5E46FD0D11046A54A176C918ABA
:10435800642303FB07F393FBF1F119F0C5FF002376
:1043680084F82F31FEF725BFB2F5007F00F0B0804A
:104378002CD8B2F5807F00F02281B2F5887FB4D1C5
:10438800DCF800205207B0D500214FF4887019F0EE
:10439800ABFF002384F82F31FEF70BBFB2F5C06FD7
:1043A80000F0AA80B2F5E06F9FD18D4A906B918A98
:1043B800642303FB00F34FF4E06093FBF1F119F081
:1043C80093FF002384F82F31FEF7F3BEB2F5047F84
:1043D80000F02481B2F5806F87D194F84031013321
:1043E800DBB2032B00F2538142F2107184F84031A2
:1043F80001FB03F17B4B1B88002B40F04E81013100
:10440800794B1B78DF07794B1B8848BF0431D807E5
:1044180048BF0A319A0748BF14311F0648BF2831E0
:10442800D80548BF28315A0748BF64311F0748BF1D
:10443800C831980548BF01F5C8719A0648BF01F50B
:104448007A71DF0648BF01F5FA61580648BF01F5E1
:104458007A614FF4806019F047FF002384F82F3108
:10446800FEF7A7BE10465E4AD76B918A642303FB0A
:1044780007F393FBF1F119F037FF84F82F91FEF75A
:1044880098BE5B4BB3F9041001EB8101104649005B
:1044980019F02AFF84F82F91FEF78BBE9EF80520AD
:1044A800002A3FF422AF9AF8001000293FF41DAF0C
:1044B800504B1B8803EB83035B004FF4116093FBA5
:1044C800F1F119F011FF002384F82F31FEF771BEC6
:1044D8009EF8061000293FF408AF474B47491B6870
:1044E800104681FB0321DB17C3EBA10119F0FCFE89
:1044F80084F82F91FEF75DBE9EF80620002A3FF44F
:10450800F4AE3D4B4FF4C060996819F0EDFE0023FE
:1045180084F82F31FEF74DBEDCF8002012F0200998
:104528007FF4E3AE364A1168090600F18D84354AF6
:10453800127B002A3FF4D9AE94F84111032900F206
:10454800F385DFE801F0322819022F4B1B685979EF
:104558009A79DB7901F1407101EB022101EB03410A
:10456800002384F841314FF4826019F0BDFE002326
:1045780084F82F31FEF71DBE244B1A68137A507940
:1045880092781B0403EB002313444A1C84F841214E
:1045980003EB0161E7E71D4B1A68D379107952786C
:1045A8001B0403EB00231344EFE7184B1A689379B5
:1045B800D07812781B0403EB00231344E5E7DCF8FA
:1045C800002051077FF591AE00214FF4807019F05B
:1045D8008BFE002384F82F31FEF7EBBD6CE2020856
:1045E800842A0020EC6E00202E5A00201639002064
:1045F8006C4300200C460020004600206766666673
:104608008C510020AC460020D03B0020684B002095
:10461800203A0020283A0020BA4600209EF80520BB
:10462800002A3FF462AE9AF8001000293FF45DAE0C
:10463800974B5B7B002B00F08B84964B1B8893FB7E
:10464800F1F101EB810149004FF4047019F04CFEBF
:10465800002384F82F31FEF7ACBD4FF0010184F838
:104668002E1184F83031A4F83A21C4E5B4F83A217F
:10467800C2F1FF0293427FF4BAAD4FF0010384F810
:104688003D31B4E54FF0010384F83C31B3E5012333
:1046980084F8403142F21071ACE60231B0E606F01F
:1046A800DDFF7D4B1B68C01A40F6B833984200F214
:1046B800E380DFF808A29AF804303A2B00F0F08281
:1046C800002388F80030FEF791BD3868FCF77CF9C4
:1046D80000287FF48CAD4FF0010384F82F318AE570
:1046E8006E49062019F020FC002384F83E0184F866
:1046F8002F31FEF75EBD94F82C1194F82D316848DF
:104708004A1CFEF73EBD4FF000093B6884F814913F
:104718005E203468DFF8A88198473B6817209847DF
:10472800484619F089FE5F4BA3FB04239B0BA8FBAB
:1047380003125209C2EB0212A3EB8203D8B219F09A
:104748007BFE3B685E2098473B6818209847564B8D
:10475800A3FB04239B09A8FB03125209C2EB021214
:10476800A3EB8203D8B219F067FE484619F064FE3D
:104778003B685E209847FEF79BBC0AF1FF3A84F835
:104788005FA1FFF77CBB0CF1FF3C84F85EC1FFF72B
:1047980040B9013B84F85631FEF743BF013B84F82A
:1047A8005731FFF75FB80024404FA0464FF050093B
:1047B80002E0DBB283F3118815F804A0601C5146AF
:1047C800284419F055FC002840F01B810AF1010328
:1047D8001C44EFF3118389F312882A6E9442E8DBB4
:1047E8000022DBB22A6683F31188FEF708BE304B3D
:1047F80032681B78C4F81C21013B012B3FF6FEAB45
:104808001022022382700371FFF7F8BB3B685E2019
:1048180098473B6810209847404619F00DFE4046DF
:1048280019F00AFE3B685E2098473B6821209847AC
:10483800404619F001FE404619F0FEFDFEF7ADBDF9
:10484800DFF880801B4BB8F80890A3FB09394FEAC2
:1048580099095FFA89F019F0EFFD4FEA192019F06C
:10486800EBFD4CE419F08EFDFEF793BC19F07AFDD0
:1048780001233B70FEF749BC0F4AB2F84A310021C8
:104888000133A2F84A3188F80010FEF7AFBC00BF28
:10489800AC4600200C460020C0580020EBE201087E
:1048A8007848002073B2E745D34D6210318D010876
:1048B8001A390020CDCCCCCCE41D0020A85800200B
:1048C80089888888283A0020AB4B1B88DA0515D4DC
:1048D800D80600F10B84990600F122845A0600F1EB
:1048E8003184180700F14E84D90700F1388413F099
:1048F800020F0CBF4FF004084FF00C089F4BA04A62
:104908001B78D27803F001030AB143F00203532065
:10491800029319F0B3FC9B4A128802EB820202EB65
:104928008202900080B219F08FFC002019F08CFCF4
:10493800954A964912883868C2EBC212520081FB28
:10494800023111444FEAE27ACAEB612A5FFA8AFA25
:104958005146FCF75DF88E4B38681A78029B48EA96
:1049680003088B4B8AEA020A002183F800A0FCF7AF
:104978004FF841463868FCF74BF8854B844A1B785A
:10498800386888EA0303DBB219461370FCF740F86D
:1049980094F84831002B7FF4A7AA4F2019F06EFC39
:1049A80022F04AFC22F048FC22F046FC012138683B
:1049B800FCF72EF8774A764B92F800801B78744AF9
:1049C800386808F0010883F0010341461370FCF7CA
:1049D8001FF86F4B6E4A1B78386888EA030319463C
:1049E8001370FCF715F894F84831FFF77DBA88463C
:1049F80089460846049105918E4606910391FEF773
:104A080043BE39463A2019F08FFA40EA08085FFA9F
:104A180088F8DBE6604B93F800A0BAF1000F3FF48A
:104A280073AB584AB4F816E111883B6802924FEA12
:104A38000E1E64201FFA8EFE00FB01A14FEA4A00F9
:104A4800B1FBF0F14EEA012E1FFA8EFEC1F30321ED
:104A58005E204EEA010998473B68062098475FFAAE
:104A680089F019F0E9FC4FEA192019F0E5FCB4F8CF
:104A78001631029A4949B2F800904A7A01339BB23A
:104A8800012A93FBFAF00AFB1033A4F8163100F060
:104A98006A836E2342484A7B03FB09F380FB0301C8
:104AA8004FEAE379C9EBA1092AB13B4B1FFA89F90F
:104AB8001B7899FBF3F93B68DFF8ECA05E20984778
:104AC8001FFA89F93B683A209847AAFB093A4FEA46
:104AD8005A1A1FFA8AF3D8B2029319F0ADFC029B56
:104AE800180A19F0A9FC3B685E2098473B683B20F0
:104AF8009847642303FB1A939BB22A48053380FB2B
:104B08000320DB17C3EBA000C0B219F095FC00200E
:104B180019F092FC3B68DFF894A0DFF888905E20DB
:104B280098473B6828209847DAF8003089FB032922
:104B3800DB17C3EBA9095FFA89F019F07DFCC9F30B
:104B4800072019F079FC3B685E2098473B680420F1
:104B58009847B8F80830002B40F0F882DAF80830A7
:104B680083F310085FFA88F019F066FCC8F3072091
:104B780019F062FCFFF7C8BA163900202E5A002037
:104B8800C86E00200C46002014390020030820803D
:104B9800A46D0020142B0020BA460020AC4600204B
:104BA800310CC330676666661F85EB5100460020EE
:104BB800B849B94B0093A1F13F06B84BB84A0991DF
:104BC80001F8404C0AA8B7490896FDF737FD089E3A
:104BD800731C08933470089B2922591C08911A7079
:104BE800089BEA22591C08911A70089BC822591C74
:104BF80008910AA81A7026F0D9F9471C0AA93A465A
:104C0800089826F0ABFF089AD31901330893D455B6
:104C1800089B5A1C08921C70089B5A1C08921C700E
:104C2800089B5A1C08921C70089B5A1C08921C70FE
:104C3800089B5A1C08921C70089B5A1C08921C70EE
:104C4800089B5A1C08921C70089B5A1C08921C70DE
:104C5800089B5A1C08921C70089B5A1C08921C70CE
:104C6800089B5A1C08921C70089B5A1C08921C70BE
:104C7800089B0122991812A808911A7050F8283D2B
:104C88009B1B337014F020F8874B2C70C3F898B234
:104C9800FEF7C3BAC4F820B187F80090FEF735BA1A
:104CA8009AF80240C4B1013CE4B20134544451467C
:104CB800002211F8013B534083EA0313DBB2120AC6
:104CC800DF0042EA03228C4287EA131382EA0302D6
:104CD800EFD1002A7FF4F4AC744A754F754B1288F3
:104CE800714CFA61DFF8E0911A68FA629B68B4F8CF
:104CF8004A21F8660021FB64D9F80000F963FA65D7
:104D080005F09EFA029000287EF46BAA0221D9F8D9
:104D18000000FBF749FE94F84C319AF803200392FF
:104D2800642B4FF0040287F8742040F0538294F803
:104D38004D31072B04BF9DF8083084F84D3194F8A5
:104D48004D31069307EB031ADAF80410029108466E
:104D580026F02CF9DAF8081005915FFA80FA08466F
:104D680026F024F9C0B204900AEB0002069B5248D0
:104D7800029902900832C27123F00F0286468272AD
:104D8800049803F00F0300EBCA008EF80D3052466A
:104D98008EF80E000EF10F0026F0E0FE474B049A45
:104DA80005990AF10900184426F0D8FE0298C3793B
:104DB80003F1010ACBB1013B5FFA83FC0CF1080C4B
:104DC800DFF808E184440023073010F8011B59403C
:104DD8008B00CA0883EA410302F018024B404EFADE
:104DE80002F253408445DBB2EFD1344A03980AF803
:104DF800023022F0EFF994F84D310022013384F8A3
:104E08004D3184F84C21029BDDF808A09B785BB1FA
:104E18001AF80510D9F80000FBF7FAFD01359AF8E1
:104E28000230EDB2AB42F3D894F84C31032201338F
:104E380084F84C3187F8742088F80020FFF70AB905
:104E4800FBF7B2FDFEF776B91023042218460AA92B
:104E58008DF82A908DF82B908DF82C908DF82D9048
:104E68008DF828308DF8292019F020FA84F82F9130
:104E7800FEF79FB9124A1268D2067FF536A9804616
:104E8800FFF736B906210F4819F0F2F884F83E0109
:104E9800FFF720BA683900205B4B0020480603085A
:104EA800500603085C060308E41D00200C46002099
:104EB8000000002000460020446900204A690020C4
:104EC8008C510020161F0020405900200007090EB1
:104ED800AE4BAF4A0B93A3F140071268002103F8C9
:104EE800401C2123BB70D30040F10E81A949032641
:104EF800A94B1B88580500F10481DA0700F11F81CE
:104F080003F00203A54A002B1CBF03261146DFF855
:104F1800BC823246404626F021FE06EB080312A862
:104F28000133A8F1020140F8203D00225B1A06F87F
:104F380008207B7013F0C8FEFEF71DBA984AD27895
:104F4800002A0CBF4FF0040C4FF0050CFEF77CBE96
:104F5800944B1988FFF775BB0123D8F800003B7004
:104F6800FBF72AFD0746D8F80000FBF725FD7F066A
:104F78007EF4CBA88E287EF4C8A89AF80030002BBF
:104F88007EF4DFA8884B894A1A602D2384F82431DF
:104F9800FEF7C2B87D4B834A0B9312AFA3F13D00D5
:104FA80047F8200D1188DFF81082A3F14002002095
:104FB8004FF00A0E03F8400C082382F801E0384647
:104FC8009370FDF73DFAD8F800307949DA1781FB7C
:104FD8000313C2EBA30399B23846FDF731FA11F077
:104FE8003DFED8F808800A9B4FEA1842591C0A91DE
:104FF8001A700A9B4FEA1822591C0A911A700A9BC8
:105008005A1C0A9283F800800A9B5A1C0A9218704C
:10501800384613F059FEFEF7ABB9DFF8B4819FEDBF
:10502800658AB8F90230594A0B9207EE903AF8EEC1
:10503800E77A12AF67EE887AA2F14003FDEEE77ACD
:10504800A2F13D0147F8201D02F8400C0822CDEDE1
:10505800027A5A701E229A70BDF808103846FDF779
:10506800EFF9B8F9003007EE903AF8EEE77A3846EB
:1050780067EE887AFDEEE77ACDED027ABDF8081082
:10508800FDF7DEF9B8F9043007EE903AF8EEE77A62
:10509800384667EE887AFDEEE77ACDED027ABDF8FC
:1050A8000810FDF7CDF9384613F00EFEFEF75DB98E
:1050B800414B9046B3F900A06420FEF7EDB9394999
:1050C8009A790B8803EB830303EB83034FEA830886
:1050D8001FFA88F8002A40F00B814FF0FF330FFACF
:1050E80083FA11F0BBFD40B2FEF7D6B94FF0340891
:1050F80004E4984699461846049305930393FEF7EB
:10510800C3BA03262D4902E72D4B224A1B682D49B5
:1051180003F48003002B16BF114604260326E7E696
:105128004FF02408FFF7EABB4B1CDBB2042B84F8D2
:1051380041314FEA01617FF416AAFFF711BA2249FB
:105148000426E4E64FF01008FFF7D8BB11F086FDFF
:1051580019F072F9002019F06FF9FEF7D5BF4FF07A
:105168000808FFF7CBBB3B685E2098473B683920AF
:1051780098475FFA89F019F05FF94FEA192019F09A
:105188005BF9C7E44FF02008FFF7B8BB6839002087
:105198000C2B0020340603081639002044060308A7
:1051A800C86E00200C46002080480020E839002006
:1051B8006766666658A08B410046002038060308DB
:1051C8008C5100202C0603083C0603082B390020CC
:1051D8006C43002097F875A0584904951AF00F0FF2
:1051E80004BF0AF1010A5FFA8AFABAF1070F28BF69
:1051F8004FF0010A4FEA0A1C07EB0C03187C504BCE
:1052080002930A18002392F824104D4A93725FFA09
:105218008CF31A464B4B964607EB0C024EEA0000FD
:1052280001291870D26803F101000CD90239C9B2FA
:105238008D1C1D44034603F8012BAB424FEA122292
:10524800F9D101310844BC4422F060030AF1010A93
:105258009CF811205FFA8AFA1343BAF1080F037019
:1052680000F1010340D04FEA0A1C07EB0C01354A54
:10527800087C324901449A1A91F8241055180EF105
:10528800100E132D5FFA8EFEC6DD049D0298DFF81E
:10529800C0E0D1B28B1DDBB243F04002C27103F112
:1052A800010CCBB14B1DDBB20833C31804930EF1CC
:1052B8000100002310F8011B59408B0083EA4103C9
:1052C800CA084B40204902F0180241FA02F2534042
:1052D800049A8242DBB2EDD103980CF80E3087F8BD
:1052E80075A021F077FF8EE5164A049D9A1ACDE73E
:1052F800164B1B68F3E698469946184604930393A1
:10530800FEF7C2B9984699461846049305939E46F7
:105318000393FEF7B9B90393FEF7B6B9984603931A
:10532800FEF7B2B9984699460393FEF7ADB9984689
:10533800994618460393FEF7A7B900BF6CE2020826
:1053480044690020516900200007090E004600202A
:105358004A6900202DE9F04F2DED0C8B3C4B1B7852
:1053680095B0012B089001F08A863A4C94F80021F8
:10537800002A41F02181072B374D01F07B8600235D
:1053880005936B6834489847002800F06981B5F8A0
:10539800B470002285F85520002F40F04787B5F9F2
:1053A8003E00AA6AB5F93C60696AB5F94030DFF891
:1053B800B4B0821AE86A6A63711A1B1A296327480B
:1053C80095F85610AB6316F09DFDDBF80030990098
:1053D80040F1F080D5ED0D5AD5ED0C7A204A94EDC8
:1053E800656AD4ED666A94ED677AD4F8A0311268DC
:1053F800B8EEE58AD5ED0E5AF8EEE77AF8EEE58ACA
:10540800013377EE867A38EE268A78EE878A9342D9
:10541800C4ED657A84ED668AC4ED678AC4F8A03164
:1054280001F0EA830A4B1F78142F02F02B87002320
:10543800D4F8A8610693062E00F2AF80DFE816F0D4
:10544800F2154F158414B71614006315E81400BF3D
:105458009C460020A820002000700020307000200A
:10546800883E00208C510020D84B1A78D4F8ACE143
:10547800DFF8D0C39FEDD67A4FEACE000CEB0003DD
:1054880083ED007A002A7DD0D249B0EE476AF0EE6B
:10549800476A0023F1EC017A013367EEA77A05EE3B
:1054A800903AB4EEE77AF1EE10FAF8EEE55AB8BFA2
:1054B800B0EE677A934276EEA76AA7EEA56AE9D1BD
:1054C800F5EEC06A0CEB0003F1EE10FA83ED007AFA
:1054D80058DDC6EE265AC04BC04A1288F7EE007A4D
:1054E80075EEE75AD3ED007A65EEA77AFDEEE77A16
:1054F80017EE903A812B43F337859342A8BF1346A2
:1055080007EE903AF8EEE77AB54B00EB0E0103EBA5
:10551800810393ED057AD3ED003A93ED066A93ED96
:10552800014AD3ED046AD3ED034A93ED025AA3EE80
:10553800A77AA4EE276A66EEC76AA7EE646ABDEE8C
:10554800C77AE5EE276A17EE101A812983ED056AF6
:10555800C3ED066A43F305858A42A8BF0A4607EEEB
:10556800902AF8EEE77AFCEEE77ACDED077ABDF8F7
:105578001C300CEB00029380BEF1000F02D1132FF8
:1055880004F05281152F42F034846044DFF8B88269
:10559800838828F81E30D4F8A861924B013683FB23
:1055A80006239A19F317C3EBA203C3EBC303F61A36
:1055B800C4F8A8618C4B1B78002B01F003818B4E3B
:1055C800DFF88892DFF880A206F5BC780027884BC0
:1055D800D5ED087A1B78172B01F0A28396ED007A97
:1055E800B8EEC78A082B28EE278A07D1B0EE480AFA
:1055F800069326F027FC069B2AF81700DBF8002004
:1056080092000BD5002F04F04284B0EE480AD5F87A
:10561800143208F170009847B0EE408AB0EE480A9C
:10562800D5F83431A8F170009847D5F8A431404630
:1056380098476F4B1B78032BB0EE408A01F07D83AF
:10564800D6F8F800D5F8B830B0EE480A98470137D0
:10565800032F08F12408A9EC010A06F10406B6D1C3
:10566800634B93F80090B9F1070F00F09C8694F80B
:10567800B831002B40F0A4865E4B5B79002B40F0DC
:10568800CF8501235A4A84F8B8311278072A02F0E4
:105698002A8000230B93584B94ED709A93ED007A6F
:1056A800564BD4ED6FCAD3F800A0554B0693F7EECE
:1056B800007A37EEC9CA534B09932CEE07CA524BEE
:1056C8000A93B4EEE7CA514B07930025F1EE10FA9E
:1056D8004F4BDFF87C91DFF87CB1DFED4E8A9FED10
:1056E8004EAADFED3BBADFED4D9A9FED4DBADFEDE7
:1056F8004DAADFF864814C4F059388BFB0EE67CAA6
:105708002E464A4B99ED008A2B44D3ED007AF5EEEC
:10571800407AF1EE10FA17D0454B2B44D3ED006ACE
:1057280038EE667AB0EEC76AF4EEC67AF1EE10FA91
:1057380008D5B5EEC07AF1EE10FACCBF37EEA68ADE
:1057480036EEE78A83ED008A069B1A88930700F0F5
:105758008580022E00F082809AF82E10354B07EED5
:10576800901A2B4493ED007A4B42F8EEE76A07EE65
:10577800903A26EE877AF8EEE77AB4EEE77AF1EE19
:1057880010FA0AD407EE901AF8EE677AF4EEC77AA0
:10579800F1EE10FA88BFF0EE477A274B274903EB62
:1057A800460331F91600B3F90C30C31A07EE103A64
:1057B800B8EEC77AD007E7EE687A40F15186204BF9
:1057C80093ED008A27EE888A48E000BF8E3E0020CD
:1057D80000000000A8200020903E00208C3E002001
:1057E800C440002093244992853E00203070002058
:1057F8009C46002068510020204A0020684B002069
:1058080016390020780000202E5A00207C510020F4
:10581800602A0020CDCCCC3DAE47813F0000C84275
:1058280000003443610BB63B6C2A0020144A002068
:105838006C22002014220020B82C00206C43002089
:10584800FC490020AC400020A046002080510020E8
:10585800AC2100200C490020782A0020079B94F8EE
:10586800D0212B44D3ED01DA38EE6DDA002A3DD091
:10587800D34BD4F8D42108991B688A1A9A4235DD8B
:105888009AF84830022B01F0B587022E04F05282B4
:10589800CC4B1B68990740F17C87CB4BCB49DFF891
:1058A80098E331F916C09EED008ADFF890E3C7ED62
:1058B80000BA03EB460028EE288AB0F90C00A0EBEA
:1058C8000C0007EE900AF8EEE77ADEF8000027EE03
:1058D800888A904238EE6DDAC1F25581F7EE007A87
:1058E800B4EEE79AF1EE10FA01F12481B84B2B449B
:1058F80093ED000A059B2CEE800A022E20EE0D0A7D
:10590800A3EC010A059304F0DC81099BDBED007A26
:1059180093ED007AAF4BD7ED006A93ED006AAE4B7A
:1059280067EE277A2B4427EE8C7AD3ED007A67EE60
:10593800277AF0EE665AE7EE8D5AB1EE467AB4EE63
:10594800E57AF1EE10FA08DCB4EEE56AF1EE10FA49
:105958008CBFB0EE657AB0EE467A94ED706AF7EED9
:10596800007AB4EEE76AF1EE10FAACBF0123002327
:1059780043B1F0EEE66AF0EEC77AF4EEE67AF1EEBD
:1059880010FA01D587ED007A022E04F07481934A4B
:10599800934B52F826001B68B0EE6D0A9847914A5F
:1059A800914B52F826001B6898479AF8373023B174
:1059B800069B1B88002B00F0BD85B0EE6B8A8B4BD5
:1059C800DBED007A38EE400A2B4493ED008A83ED34
:1059D800000A9AF8483030EE480A80EE278A3BB32E
:1059E8000A9B1B7813F0010300F0258594F8D03149
:1059F800F7EE007AB4EEE79AF1EE10FAC0F2E88416
:105A0800002B40F0E8847A4AD2ED007AB0EEC87AEA
:105A1800B4EEE77AF1EE10FA0ADD764AD2ED007AB2
:105A2800B0EECD7AB4EEE77AF1EE10FA02F33F84E5
:105A3800714B94F8E0212B44D3ED007A6CEEA77AF1
:105A480027EE888A88ED008A32B9059BC7ED00BA2F
:105A580043ED01BAC8ED00BA0136032E09F1040975
:105A680008F1040807F1040705F104057FF449AEBD
:105A7800624B1B78072B01F02083012B01F038863D
:105A8800002794F8E831002B40F04D865C4A5D4BC6
:105A980010681B6810F4805A93F82C3040F0BC86CC
:105AA800594A5A4992ED006A498B594A84ED7E6AEF
:105AB80092ED007A574A84ED7F7A07EE901AF8EE55
:105AC800E76AD2ED037A544A84ED7C6A37EE467A67
:105AD80077EEE67AD2ED006A84ED7B7A012284F8CB
:105AE8000022C7EEA65A4D494D4A91ED005A4D493C
:105AF8009FED4D6A91ED004A4C49DFED4D6AD1EDBD
:105B0800004A92ED007A35EE045AF7EE007AF4EE88
:105B1800E75A35EE245AF1EE10FA88BFF0EE675ACC
:105B280025EE065AF4EEE65AB1EE476AF1EE10FA9F
:105B3800B4EEC65AB8BFF0EE665AF1EE10FAC4EDEC
:105B4800815A01F1E680B4EEC75AF1EE10FA88BF27
:105B5800B0EE475A314ADFED346AD2ED017A314A64
:105B680092ED014A314A77EE847AD2ED014A77EE16
:105B7800A47A67EEA67AB4EEE76AF1EE10FA08DCCA
:105B8800B4EEE77AF1EE10FA8CBFB0EE676AB0EEC9
:105B9800476A224ADFED246AD2ED027A214AD2ED21
:105BA800024A244A77EEA47A92ED007A67EEA67A42
:105BB800B1EE473AF4EEC37AF1EE10FA49D43FE079
:105BC800284A0020203A0020B82C00206C430020EE
:105BD800D0490020444A0020DC4900201449002014
:105BE80010490020684900206449002080220020D4
:105BF800384A0020344A0020E84900209C4600200A
:105C08008C510020684B0020302B002010570020BA
:105C1800882C0020BC460020044B0020602A00206D
:105C2800484A00206C2A00206F12833A782A002004
:105C3800000000004C4A0020FC490020244A0020B3
:105C4800F4EEC77AF1EE10FA8CBFB0EE473AB0EE38
:105C5800673AF04A52780AB9B1EE433A002B41F05C
:105C68007A83F7EE003AEC4D2A78002A02F06B8628
:105C7800EA4BDFEDEB6AD3ED024A93ED017AD3EDFF
:105C8800037A66EE244AE5EE074AE3EE274A63EE16
:105C9800A44AF4EEE64AF1EE10FAB4BFB0EE664A52
:105CA800B0EE644A98BFF0EE646A012ACDED0C4A62
:105CB80002F06E8693ED067AD3ED052AD3ED077AC6
:105CC80026EE077AA5EE227AA3EE277A23EE877AC4
:105CD800B4EEE67AF1EE10FAB4EEC47A8CBFF0EEC8
:105CE800667AF0EE477AF1EE10FA98BFF0EE676A3E
:105CF800B4BFF0EE447AF0EE477A022A8DED0D7AC1
:105D080000F0DE8093ED0A7AD3ED092A93ED0B4A71
:105D180026EE077AA5EE227AA3EE047A23EE877A96
:105D2800B4EEE67AF1EE10FAB4EEE77A8CBFB0EE94
:105D3800664AB0EE474AF1EE10FA98BFF0EE446AB0
:105D4800A8BFF0EE477A032A8DED0E7A00F0B880EE
:105D580093ED0E7AD3ED0D2A93ED0F4A26EE077ACE
:105D6800A5EE227AA3EE047A23EE877AB4EEE67AD9
:105D7800F1EE10FAB4EEE77A8CBFB0EE664AB0EEF8
:105D8800474AF1EE10FA98BFF0EE446AA8BFF0EE69
:105D9800477A042A8DED0F7A00F0928093ED124A2B
:105DA800D3ED112A93ED137A26EE044AA5EE224A82
:105DB800A3EE074A23EE844AB4EEE64AF1EE10FA5F
:105DC800B4EEE74A8CBFB0EE667AB0EE447AF1EEF4
:105DD80010FA98BFF0EE476AA8BFF0EE447A052A99
:105DE8008DED104A6CD093ED164AD3ED152A93ED3C
:105DF800177A26EE044AA5EE224AA3EE074A23EEB6
:105E0800844AB4EEE64AF1EE10FAB4EEE74A8CBFE3
:105E1800B0EE667AB0EE447AF1EE10FA98BFF0EE82
:105E2800476AA8BFF0EE447A062A8DED114A47D09A
:105E380093ED1A4AD3ED192A93ED1B7A26EE044AFC
:105E4800A5EE224AA3EE074A23EE844AB4EEE64AB8
:105E5800F1EE10FAB4EEE74A8CBFB0EE667AB0EE17
:105E6800447AF1EE10FA98BFF0EE476AA8BFF0EE58
:105E7800447A072A8DED124A22D093ED1E7AD3ED8B
:105E88001D2A93ED1F4A26EE077AA5EE227AA4EE84
:105E9800037A27EE237AB4EEE67AF1EE10FAB4EE3E
:105EA800E77A8CBFB0EE666AB0EE476AF1EE10FA98
:105EB8008DED137A98BFF0EE466AA8BFF0EE477AE8
:105EC80077EEE67AF7EE006AF4EEE67AF1EE10FA8B
:105ED800C4ED707A43F38D8486EEA77A022ADDED4D
:105EE8000D7A67EE244A67EE877ACDED0C4ACDED40
:105EF8000D7A2DD0DDED0E7A67EE877A032ACDED87
:105F08000E7A25D0DDED0F7A67EE877A042ACDED7B
:105F18000F7A1DD0DDED107A67EE877A052ACDED70
:105F2800107A15D0DDED117A67EE877A062ACDED65
:105F3800117A0DD0DDED127A67EE877A072ACDED5A
:105F4800127A05D0DDED137A27EE877A8DED137A74
:105F5800344B1E6816F0805601F0AA80F6EE005AFF
:105F6800C4ED815A002A02F0E3842F4BD4ED7F4A16
:105F780093F8038094F900320A99D4ED7E6A91F877
:105F880000E0DFF8B0C02949DFF8AC90B1F906109D
:105F98009CED007A059106EE103AFDEEE44A244B9A
:105FA80099F80090B3F81AB094ED7B5AD4ED7C7A46
:105FB80014EE903AFDEEE64A00F0100C00F4800072
:105FC8000EF0010EB8EEC66A14EE901A0690B8F1FB
:105FD800000F41F00182DFF84480BCF1000F41F06E
:105FE800AE8098ED007ADDED0C6ADFF850C025EE42
:105FF800877AA6EE267AF0EE676AE5EE076ABDEEC6
:10600800E67A17EE106A17EE100A9E42A8BF1846E5
:1060180016E000BFF42C00204A460020744A0020F5
:10602800000000000C2B0020C86E0020EC38002077
:1060380010570020504A0020B0530020DC2A0020CE
:10604800B142C8BF084607EE100AB8EEC77A012A5F
:106058008CED007A00F0DC8098ED047ADDED0D6AB5
:1060680025EE877AA6EE267AF0EE676AE5EE076AED
:10607800BDEEE67A17EE106A17EE100A9E42A8BF28
:106088001846B142C8BF084607EE100AB8EEC77AEC
:10609800022A8CED017A00F0BB8098ED087ADDEDDC
:1060A8000E6A25EE877AA6EE267AF0EE676AE5EEA6
:1060B800076ABDEEE67A17EE106A17EE100A9E42DE
:1060C800A8BF1846B142C8BF084607EE100AB8EE86
:1060D800C77A032A8CED027A00F09A8098ED0C7A40
:1060E800DDED0F6A25EE877AA6EE267AF0EE676A6E
:1060F800E5EE076ABDEEE67A17EE106A17EE100AAB
:106108009E42A8BF1846B142C8BF084607EE100A0B
:10611800B8EEC77A042A8CED037A79D098ED107A14
:10612800DDED106A25EE877AA6EE867AF0EE676ACC
:10613800E7EE056ABDEEE67A17EE106A17EE100A6A
:106148009E42A8BF1846B142C8BF084607EE100ACB
:10615800B8EEC77A052A8CED047A59D098ED147AEE
:10616800DDED116A25EE877AA6EE867AF0EE676A8B
:10617800E7EE056ABDEEE67A17EE106A17EE100A2A
:106188009E42A8BF1846B142C8BF084607EE100A8B
:10619800B8EEC77A062A8CED057A39D098ED187AC8
:1061A800DDED126A25EE877AA6EE867AF0EE676A4A
:1061B800E7EE056ABDEEE67A17EE106A17EE100AEA
:1061C8009E42A8BF1846B142C8BF084607EE100A4B
:1061D800B8EEC77A072A8CED067A19D098ED1C7AA2
:1061E800DDED136A65EE875AE6EE265AE5EE257A66
:1061F800FDEEE77A17EE900A8342A8BF0346814274
:10620800C8BF0B4607EE903AF8EEE77ACCED077A6E
:10621800BEF1000F40F09482002A40F08C828FE299
:10622800D24B1B78013BDBB2FFF72CBAD04B07935C
:106238004FF47A761B68B6FBF3F3C3EB4316CD49EC
:10624800DFF8708391F801A0CB49B8F9060091F8FE
:10625800009003EB8603DE00B6B2B74202F00D8170
:10626800D5F88810B5F93CE0EB6E4A1C07EE90EAC9
:106278007344012AC5F88820EB66F8EEE77A02F045
:106288000781D5ED1E5AD5ED206A07EE102A37EEA4
:10629800E56AB8EEC75A012F86EE057A37EE257AF9
:1062A80077EEC77A85ED1F7AE7EE866A85ED1E7A66
:1062B800F0EE667AC5ED216AC5ED206A02F0AC847D
:1062C800D5F89C10B5F93EE02B6F4A1C07EE90EA12
:1062D8007344012AC5F89C202B67F8EEE77A02F090
:1062E800F080D5ED235AD5ED256A07EE102A37EE52
:1062F800E56AB8EEC75A012F86EE057A37EE257A99
:1063080077EEC77A85ED247AE7EE866A85ED237AFB
:10631800F0EE667AC5ED266AC5ED256A02F0B0840E
:10632800D5F8B010B5F940E06B6F4A1C07EE90EA5B
:106338007344012AC5F8B0206B67F8EEE77A02F0DB
:10634800D980D5ED285AD5ED2A6A07EE102A37EEFE
:10635800E56AB8EEC75A012F86EE057A37EE257A38
:1063680077EEC77A85ED297AE6EE276A85ED287AF1
:10637800F0EE667AC5ED2B6AC5ED2A6A02F07484E0
:10638800A8F80600B5F8B4307B4A013B92F80090B3
:10639800A5F8B43007990023B9F1070F4B608B605B
:1063A800CB607FF464A905F059F9059BDFF80482F6
:1063B800C01A94F8B831A8F80000002B3FF45CA983
:1063C800013B84F8B83115B0BDEC0C8BBDE8F08FFB
:1063D800002B3FF42DABD4F8D431089AD31A674A6E
:1063E80012689A427FF724AB654BD3ED007AB0EE82
:1063F800CDDAB4EEE7DAF1EE10FA0CD4614BD9ED50
:10640800007A93ED007AF0EEE77AF4EEC77AF1EECF
:1064180010FA7FF70DAB5C4B1A88002384F8D03153
:10642800A2B15A494A69002A3FF402AB0A681360CC
:106438004B74FFF7FDBA94F8D021002A3FF4F8AA6C
:10644800514A84F8D0311288002AEAD1504A514B77
:106458001178186881F00101FBF7D2FBFFF7E8BA61
:1064680094ED5E7AB1F90000D4ED5F6AB1F902E00B
:10647800494AF4EEC76A80EAE0738EEAEE71A3EB4C
:10648800E073F1EE10FAA1EBEE71B8BFF0EE476AD7
:106498008B42B8BF0B4607EE103A1378B8EEC77AAE
:1064A80027EE287A002B00F031823C4B93ED005AFE
:1064B800B5EEC05AF1EE10FA40F3F685384BD3ED3D
:1064C800004AF5EEC04AF1EE10FA40F3ED8534EEDD
:1064D800C77A66EEE95A87EE246AC5EE856AB7EE92
:1064E800007AB4EEC76AF1EE10FA88BFB0EE476AD8
:1064F800B5EEC06AF1EE10FA76EE876AB8BFB0EE74
:106508006B6A66EE266AF4EEC76AF1EE10FA88BF87
:10651800F0EE476AF5EEC06AF1EE10FAB8BFF0EE99
:106528006B6A204B93ED007A67EE877AA7EEA68A0E
:10653800FFF794B91C4B1D4A2B4493ED007AD2ED1A
:10654800007A1B4B67EE277AF7EE006AF4EEE67ADC
:10655800F1EE10FA93ED007A88BFF0EE667A67EEF6
:10656800877A27EE888AFFF72ABA00BFAC2C00206A
:106578007C510020685100209C460020284A0020B9
:10658800344A00203C4A0020AC6F0020B46F002041
:10659800AE6F0020B06F0020084A0020044A002097
:1065A8000C4A0020004A002020220020F849002040
:1065B800F4490020A0460020072B02F0E4810026C1
:1065C800DFF83CB3B64DDBF80030590501F1258002
:1065D800B44B1B78002B40F0C281B34F94F81231B2
:1065E80023B1B24A1288920742F0638194F81821C5
:1065F800002A41F01C80BB7F002B00F0AD83022BEA
:1066080001F0E387032B01F07882A94B5B88F97FBF
:106618000231C9B2002A01F0C987002B01F0C687F0
:10662800A4480068B3FBF0F30FFA83F9A4F8489183
:10663800002903F0E68007EE909AF8EEE77AF7EE85
:10664800006A86EEA77A9C4B0129D4ED576AD3EDF0
:10665800007A77EEE67A67EE877AC4ED537A21D02E
:10666800D3ED017AD4ED586A77EEE67A022967EE1F
:10667800877AC4ED547A15D0D3ED027AD4ED596AED
:1066880077EEE67A032967EE877AC4ED557A09D062
:10669800D3ED037AD4ED5A6A77EEE67A67EE877A15
:1066A800C4ED567A85480078092803F0E280B9F1EC
:1066B800000F40F3588391B394ED577AD4ED537A91
:1066C80077EE877A0129C4ED577AC3ED007A21D095
:1066D80094ED587AD4ED547A77EE877A0229C4ED8E
:1066E800587AC3ED017A15D094ED597AD4ED557ADC
:1066F80077EE877A0329C4ED597AC3ED027A09D077
:10670800D4ED5A7A94ED567A77EE877AC4ED5A7AB0
:10671800C3ED037A01390229B8BF0221C9B2002AA0
:1067280018BF022120E30A9B654D1B78DE0700F1A4
:1067380032812A7822B192006249634825F00EFA24
:10674800624B1B68002B40F0E882614B1B789BB1C1
:10675800287870B1DFF87081DFF8A8910026F0B2D0
:10676800D9F80030B8EC010A9847287801368642F3
:10677800F5DB584B1B689847504B1B78072B00F0EC
:10678800D784012384F8003115B0BDEC0C8BBDE82B
:10679800F08F514BC7ED00BA1B689342BFF69EA815
:1067A8004E4B1A88002384F8D031002A41F05B86CA
:1067B8004B4A4C4B1178186881F00101FBF720FA1D
:1067C800FFF794B8484EDFF8409106F5F47806F5DF
:1067D8001577F6EC017A95ED080AD5F81432F8EE3B
:1067E800E77A404627EE800A9847A8F1E000D5F8F6
:1067F80034319847A8F17000D5F8A4319847D6F8F5
:10680800F400D5F8B830984708F124084745A9ECB2
:10681800010ADED1FEF724BF0A9A1278D50703D4FD
:10682800214A128BA4F8F421304A2349128891EDA9
:10683800037A07EE902AF8EEE77AB4EEE77AF1EEFB
:1068480010FA41F23B802A49098807EE901AF8EEBF
:10685800E77AB4EEE77AF1EE10FAC0F2A18725499B
:10686800254AD1ED006A92ED006A2449C4ED7E6A9A
:10687800BCEEC75A76EE665A15EE102AC4ED7C6A4D
:10688800C4ED7B5A84ED7F6AA4F8F4210122D1ED8E
:10689800006A84F8002277EE677AFFF722B900BF12
:1068A80000700020A4040020105700201639002092
:1068B800203E0020DC2C0020BC4600209C46002006
:1068C8004A460020544A0020DC2A0020D8440020F0
:1068D800B8560020AC530020244A0020AC6F00209A
:1068E800AE6F0020B06F002030700020084B0020F1
:1068F8000A4B0020F44A0020882C0020104B00206E
:106908008C510020A453002080510020AC4B93ED03
:10691800006AB4EECA6AF1EE10FA40F17986F7EE31
:10692800005A75EEC65A3BEE477A65EEAA5AA54B51
:10693800A7EE256A93ED007A26EE076AB5EEC06ADF
:10694800F1EE10FA40F2B083C9EE865AB7EE007A3B
:10695800B0EE476AA6EEE56AF0EE466AD3E59A4BD2
:106968009A4FB3F906207B8B9A423FF737AE984B84
:106978001B78012B01F00586192B01F002860E2BDE
:106988003FF42CAE082B3FF429AE924B00229A60BC
:10699800C4F80C2122E62B78002B3FF4D1AED4EDBD
:1069A8005F3A94ED5E6AD4ED7C7A8B4A94ED7B7AFB
:1069B800D2ED005A94ED5C4AD4ED5B4ADFF83082A0
:1069C800DFF830C2F4EEC63AF3EE046AF1EE10FADC
:1069D80037EEA65A00F1E28798ED026A26EE446A7D
:1069E800F0EE674AE6EE074AF4EEC54A34EEE66A88
:1069F800F1EE10FA48BFB0EE656A012B8CED006A23
:106A08003FF49EAE98ED066A26EE446AF0EE674AB9
:106A1800E6EE074AB4EEE45A34EEE66AF1EE10FA0E
:106A280088BFB0EE656A022B8CED016A3FF488AE30
:106A380098ED0A6A26EE446AF0EE674AE6EE074ADF
:106A4800F4EEC54A34EEE66AF1EE10FA48BFB0EE4D
:106A5800656A032B8CED026A3FF472AE98ED0E6AFC
:106A680026EE446AF0EE674AE6EE074AB4EEE45AC8
:106A780034EEE66AF1EE10FAC8BFB0EE656A042B90
:106A88008CED036A3FF45CAE98ED126A26EE446A18
:106A9800F0EE674AE6EE074AB4EEE45A34EEE66AE8
:106AA800F1EE10FAC8BFB0EE656A052B8CED046AEA
:106AB8003FF446AE98ED166A26EE446AF0EE674A51
:106AC800E6EE074AF4EEC54A74EEE66AF1EE10FA0D
:106AD80048BFF0EE656A062BCCED056A3FF430AE90
:106AE800D8ED1A6A66EEC46AF0EE674AE6EE874A9F
:106AF800B3EE046AB4EEE45A74EEC66AF1EE10FA24
:106B0800C8BFF0EE656A072BCCED066A3FF418AEF5
:106B1800D8ED1E6A26EEC44AE4EE077AF4EEC57A8A
:106B280077EEC67AF1EE10FA48BFF0EE657ACCED52
:106B3800077A05E60799294BD1ED017A93ED007A9A
:106B4800F0EEE77AF4EEC77AF1EE10FA7EF5CEAE03
:106B5800D1ED027AF0EEE77AB4EEE77AF1EE10FAC8
:106B68007EF7C4AED1ED037AF0EEE77AB4EEE77AB9
:106B7800F1EE10FA7EF7BAAE194B1B689B077FF54A
:106B88000FAE1849184BB3F90C20B1F900E01748BB
:106B9800AEEB020E00688EEAEE72A2EBEE72824253
:106BA800BEF6A4AEB3F90E30B1F90220D21A82EAC9
:106BB800E273A3EBE27398427EF798AEF0E500BF6C
:106BC800104A0020044A0020EC380020105700200A
:106BD800F42C0020BC460020504A0020304A0020F7
:106BE800203A00206C430020B82C00202C4A0020BA
:106BF800744A0020DC2A002007EE103A524BDFF8D6
:106C080054811B78C4F8A071B8EEC77AF7EE006A11
:106C1800132B86EE879AB8F90400B4F8A47195EDA1
:106C2800080A01F0AB83494B494A93ED001A93EDEA
:106C3800053A93ED122A93ED176AD3ED091A93EDED
:106C48000E4AD3ED015AD3ED063A93ED0A7A93ED45
:106C58000F5AD3ED132AD3ED186AD3ED044AD3EDB6
:106C6800030A67EE897A69EE288A29EE088AA1EE76
:106C7800273A02EB87060021A2EE286AC4F894118D
:106C8800C4F89811A1EE884AE5EEA73AA7EE085A8B
:106C980093ED167AD3ED0D5A93ED021AD3ED0C1A33
:106CA80086ED003AE2EEA86A64EEC34A27EE467A19
:106CB80093ED0B2AD3ED152A86ED204AE0EEC33A70
:106CC80065EEC45A93ED143AC3ED053AE1EE274A4E
:106CD800F0EE477AA1EEC45AE2EE085AE2EEC66A2E
:106CE800E3EE287AC3ED064A83ED0E5AC3ED0F5A38
:106CF80086ED406AC3ED176AC3ED187AC4F89C1193
:106D08007B1C03F01F03A4F8A431A8F80400FEF7C5
:106D180089BBB0EE465AFEF71DBF15F09DFF14E57E
:106D280096ED007A05EB4702B8EEC78A928F2AF8EB
:106D3800172028EE278AFEF761BC25F083F82AF889
:106D48001700FEF77DBC00BF9C46002030410020A4
:106D5800AC3E0020A0460020A4F848319946002AFD
:106D680000F07281DF4B0221DF4ADFEDE06A106834
:106D7800DF4A90F802C092F800E0027807EE902A05
:106D8800F8EEE77AB0EE007A67EEA67AF4EEC77A04
:106D9800F1EE10FA40F3108337EEC77ADFEDD56ACB
:106DA800B0EE676AA7EE266AB0EE467A9FEDD26A21
:106DB800D3ED006A66EE866AB0EEE66AC4ED5B6AF9
:106DC80084ED5E6ABCF1000F13D005EE90CAB8EEF0
:106DD800E55ADFEDC65A66EEA64A25EE255AF7EEC5
:106DE800005A75EEC55A64EE864AE4EE855A66EE98
:106DF800A56ADFEDC25A427927EE257A27EE267A70
:106E0800CAB1DFEDBA6ADFEDBE5A26EE266A06EE93
:106E1800902AF8EEE66A26EE266AB4EEE56AF1EE06
:106E280010FA00F37285F7EE005A35EEC66AC5EE21
:106E3800866A27EE267ABEF10C0F9FEDB28ADFED47
:106E4800B26A00F00985B4EEC87AF1EE10FA98BF7C
:106E5800B0EE478AB4EEE68AF1EE10FAB8BFB0EEAB
:106E6800668A84ED418A002900F0E280B0EE007A5B
:106E7800F4EEC77AF1EE10FA05DD37EEC77ADFEDEA
:106E88009D6AE7EE267A93ED017ADFED9B6A27EE9D
:106E9800267AB0EEC76A84ED5C7A84ED5F6ABCF14D
:106EA800000F13D006EE90CADFED905AF8EEE66AAE
:106EB80027EE075A66EEA56AF7EE005A75EEE65A0F
:106EC80025EE065AE5EE265A27EE257ADFED8B6A7F
:106ED800827967EEA67A67EE877AAAB107EE102A5A
:106EE800B8EEC77ADFED815ADFED856A27EE067ABC
:106EF80027EE257AB4EEE67AF1EE10FA40F309852A
:106F0800DFED826A67EEA67ABEF10C0F00F083848B
:106F1800DFED7C6A9FED7C7AF4EEE67AF1EE10FA0A
:106F280088BFF0EE667AF4EEC77AF1EE10FAB8BFD1
:106F3800F0EE477A0129C4ED427A79DD4278DFED37
:106F48006B6A07EE902AF8EEE77AB0EE007A67EE01
:106F5800A67A427AF4EEC77AF1EE10FA05DD37EE3A
:106F6800C77ADFED646AE7EE267A93ED027ADFED01
:106F7800626A27EE267AB0EEC76A84ED5D7A84ED00
:106F8800606A9AB106EE902ADFED585AF8EEE66A82
:106F980027EE075A66EEA56AF7EE005A75EEE65A2E
:106FA80025EE065AE6EE855A27EE257ADFED536A76
:106FB800C37967EEA67A67EE877A0BB307EE103AC5
:106FC800B8EEC77ADFED495ADFED4D6A27EE067A4B
:106FD80027EE257AB4EEE67AF1EE10FA0CDCB5EE7F
:106FE800C07AF1EE10FA01F1D382B7EE006A36EEFC
:106FF800477AC6EE076A01E0DFED446A67EEA67AD3
:10700800BEF10C0F00F04584DFED3E6A9FED3E7A3D
:10701800F4EEE67AF1EE10FA88BFF0EE667AF4EE56
:10702800C77AF1EE10FAB8BFF0EE477AC4ED437AAA
:10703800BEF1090F00F0D38397F82170002F40F0BC
:107048006A83002384F81831314B1B7823B9314FF8
:10705800BB78002B41F0C0820898F9F7D1FA244B8D
:107068001B78072B00F01F840022072B84F80021CF
:107078007EF485A904F0F2FA0590FEF782B9264B52
:10708800264C1A68264BDFF8A48094F80001D269D0
:107098001B88A8F80020A8F8023000287FF48FAADF
:1070A8000590204DFEF76DB9DFED1F6AFFF739BA7D
:1070B80041023EF553AFFEF755BF04F0CFFA0C4B33
:1070C8000B9A1B78DFF86480801A012BA8F802005D
:1070D80000F01083072B7EF4D3AC04F0BFFA074608
:1070E800FEF7CFBCBC460020D03B00200AD7233C8B
:1070F8009C460020D7A368416F12033B0000484319
:10710800A4707D3F00C0F94400C0F9C40000C84223
:10711800BD6E0020B64C0020CC3B0020A8200020EB
:107128002E3600200070002000000000A04600203D
:1071380004F094FAA24BC01BD880FFF722BBBEF123
:10714800000F41F05B8498ED007ADDED0C6ADFF802
:1071580084C225EE877AA6EE867AF0EE676AE7EEB5
:10716800056ABDEEE67A17EE106A17EE100A9E421F
:10717800A8BF1846B142C8BF084607EE100AB8EEC5
:10718800C77A012A8CED007A3FF4D5AA98ED047AE3
:10719800DDED0D6A25EE877AA6EE867AF0EE676A4F
:1071A800E7EE056ABDEEE67A17EE106A17EE100AEA
:1071B8009E42A8BF1846B142C8BF084607EE100A4B
:1071C800B8EEC77A022A8CED017A3FF4B4AA98ED9A
:1071D800087ADDED0E6A25EE877AA6EE867AF0EE5D
:1071E800676AE7EE056ABDEEE67A17EE106A17EEF3
:1071F800100A9E42A8BF1846B142C8BF084607EE0B
:10720800100AB8EEC77A032A8CED027A3FF493AAE3
:1072180098ED0C7ADDED0F6A25EE877AA6EE867A70
:10722800F0EE676AE7EE056ABDEEE67A17EE106AD9
:1072380017EE100A9E42A8BF1846B142C8BF0846BA
:1072480007EE100AB8EEC77A042A8CED037A3FF4E9
:1072580072AA98ED107ADDED106A25EE877AA6EE0F
:10726800867AF0EE676AE7EE056ABDEEE67A17EE13
:10727800106A17EE100A9E42A8BF1846B142C8BF4E
:10728800084607EE100AB8EEC77A052A8CED047A8C
:107298003FF451AA98ED147ADDED116A25EE877A4C
:1072A800A6EE867AF0EE676AE7EE056ABDEEE67A44
:1072B80017EE106A17EE100A9E42A8BF1846B14290
:1072C800C8BF084607EE100AB8EEC77A062A8CED42
:1072D800057A3FF430AA98ED187ADDED126A25EEAA
:1072E800877AA6EE867AF0EE676AE7EE056ABDEE63
:1072F800E67A17EE106A17EE100A9E42A8BF1846E3
:10730800B142C8BF084607EE100AB8EEC77A072A86
:107318008CED067A3FF40FAA98ED1C7ADDED136A1E
:1073280065EE875AE6EE265AE5EE257AFDEEE77A0F
:1073380017EE900A8342A8BF03468142C8BF0B4696
:1073480007EE903AF8EEE77ACCED077A002A7FF458
:10735800F2A9FFF7F5B91B4B5A79002A3EF481AC24
:10736800194A1278002A3EF47CAC1B78DFED174AE4
:1073780007EE903A164BB8EE677A1B8807EE902A0C
:1073880006EE903AF8EEE77AF8EE666A67EE277A44
:10739800B7EE007AC7EEA63AF4EEE43AF1EE10FA48
:1073A80088BFF0EE643AF4EEC73AF1EE10FAB8BFCF
:1073B800F0EE473AFEF757BCB0EE677AF6E400BF46
:1073C800A0460020283A0020BA460020713DAA3F76
:1073D8000C460020DC2A0020BCF1000F00F0978347
:1073E800BEF1000F41F08A87DFF8A485B9F1000FDC
:1073F80041F0E285D8ED006ADDED0C4ADFF894C56E
:1074080065EEA66ABDEEC77A17EE101AB0EE667A78
:10741800A4EE867AF0EE676AE7EE056ABDEEE67AD4
:1074280017EE106A17EE100A9E42A8BF1846B1421E
:10743800C8BF084607EE100AB8EEC77A012A8CEDD5
:10744800007A3FF478A998ED047ADDED0D6A25EE0F
:10745800877AA6EE867AF0EE676AE7EE056ABDEEF1
:10746800E67A17EE106A17EE100A9E42A8BF184671
:107478008E42B8BF084607EE100AB8EEC77A022A4D
:107488008CED017A3FF457A998ED087ADDED0E6A84
:1074980025EE877AA6EE867AF0EE676AE7EE056A49
:1074A800BDEEE67A17EE106A17EE100A9E42A8BFE4
:1074B80018468E42B8BF084607EE100AB8EEC77ADB
:1074C800032A8CED027A3FF436A998ED0C7ADDEDAB
:1074D8000F6A25EE877AA6EE867AF0EE676AE7EEFF
:1074E800056ABDEEE67A17EE106A17EE100A9E429C
:1074F800A8BF18468E42B8BF084607EE100AB8EE75
:10750800C77A042A8CED037A3FF415A998ED107A0E
:10751800DDED106A25EE877AA6EE867AF0EE676AC8
:10752800E7EE056ABDEEE67A17EE106A17EE100A66
:107538009E42A8BF18468E42B8BF084607EE100AFA
:10754800B8EEC77A052A8CED047A3FF4F4A898EDD2
:10755800147ADDED116A25EE877AA6EE867AF0EECA
:10756800676AE7EE056ABDEEE67A17EE106A17EE6F
:10757800100A9E42A8BF18468E42B8BF084607EEBA
:10758800100AB8EEC77A062A8CED057A3FF4D3A81C
:1075980098ED187ADDED126A25EE877AA6EE867ADE
:1075A800F0EE676AE7EE056ABDEEE67A17EE106A56
:1075B80017EE100A9E42A8BF18468E42B8BF08466A
:1075C80007EE100AB8EEC77A072A8CED067A3FF460
:1075D800B2A898ED1C7ADDED136A65EE875AE6EEDF
:1075E800265AE5EE257AFDEEE77A17EE900A8342F1
:1075F800A8BF03468142D8BF194607EE901AF8EE95
:10760800E77ACCED077A002A7FF495A8FFF798B8B7
:10761800C74B93ED006AFFF791B9AB68002B3EF4B6
:10762800D7AF05F1500128469847FEF7D1BFC14BA7
:10763800C149D3F8EC30086844F620618B42A8BFF2
:107648000B46B3F57A7FB8BF4FF47A7399B2C00688
:10765800A4F81A11DBF8003041F1D982DB0400F1FB
:107668006B83B64BD3F800C0BCF932E0B44BB548D5
:10767800D3ED037AD4F81C31A0FB010188096421F9
:1076880091FBF0F11429BDEEE77A04EB4308A8BF9B
:10769800142101338B42C4F81C3117EE109AA4BF91
:1076A8000023C4F81C3104EB4303A8F82091B3F974
:1076B800203107EE103AB8EEC77A77EEC77AFDEEBA
:1076C800E77ACDED057ABDF9141081EAE173A3EBF1
:1076D800E173734502F37E809B4B19464FF07E534E
:1076E8000B60FEF788BF03F0B9FF0B90FDF7D3BF1F
:1076F800DFF8A48203F0B2FF944AD4F8E4311268A8
:10770800C4F8E401C31A9A1A0746A8F80430A8F87E
:107718000620FEF7B6B91E218748FBF79DF800281A
:107728003FF48FAC8A4B1B885A063FF58AAC94F815
:107738008431BB4242F0C380834BD4ED627A93ED2F
:10774800010AD4ED435A9FED836ADFED836A27EE81
:10775800E57A68EE277AA8EE007AE5EE807AB4EE4C
:10776800C67AF1EE10FA88BFB0EE467AB4EEE67A41
:10777800F1EE10FAF4EEC67AB8BFB0EE667AF1EE22
:1077880010FA88BFF0EE467AF4EEE67AF1EE10FAD7
:10779800B8BFF0EE667A84ED417AC4ED437A50E4DE
:1077A800B4F8F411914240F297856C496C4AD1EDD6
:1077B800007A92ED007A6B49C4ED7E7A77EE676ABB
:1077C800C4ED7C7A0122C4ED7B6A84ED7F7AD1ED29
:1077D800006ADFED657A84F80022FEF782B9FDEED3
:1077E800C87ADFF8B48117EE903AA8F80490A8F8A0
:1077F800063021E45D4B1B88002B40F08C855C4AE9
:107808005C4B11781868FAF7FBF9D4F8D421089B77
:107818009A1AFEF73AB89FED4F7ADFED4F6ADFF814
:107828007881F4EEC77AF1EE10FA98BFB0EE677A75
:10783800FDEEE77AB4EEE67AF1EE10FA17EE902A4A
:10784800B8BFB0EE667A012984ED427AA8F8022022
:107858003FF774ABFFF7F0BBB4EEC87AF1EE10FA5D
:1078680098BFB0EE478ABDEEC77AB4EEE68ADFF875
:107878002881F1EE10FA17EE102AB8BFB0EE668A2A
:1078880084ED418AA8F8002000297FF4EFAAFFF7C9
:10789800D3BBBDEEE77ADFF8008117EE103AA8F8FF
:1078A8000430FFF7B1BB03F0D9FEDFF8EC80324BB0
:1078B800801B1B78A8F80400FFF7D6BB2F4A304975
:1078C800D2ED006A2F4A91ED006A1278C4ED7E6A03
:1078D80084ED7F6A002A40F0E68476EEC65AF0EE20
:1078E800466ABCEEC76A2849C4ED7B5A16EE102AD0
:1078F800C4ED7C6AA4F8F421FF22D1ED006A84F873
:10790800002277EEC77AFEF7ECB8DFED206AFFF7C2
:1079180090BAB5EEC07AF1EE10FA00F13D86B7EEF6
:10792800006A36EE477AC6EE076AFFF7EBBA00BF81
:10793800044A0020FC0000200C2B0020684B00208B
:10794800BC460020D34D621078000020DC2C0020BB
:107958001639002000C0F94400C0F9C4F44A0020D8
:10796800882C0020104B002000000000AC6F002085
:10797800AE6F0020B06F00209C460020302B002006
:10798800F84A0020B05300200C4B00200000C842E9
:10799800744A0020DC2A0020A046002098ED016AE5
:1079A80026EE646AB0EE674AA6EE074AB4EEC45AF9
:1079B80034EE666AF1EE10FAC8BFB0EE656A012BC4
:1079C8008CED006A3EF4BCAE98ED056A26EE646A5A
:1079D800B0EE674AA6EE074AB4EEC45A34EE666AB9
:1079E800F1EE10FAC8BFB0EE656A022B8CED016AA1
:1079F8003EF4A6AE98ED096A26EE646AB0EE674AD0
:107A0800A6EE074AB4EEC45A34EE666AF1EE10FAEE
:107A1800C8BFB0EE656A032B8CED026A3EF490AEE7
:107A280098ED0D6A26EE646AB0EE674AA6EE074A3C
:107A3800B4EEC45A34EE666AF1EE10FAC8BFB0EE7E
:107A4800656A042B8CED036A3EF47AAE98ED116AF0
:107A580026EE646AB0EE674AA6EE074AB4EEC45A48
:107A680034EE666AF1EE10FAC8BFB0EE656A052B0F
:107A78008CED046A3EF464AE98ED156A26EE646AED
:107A8800B0EE674AA6EE074AB4EEC45A74EE666AC8
:107A9800F1EE10FAC8BFF0EE656A062BCCED056A68
:107AA8003EF44EAED8ED196A66EEE46AB0EE674A67
:107AB800A6EE874AB3EE046AB4EEC45A74EE466A78
:107AC800F1EE10FAC8BFF0EE656A072BCCED066A36
:107AD8003EF436AED8ED1D6A66EEE44AE4EE877AE7
:107AE800F4EEC57A77EEC67AF1EE10FAB8BFF0EE8A
:107AF800657ACCED077AFEF723BE97F82030C3EB02
:107B0800431103EB8103DB009BB2FEF780BDDFF876
:107B18000485B9F1000F41F0E580D8ED006ADDED8C
:107B28000C4ADFF8F4C465EEA66ABDEEC77A17EE14
:107B3800101AB0EE667AA4EE867AF0EE676AE7EE7F
:107B4800056ABDEEE67A17EE106A17EE100A9E4235
:107B5800A8BF1846B142C8BF084607EE100AB8EEDB
:107B6800C77A012A8CED007A3EF452AB98ED047A7C
:107B7800DDED0D6A25EE877AA6EE867AF0EE676A65
:107B8800E7EE056ABDEEE67A17EE106A17EE100A00
:107B98009E42A8BF18468E42B8BF084607EE100A94
:107BA800B8EEC77A022A8CED017A3EF431AB98ED33
:107BB800087ADDED0E6A25EE877AA6EE867AF0EE73
:107BC800676AE7EE056ABDEEE67A17EE106A17EE09
:107BD800100A9E42A8BF18468E42B8BF084607EE54
:107BE800100AB8EEC77A032A8CED027A3EF410AB7D
:107BF80098ED0C7ADDED0F6A25EE877AA6EE867A87
:107C0800F0EE676AE7EE056ABDEEE67A17EE106AEF
:107C180017EE100A9E42A8BF18468E42B8BF084603
:107C280007EE100AB8EEC77A042A8CED037A3EF400
:107C3800EFAA98ED107ADDED106A25EE877AA6EEA8
:107C4800867AF0EE676AE7EE056ABDEEE67A17EE29
:107C5800106A17EE100A9E42A8BF18468E42B8BF97
:107C6800084607EE100AB8EEC77A052A8CED047AA2
:107C78003EF4CEAA98ED147ADDED116A25EE877AE6
:107C8800A6EE867AF0EE676AE7EE056ABDEEE67A5A
:107C980017EE106A17EE100A9E42A8BF18468E42C9
:107CA800B8BF084607EE100AB8EEC77A062A8CED68
:107CB800057A3EF4ADAA98ED187ADDED126A25EE44
:107CC800877AA6EE867AF0EE676AE7EE056ABDEE79
:107CD800E67A17EE106A17EE100A9E42A8BF1846F9
:107CE8008E42B8BF084607EE100AB8EEC77A072AD0
:107CF8008CED067A3EF48CAA98ED1C7ADDED136AB9
:107D080065EE875AE6EE265AE5EE257AFDEEE77A25
:107D180017EE900A8342A8BF03468142D8BF19468E
:107D280007EE901AF8EEE77ACCED077ABEF1000F6D
:107D38007EF406ADFEF770BAAA4BD3F800C0BCF8C3
:107D480032E04FEA5E0E91E4DFF8D092D4ED017A8A
:107D580094ED006AB9F80000D9F8143077EEA77AE4
:107D6800F0EE006AB0EE677AA6EE267A013804EBE8
:107D7800C002D6EE267A083A1033F6EE003A27EE1D
:107D8800237A67EEA37A84ED207AC4ED217A964CA3
:107D9800A64604F1800192ED027A92ED036ADEEDC7
:107DA800036ADEED027A53ED014A13ED025A37EE0B
:107DB800674A76EEC65A77EE277AE4EE845A013897
:107DC800A2F10802E5EE047A0EF1080E03F10803A9
:107DD80036EE267A01F10801E4EE877AE5EE475A95
:107DE80067EEA37A25EEA37AC1ED007A81ED017AD8
:107DF800D1D1142F7DF4D1AB03F030FC069BDFF812
:107E08002082C01AA8F80200D4F8A861FDF7C5BB03
:107E1800D4F8AC81B4F8A4A1744BCAF120095FFA74
:107E280089F90AEB481E03EB8E0E5FEA990301F00D
:107E38001B85013318016E496E4A0EEB000C0EF1DA
:107E4800100313ED024A13ED035A13ED016A13ED03
:107E5800047A51ED024A51ED035A51ED016A51ED90
:107E6800047A64EE244A65EE255A66EE266A67EEC1
:107E7800277A10339C4542ED024A42ED035A42EDFF
:107E8800016A42ED047A01F1100102F11002D8D121
:107E98005949A0F11002964401EB020C224419F052
:107EA800030309D0BEEC017AFCEC017A67EE277A6D
:107EB800013BE2EC017AF5D1BAF1000F41F0BF8144
:107EC800142F7DF46AAB03F0C9FB069BDFF85081E1
:107ED800D4F8A861C01AA8F80200FDF75EBBDFF865
:107EE8003C914148D9F80820B9F80C1022F0FEFF5F
:107EF800424B1F78142F01F08D85D4F8A861013604
:107F0800C4F8A86122E7D4F8AC913D4B3D4ADFEDB7
:107F18003E7AD2ED008A3D4A4FEAC9010B44F8EE99
:107F2800688A9B8809EE103A643BC82BA8BFC8230F
:107F380068EEA78AF8EE497A782BB8BF782368EEFE
:107F4800A78A07EE903A4944B0EE680A02EB810826
:107F5800B8EEE78A23F0C2FFB8EEC99AF0EE409A6D
:107F6800B0EE680A23F01CFF38EE097A79EE487AF9
:107F780028EE098A67EE877AB7EE006A88EE277AD4
:107F8800142FF8EE007A77EE076A60EE277A89EE0A
:107F9800A67A77EE065A36EE477AC6EE256A67EE77
:107FA800A67A27EE267AC8ED006A88ED047AC8ED2D
:107FB800026AC8ED017AC8ED037A01F07D85144B99
:107FC8000E4A09F1010983FB0938A8EBE97808EBA7
:107FD80048080136A9EB08081778C4F8A861C4F85E
:107FE800AC8117E7684B0020A8200020AC3E002099
:107FF8003C400020B82000202C4000209C46002057
:10800800AC4000207C51002027D4D23618720020C2
:1080180056555555744A0020DC2A0020943E00200D
:10802800A0460020DFF84493B9F800E0D9F804C06E
:108038004FEA5E084FEA880204EB8E065FEADE0E1E
:1080480004EB020300F0A08010320EF1010EBB48D1
:1080580003EB0E1E324410330CF1100706F1100129
:1080680051ED032A51ED043A10ED043A10ED032ABC
:1080780051ED026A11ED016A10ED020A10ED018A54
:1080880012ED044A12ED035A53ED044A53ED035A14
:1080980013ED027A53ED017A52ED020A12ED011A3C
:1080A80073EE238A72EE221A40ED048A40ED031A19
:1080B80070EE268A78EE061A40ED028A40ED011A23
:1080C80074EE848A75EE851A43ED048A43ED031A2B
:1080D80077EE208A77EE811A43ED028A43ED011A82
:1080E80073EE633A75EE655A17ED035A32EE623A4B
:1080F80074EE644A65EE631A17ED044A23EE052A06
:1081080064EE652AE3EE041A10339E4524EE843AA1
:10811800A3EE842A00F1100007F11007A5EE853AB6
:1081280001F1100102F11002E4EE852A41ED071A6F
:1081380001ED082A02ED073A42ED082A57ED055AE3
:1081480017ED065A70EE666A38EE466A30EEC77A60
:1081580071EE677A26EE253A65EEE63A25EE674A2D
:1081680067EE054AE6EE053AA6EE853AA7EE254AF9
:10817800E7EEA54A01ED063A41ED053A02ED064A59
:1081880042ED054A7FF46CAF1FFA88F86246414613
:108198006B481DF0B9FC4146D9F8042030461DF063
:1081A800B3FC684B1B78142B7FF42EAE24E6DFF863
:1081B800C09199F80020900801F0E584DFF8B4C177
:1081C80000F101084FEA48180CEB080E0CF12003E7
:1081D800ACF1700113ED076A53ED056A13ED037AEC
:1081E80053ED017A53ED025A13ED084A53ED064A4E
:1081F80013ED045A26EE066A66EEA66A27EE077A9B
:1082080067EEA77AA4EE046A20339E45E4EEA46ADA
:1082180001F11001A5EE057AE5EEA57AF1EEC65A50
:10822800B1EEE66AF1EEC76AB1EEE77A41ED085AB7
:1082380001ED076A41ED066A01ED057ACAD1A8F198
:108248002008C44404EB001012F0030318BF0CF11B
:10825800080C0FD05CED017A1CED027A67EEA77A64
:10826800013BE7EE077A0CF1080CB1EEE77AA0ECD7
:10827800017AEFD1142F01F02D840136C4F8A861DA
:10828800FDF7F4B803F0EAF92E4B06901F78142F87
:1082980005BFDFF8E480D4F8A861D4F8A861A8F88D
:1082A8000060FDF7C8B876EE665AFFF71ABB264A93
:1082B800D9ED007A92ED007AF0EEE77AF4EEC77A1B
:1082C800F1EE10FA7DF5B4AB01220899C4F8D41187
:1082D80084F8D021FEF783B81C4A1D49D2ED007AF4
:1082E8001C4A91ED007A1278C4ED7E7A84ED7F7A8B
:1082F800002A01F0698277EE676A1749C4ED7C7A33
:10830800C4ED7B6AFF22D1ED006ADFED147A84F8B0
:108318000022FDF7E6BB12494B69002B3DF4B5AAD4
:108328001048114B008893FBF0F00B684FF0010EDA
:10833800186081F811E0FDF7A8BA00BFB820002046
:10834800A82000209C4600203C4A0020302B00201A
:10835800F84A0020B05300200C4B00200000000019
:10836800B46F0020CC6F002020A10700943E0020AD
:108378008E3E002028210020A0460020D04EDFF8A5
:10838800749396ED004A96ED057AD6ED014A96ED7E
:10839800066AD6ED046A96ED035AD6ED025A67EEE0
:1083A800897A09EB8703A4EE277AA4EEA76A66EE1A
:1083B800C76AA5EE476AE5EEA76A20EE070A86EDCA
:1083C800056AC6ED066A83ED007A29EE088A23F06D
:1083D80039FD69EE288AD6ED0E5AD6ED176A96ED64
:1083E800091AD6ED121A96ED0F5A96ED187A96EDEF
:1083F8000A2AD6ED132A96ED0D6AD6ED167A96ED71
:108408000C3AD6ED0B3A96ED154AD6ED144AE1EE44
:10841800085A002209EB8703E8EEA16A00B2C4F803
:108428009421A2EE085AC4F89821C4F89C21A8EE19
:10843800A27A26EE656A67EEE67AA3EE655AA3EE9F
:10844800886AA6EEC47AE8EEA47A86ED0E5AC3EDE1
:10845800205A86ED0F6AC3ED406A86ED177AC6ED9D
:10846800187AFEF74DBC97494A69002A3DF43EAA9E
:108478000A6813604B74FDF739BAB5F93C306A6283
:1084880007EE903A0122F8EEE77AEB66C5F8882005
:108498000023012FC5ED1F7AC5ED1E7AC5F880307F
:1084A80001F0BE81B7427DF40BAFB5F93E302B67C2
:1084B80007EE903A00220123F8EEE77AAA62C5F89F
:1084C8009C300023012FC5ED247AC5ED237AC5F829
:1084D800943001F0A181B7427DF422AFB5F9403064
:1084E8006B6707EE903A00220123F8EEE77AEA621A
:1084F800C5F8B0300023012FC5ED297AC5ED287ADB
:10850800C5F8A8307DF43CAF9FED6F8AB9F1030F31
:1085180046D0BAF1000F09D007EE90AAF8EEE77A34
:10852800F4EEC87AF1EE10FA01F17883674A6B6FBE
:10853800126894F8B011A8F8060003EB560393FBF1
:10854800F6F60023EE6293621363D36231B1604B97
:108558001B8823F48063002B7DF414AF5D4B1B68EC
:1085680013F4003341F050815B491A46C85C012876
:1085780003F10C0300F0FC840132152AF6D1FDF753
:1085880001BF564B9B7B002B3EF4FFA9FEF726B894
:10859800F7EE006AFEF732BDF7EE006AFEF7B2BCEE
:1085A800B0EE480A23F04EFC00B2B2E7B4F84891A6
:1085B80009F1FF390FFA89F9B9F1000FA4F84891C8
:1085C8007EF7CDAB464BFEF776B8B4F81A3103F513
:1085D8007A739BB2FEF71BB8DFF81C8198F800206D
:1085E800013A0A2A1DD8DFE812F0C2005801020138
:1085F8003C011C001C00EC00AE00890054000B007C
:10860800384A394952680968C8328A4203D320F087
:1086180005FC30B1BB78032B01F03483012388F8C3
:108628000030FB78002B3EF417AD304B1B78D80791
:1086380040F1A680DFF8B090D4F89021D9F8003046
:108648009A4200F2A98098F80030012B3EF404AD5C
:1086580094F88C21002A3EF4FFAC0B2B0DD8012294
:108668009A4040F6030112EA01070DD112F4C06FD7
:1086780003D0093B012B41F2DE831A4BD9F80020C5
:108688005A600B2388F80030002384F88C31FEF7F9
:10869800E3BC174B1B78002B01F02C821A2011F039
:1086A800F5FC002841F0268294F88C31002B41F02B
:1086B8002182092388F800300BF024F8B1E700BFC5
:1086C80030410020B46F002000000000CC3B0020A7
:1086D800EC6E0020503600208CF402082C5E00203E
:1086E800BC4600208C2C0020D46F00202E5A00207D
:1086F800482D0020AC3E0020B34C00201A2011F079
:10870800C5FC0028D8D0AB4B1B88002BD4D1AA4B72
:108718004520D3F8009020F0A5FB0E2020F0A2FB06
:1087280048460AF06DFCDDF8209048460AF068FCDF
:10873800A24AA34B12681A6048460A2388F80030F8
:108748000AF032FDB8E720F049FB0BF011F80028D9
:108758003FF467AF20F062FB00283FF462AF974A0E
:10876800974B12681A600A2388F8003059E7954B2E
:108778001B78DB0701F17582FB78002B3EF46CACAB
:1087880017F07EFA00283FF455AF8F4B1B6803F5AE
:108798009C530833C4F8903198F80030012B7EF4CC
:1087A8005BAC94F88C31002B7EF456ACBB78032B71
:1087B80001F04F830BF094FD012384F88C31FEF710
:1087C8004BBC20F00BFB814B002105208DE80300FA
:1087D800A3F10802029153200BF0B8FC00287FF4A3
:1087E80020AF7B4A0823106088F8003019E7DFF8CB
:1087F800E09120F0F3FA744AD9F80430126864332F
:108808009342BFF40EAF402020F0CCFA00287FF44A
:1088180008AFD9F80030DFF8E0B16E494FF0400AF0
:108828000FE0059120F01EFB0599D9F800300A6881
:108838000133013ABAF1010A0A60C9F8003001F0BF
:1088480033821BF803301846002BEAD100234FF07F
:10885800FF32C9F800300423C9F8042088F8003032
:10886800DFE620F0BBFA5C4A0292A2F10C03252154
:1088780001930091A2F10A035021163A49200BF006
:1088880065FC00287FF4CDAE514B4FF0FF31072235
:108898001860596088F80020C3E64B4B4C4A1B68A7
:1088A80053604C490023136003220B6088F80020B2
:1088B800B7E64A4ADFED4A7A92ED080A0593B4EE24
:1088C800E70AF1EE10FA40F2B68423F051FBD4ED3A
:1088D800457A20EE270A23F0B5FAB0F5617F059BAB
:1088E80000F3438607EE900AF8EEE76ADFED3D7A7B
:1088F80066EEA76A07EE903AB8EEE77AFDEEE67AFA
:1089080017EE903A2033402B41F2F9809FED360A5A
:1089180023F098FA00B207EE900AB8EEE77A334BE4
:10892800D3ED037A77EE877AC3ED037AFDF75EBE5F
:108938000A9B93F800E00EF0010EBEF1000F7DF4E3
:10894800FFAEFDF769BC2A4BDFED2A7A1E68C4ED3D
:10895800707A16F0805640F0238310F4800600F0F9
:10896800B7810026B6EE007A67EE877AF4EEE75A0A
:10897800F1EE10FA48BFF0EE675A40F11183C4EDEA
:10898800815AFDF7EFBA02F069FE0646FDF718BEF8
:1089980074EE667AB7EE007AF4EEC77AF1EE10FA62
:1089A800C4ED707A40F3258784EEA77A8DED0C7AB2
:1089B800FDF7CEBA1C2B0020182B0020002B00201E
:1089C800FC2A00202E5A0020D46F0020D8E4020888
:1089D8008C2C0020AC6E00202AE30208A848002056
:1089E8008FC2753CD06D393A00000000BC460020AB
:1089F8000C2B002000000080C4E20208BAF1000F2E
:108A080000F0CD8598ED007ADDED0C6ADFF8E8C856
:108A180025EE877AA6EE867AF0EE676AE7EE056AB3
:108A2800BDEEE67A17EE106A17EE100A9E42A8BF4E
:108A38001846B142C8BF084607EE100AB8EEC77A12
:108A4800012A8CED007A3DF47BAE98ED047ADDEDD9
:108A58000D6A25EE877AA6EE867AF0EE676AE7EE6B
:108A6800056ABDEEE67A17EE106A17EE100A9E4206
:108A7800A8BF1846B142C8BF084607EE100AB8EEAC
:108A8800C77A022A8CED017A3DF45AAE98ED087A3D
:108A9800DDED0E6A25EE877AA6EE867AF0EE676A35
:108AA800E7EE056ABDEEE67A17EE106A17EE100AD1
:108AB8009E42A8BF1846B142C8BF084607EE100A32
:108AC800B8EEC77A032A8CED027A3DF439AE98EDF8
:108AD8000C7ADDED0F6A25EE877AA6EE867AF0EE3F
:108AE800676AE7EE056ABDEEE67A17EE106A17EEDA
:108AF800100A9E42A8BF1846B142C8BF084607EEF2
:108B0800100AB8EEC77A042A8CED037A3DF418AE41
:108B180098ED107ADDED106A25EE877AA6EE867A52
:108B2800F0EE676AE7EE056ABDEEE67A17EE106AC0
:108B380017EE100A9E42A8BF1846B142C8BF0846A1
:108B480007EE100AB8EEC77A052A8CED047A3DF4D0
:108B5800F7AD98ED147ADDED116A25EE877AA6EE69
:108B6800867AF0EE676AE7EE056ABDEEE67A17EEFA
:108B7800106A17EE100A9E42A8BF1846B142C8BF35
:108B8800084607EE100AB8EEC77A062A8CED057A71
:108B98003DF4D6AD98ED187ADDED126A25EE877AA8
:108BA800A6EE867AF0EE676AE7EE056ABDEEE67A2B
:108BB80017EE106A17EE100A9E42A8BF1846B14277
:108BC800C8BF084607EE100AB8EEC77A072A8CED28
:108BD800067A3DF4B5AD98ED1C7ADDED136A65EEC5
:108BE800875AE6EE865AE5EE257AFDEEE77A17EE25
:108BF800902A9342A8BF13468A42A8BF194607EE97
:108C0800901AF8EEE77ACCED077AFDF799BDD8000F
:108C18003EF524ADFDF7EFBC012A40F3018607EECF
:108C2800101AB8EEC77AC7EE876AB1EEE68AB9F1CC
:108C3800030F13D0BAF1000F09D007EE90AAF8EE8F
:108C4800E77AF4EEC87AF1EE10FA00F1E787EB6EF6
:108C580003EB560393FBF6F36B6223E4B0EE480A8A
:108C680023F0F0F800B2E5E7012A7FF74DAC07EEF4
:108C7800101AB8EEC77AC7EE876AB1EEE68A45E4FD
:108C8800012A40F3C98507EE101AB8EEC77AC7EE75
:108C9800876AB1EEE68AB9F1030F13D0BAF1000F73
:108CA80009D007EE90AAF8EEE77AF4EEC87AF1EE6A
:108CB80010FA00F1B3872B6F03EB560393FBF6F31F
:108CC800AB6208E4B0EE480A23F0BCF800B2E5E76E
:108CD800B6EE007AF4EEC75AF1EE10FA3FF742AE5C
:108CE800FDF740B9D8ED004A9DED0C4ADFF808C6FB
:108CF80065EEA44AFDEEC73AE4EE064AB0EE674ACE
:108D0800A4EE854A13EE901AF4EEC46AF1EE10FA56
:108D1800F0EE444A88BFF0EE474AFDEEE44A14EE0E
:108D2800900A14EE906A9842A8BF1E468142C8BFB6
:108D38000E4604EE906AF8EEE44A012ACCED004AA9
:108D48003DF466AAD8ED044A9DED0D4A65EEA44AA5
:108D5800E4EE064AB0EE674AA4EE854AF4EEC46A29
:108D6800F1EE10FAF0EE444A88BFF0EE474AFDEE05
:108D7800E44A14EE900A14EE906A9842A8BF1E4680
:108D88008842B8BF0E4604EE906AF8EEE44A022A1A
:108D9800CCED014A3DF43CAAD8ED084A9DED0E4AB7
:108DA80065EEA44AE4EE064AB0EE674AA4EE854AA8
:108DB800F4EEC46AF1EE10FAF0EE444A88BFF0EE21
:108DC800474AFDEEE44A14EE900A14EE906A98427F
:108DD800A8BF1E468842B8BF0E4604EE906AF8EE59
:108DE800E44A032ACCED024A3DF412AAD8ED0C4A13
:108DF8009DED0F4A65EEA44AE4EE064AB0EE674AD6
:108E0800A4EE854AF4EEC46AF1EE10FAF0EE444A94
:108E180088BFF0EE474AFDEEE44A14EE900A14EEDD
:108E2800906A9842A8BF1E468842B8BF0E4604EE14
:108E3800906AF8EEE44A042ACCED034A3DF4E8A926
:108E4800D8ED104A9DED104A65EEA44AE4EE064AB4
:108E5800B0EE674AA4EE854AF4EEC46AF1EE10FA61
:108E6800F0EE444A88BFF0EE474AFDEEE44A14EEBD
:108E7800900A14EE906A9842A8BF1E468842B8BF6E
:108E88000E4604EE906AF8EEE44A052ACCED044A50
:108E98003DF4BEA9D8ED144A9DED114A65EEA44AE9
:108EA800E4EE064AB0EE674AA4EE854AF4EEC46AD8
:108EB800F1EE10FAF0EE444A88BFF0EE474AFDEEB4
:108EC800E44A14EE900A14EE906A9842A8BF1E462F
:108ED8008842B8BF0E4604EE906AF8EEE44A062AC5
:108EE800CCED054A3DF494A9D8ED184A9DED124AF7
:108EF80065EEA44AE4EE064AB0EE674AA4EE854A57
:108F0800F4EEC46AF1EE10FAF0EE444A88BFF0EECF
:108F1800474AFDEEE44A14EE900A14EE906A98422D
:108F2800A8BF1E468842B8BF0E4604EE906AF8EE07
:108F3800E44A072ACCED064A3DF46AA9D8ED1C4A52
:108F48009DED134A65EEA45AE6EE045AE5EE257A3D
:108F5800F4EEE76AF1EE10FAC8BFF0EE477AFEF7D2
:108F6800D5BE8223FCF705BBDFEDE07AFCF7CCBA6F
:108F7800D4F8B46153003EB1981801EB80007678BC
:108F88004078B042BDF4FEA9134401EB83010023ED
:108F9800C4F8B411A4F80832C4F80C32FDF7F2B9D9
:108FA800B7EE007A77EE677AF4EEE75AF1EE10FA48
:108FB80088BFF0EE675AE2E4D8ED004A9DED0C4A0E
:108FC800DFF834C365EEA44AFDEEC73AE4EE064A7C
:108FD800B0EE674AA4EE854A13EE901AF4EEC46A1E
:108FE800F1EE10FAF0EE444A88BFF0EE474AFDEE83
:108FF800E44A14EE900A14EE906A9842A8BF1E46FE
:109008008142C8BF0E4604EE906AF8EEE44A012A8F
:10901800CCED004A3DF48FABD8ED044A9DED0D4AE6
:1090280065EEA44AE4EE064AB0EE674AA4EE854A25
:10903800F4EEC46AF1EE10FAF0EE444A88BFF0EE9E
:10904800474AFDEEE44A14EE900A14EE906A9842FC
:10905800A8BF1E468842B8BF0E4604EE906AF8EED6
:10906800E44A022ACCED014A3DF465ABD8ED084A42
:109078009DED0E4A65EEA44AE4EE064AB0EE674A54
:10908800A4EE854AF4EEC46AF1EE10FAF0EE444A12
:1090980088BFF0EE474AFDEEE44A14EE900A14EE5B
:1090A800906A9842A8BF1E468842B8BF0E4604EE92
:1090B800906AF8EEE44A032ACCED024A3DF43BAB51
:1090C800D8ED0C4A9DED0F4A65EEA44AE4EE064A37
:1090D800B0EE674AA4EE854AF4EEC46AF1EE10FADF
:1090E800F0EE444A88BFF0EE474AFDEEE44A14EE3B
:1090F800900A14EE906A9842A8BF1E468842B8BFEC
:109108000E4604EE906AF8EEE44A042ACCED034ACF
:109118003DF411ABD8ED104A9DED104A65EEA44A16
:10912800E4EE064AB0EE674AA4EE854AF4EEC46A55
:10913800F1EE10FAF0EE444A88BFF0EE474AFDEE31
:10914800E44A14EE900A14EE906A9842A8BF1E46AC
:109158008842B8BF0E4604EE906AF8EEE44A052A43
:10916800CCED044A3DF4E7AAD8ED144A9DED114A26
:1091780065EEA44AE4EE064AB0EE674AA4EE854AD4
:10918800F4EEC46AF1EE10FAF0EE444A88BFF0EE4D
:10919800474AFDEEE44A14EE900A14EE906A9842AB
:1091A800A8BF1E468842B8BF0E4604EE906AF8EE85
:1091B800E44A062ACCED054A3DF4BDAAD8ED184A82
:1091C8009DED124A65EEA44AE4EE064AB0EE674AFF
:1091D800A4EE854AF4EEC46AF1EE10FAF0EE444AC1
:1091E80088BFF0EE474AFDEEE44A14EE900A14EE0A
:1091F800906A9842A8BF1E468842B8BF0E4604EE41
:10920800906AF8EEE44A072ACCED064A3DF493AAA0
:10921800D8ED1C4A9DED134A65EEA45AE6EE045AB1
:10922800E5EE257AF4EEE76AF1EE10FAC8BFF0EE43
:10923800477AFEF7D8B99FED2E7AFFF770BB2D4B12
:109248004FEA890E5FEA9A0901EB0E0C03EBC81886
:10925800A64400F0FF8409F101094FEA091908EB57
:10926800090008F110030CF110010EF1100213EDC2
:10927800024A13ED035A13ED016A13ED047A51ED16
:10928800024A51ED035A51ED016A51ED047A64EE38
:10929800244A65EE255A66EE266A67EE277A103369
:1092A800984242ED024A42ED035A42ED016A42ED0C
:1092B800047A01F1100102F11002D8D1A9F11009C4
:1092C800C8440CEB0901CE441AF0030A3EF4F8AD89
:1092D800B8EC017AF1EC017A67EE277ABAF1010A63
:1092E800EEEC017AF4D1FEF7EBBD00BF00000243BB
:1092F80000000000AC3E0020DC2A0020BAF1000F7C
:1093080000F09483DFF854869DED0C4AD8ED004AAE
:1093180065EEA44AE4EE064AB0EE674AA4EE854A32
:10932800F0EE444AB9F1000F06D0F4EE446AF1EECB
:1093380010FAC8BFF0EE474ABDEEC77A17EE101A0A
:10934800BDEEE47A04EE901A17EE100A814200F39B
:1093580071849842A8BF184607EE100AB8EEC77A7B
:10936800DFF8FCC5012A8CED007A3DF4E9A998EDF7
:10937800047A9DED0D4A25EE877AA4EE067AB0EEC2
:10938800674AA7EE054AB0EE447AB9F1000F00F03B
:109398003A84F4EEC46AF1EE10FA40F334840846D5
:1093A8009842A8BF184607EE100AB8EEC77A022AF4
:1093B8008CED017A3DF4C4A998ED087A9DED0E4A2A
:1093C80025EE877AA4EE067AB0EE674AA7EE054A3C
:1093D800B0EE447AB9F1000F00F00A84F4EEC46AE2
:1093E800F1EE10FA40F3048408469842A8BF1846E4
:1093F80007EE100AB8EEC77A032A8CED027A3DF41C
:109408009FA998ED0C7A9DED0F4A25EE877AA4EE78
:10941800067AB0EE674AA7EE054AB0EE447AB9F18B
:10942800000F00F0DB83F4EEC46AF1EE10FA40F3AB
:10943800D58308469842A8BF184607EE100AB8EE2A
:10944800C77A042A8CED037A3DF47AA998ED107A4C
:109458009DED104A25EE877AA4EE067AB0EE674AAB
:10946800A7EE054AB0EE447AB9F1000F00F0AC83DC
:10947800F4EEC46AF1EE10FA40F3A6830846984267
:10948800A8BF184607EE100AB8EEC77A052A8CED71
:10949800047A3DF455A998ED147A9DED114A25EE0C
:1094A800877AA4EE067AB0EE674AA7EE054AB0EED0
:1094B800447AB9F1000F00F07D83F4EEC46AF1EE4E
:1094C80010FA40F3778308469842A8BF184607EE7B
:1094D800100AB8EEC77A062A8CED057A3DF430A951
:1094E80098ED187A9DED124A25EE877AA4EE067A51
:1094F800B0EE674AA7EE054AB0EE447AB9F1000F1C
:1095080000F04E83F4EEC46AF1EE10FA40F348839B
:1095180008469842A8BF184607EE100AB8EEC77A60
:10952800072A8CED067A3DF40BA998ED1C7A9DED7F
:10953800134A65EE875AE4EE065AE5EE857AB9F1E4
:10954800000F00F02583F4EEE67AF1EE10FA40F110
:109558001F830A469A42A8BF1A4604EE902AF8EEDC
:10956800E44ACCED074AFDF7EBB807EE903ADFED99
:10957800EC6AB8EEE77A66EEA65A9FEDEA5A9FEDD6
:10958800EA6ADFEDEA7AA5EE856A26EEA55AE5EEE7
:10959800867AE5EE276A26EE870AFFF7B9B9D8ED8D
:1095A800006ADDED0C4A65EEA66AE4EE866AF0EE26
:1095B800674AE6EE854AFDEEE46A16EE90EA7145E2
:1095C80000F325829E45A8BF9E4606EE90EAF8EE77
:1095D800E66A002E00F02484DFF884C3012ACCED6B
:1095E800006A3DF4ADA8D8ED046ADDED0D4A65EEDC
:1095F800A66AE4EE866AF0EE674AE6EE854AFDEE74
:10960800E46A16EE90EA714500F31F819E45A8BFF3
:109618009E4606EE90EAF8EEE66A002E00F02C84EC
:10962800022ACCED016A3DF48BA8D8ED086ADDED7D
:109638000E4A65EEA66AE4EE866AF0EE674AE6EE42
:10964800854AFDEEE46A16EE90EA714500F3098159
:109658009E45A8BF9E4606EE90EAF8EEE66A002E02
:1096680000F0FF83032ACCED026A3DF469A8D8ED27
:109678000C6ADDED0F4A65EEA66AE4EE866AF0EE46
:10968800674AE6EE854AFDEEE46A16EE90EA714511
:1096980000F3E4809E45A8BF9E4606EE90EAF8EEE9
:1096A800E66A002E00F0A883042ACCED036A3DF494
:1096B80047A8D8ED106ADDED104A65EEA66AE4EE1B
:1096C800866AF0EE674AE6EE854AFDEEE46A16EE33
:1096D80090EA714500F3BF809E45A8BF9E4606EEFE
:1096E80090EAF8EEE66A002E00F07C83052ACCEDBD
:1096F800046A3DF425A8D8ED146ADDED114A65EE3B
:10970800A66AE4EE866AF0EE674AE6EE854AFDEE62
:10971800E46A16EE90EA714500F39A809E45A8BF68
:109728009E4606EE90EAF8EEE66A002E00F06E839A
:10973800062ACCED056A3DF403A8D8ED186ADDEDDC
:10974800124A65EEA66AE4EE866AF0EE674AE6EE2D
:10975800854AFDEEE46A16EE90EA714572DC9E4594
:10976800A8BF9E4606EE90EAF8EEE66A002E00F0E4
:10977800AF83072ACCED066A3CF4E2AFD8ED1C6A49
:10978800DDED134A65EEA65AE4EE865AE5EE857AD3
:10979800FDEEE77A17EE902A914203DC9A42A8BFC1
:1097A8001A46114607EE901AF8EEE77A002E7FF473
:1097B8002AAA069B002B7FF426AA059B5B45B8BF07
:1097C800F0EE477AFFF71FBA77EEC76AF0EE477AEE
:1097D800FEF793BDBCF834309FED557A07EE903A0A
:1097E800F8EEE77A534B67EE877AC3ED007AFCF719
:1097F80002BF514B1E6816F080567FF4B3A8FFF7DE
:10980800ACB84E4BFCF74EBF4D4B1B78032B00F00A
:1098180024820023FEF7A8BE9FED4A8AFFF73BBAD1
:109828009FED488AFFF703BA9FED470ADFF83481B6
:1098380025EE800A22F006FBD4F8A861A8F80600F5
:10984800FBF7ABBE06EE901A8EE706EE901AE2E63C
:1098580006EE901A67E706EE901A42E706EE901AAF
:109868001DE706EE901AF8E63849394A8C46FEF7A5
:1098780016BB93ED000A05930791069222F0E2FACF
:10988800DFF8E4E0DFF8E4C0DEF8ECE0DFF8D480ED
:10989800069AA8F800008CFB0E3C4FEAEE7ECEEB51
:1098A800AC1E07EE90EAF8EEE77A059B0799FDEE05
:1098B800E77A17EE900AA8F80200FCF7F8BE07EE60
:1098C800907AF8EEE78ADFED237A9FED2C0A84F888
:1098D800847168EEA78A38EE800AFDEEC07A17EE2A
:1098E800903A2033402B40F29F819FED160A114B8E
:1098F800FDEEE87A83ED010A17EE903A2033402B0B
:1099080000F29581DFED1E7AF4EEE78AF1EE10FAA7
:1099180040F3D481DFED176ADFED0F7A3AE000BF3C
:1099280084F9223F92E741B99730083C15A82ABE2E
:109938006F12833A780000200C2B0020BC460020D0
:109948001A390020000000000000C8422C40002006
:10995800A820002035FA8E3CE4CB1641744A00203A
:10996800DC2A0020A0460020FC000020D34D621015
:10997800DB0F49C0DB0FC940E4CB16C1DB0FC93F81
:10998800DB0F494092E741B99730083C15A82ABE39
:10999800F0EE478AF4EEE78AF1EE10FA38EEE67A4E
:1099A800F6DC5FED0D7AB4EEE77AF1EE10FA40F1ED
:1099B80082811FED106A5FED106A01E0B0EE677AF0
:1099C800B4EEE67AF1EE10FA77EE067AF6D41FEDE9
:1099D800157AF4EEC77AF1EE10FA40F32F811FEDF5
:1099E800187A77EE677A27EEA76A5FED1A5A5FED65
:1099F8001A6A1FED1A7AE6EE256A67EE865AA6EE0F
:109A0800267AE5EE877AC4ED627AFDF79ABE06EE0D
:109A1800901ADCE501F022FEDA4BDFF8B8831F78F4
:109A2800069BC01AA8F80200FEF767BAFDEEC74AFF
:109A38000DF1300E9A46DFF8A0C3DFF8A08314EECC
:109A4800901A0EEB82024B4606E07245E8EC014A9A
:109A58000CF1100C3CF474AEDCED004ABEEC014A8B
:109A680065EEA44AE6EE044AB0EE674AA5EE244A3B
:109A7800F0EE444A33B1F4EE446AF1EE10FAC8BF8E
:109A8800F0EE474AFDEEE44A14EE909A494504EE9A
:109A9800901A04DCD145A8BFD14604EE909AF8EE9E
:109AA800E44A002ED1D106980028CED10598584511
:109AB800B8BFF0EE474AC8E701F0D0FD069BDFF8D3
:109AC8001483D4F8AC91D4F8A861C01AA8F802009D
:109AD800FEF775BA01F0C2FDAA4BDFF8F8821F78CD
:109AE800069B99F80020D4F8A861C01AA8F80400C9
:109AF800FEF7C3BB089809F057FBFEF7DDBDDFEDA5
:109B0800A27AF4EEE76AF1EE10FA40F3DE81DFEDB7
:109B18009F5A9FED9F6A01E0F0EE676AF4EEC66A0D
:109B2800F1EE10FA76EEE57AF6DCDFED9A6AF4EEFD
:109B3800E67AF1EE10FA40F1C581DFED945A9FED17
:109B4800966A01E0F0EE667AF4EEC67AF1EE10FA63
:109B580077EEA56AF6D4DFED917AF4EEE76AF1EED6
:109B680010FA04DDDFED887A77EEE66A03E5DFEDCB
:109B78008C7AF4EEE76AF1EE10FA44BFDFED857AED
:109B880077EEE66AF7E4874800F1800CFEF75CBBE5
:109B9800FDEEE77A17EE902A8A42FFF6E0ACD9E4A8
:109BA800BDEEC77A17EE100A8842BFF6B2AC07EED0
:109BB800101AB3E4BDEEC77A17EE100A8842BFF652
:109BC80083AC07EE101A84E4BDEEC77A17EE100ACC
:109BD8008842BFF654AC07EE101A55E4BDEEC77ABA
:109BE80017EE100A8842BFF625AC07EE101A26E4D5
:109BF800BDEEC77A17EE100A8842BFF6F6AB07EE3D
:109C0800101AFFF7F7BBBDEEC77A17EE100A8842A5
:109C1800BFF6C6AB07EE101AFFF7C7BBA8F80600D9
:109C2800A5F8B460FCF7B6BBF8F73EFD5FE6DFEDDC
:109C38005E7AE8E607EE101AFFF790BB9FED587AB8
:109C4800F4EEC77AF1EE10FA44BF9FED527A77EE40
:109C5800677AC8E66146FFF737BB08F0CDFFFCF727
:109C680091BB80201DF05AFA08B108F07DFA0AF07D
:109C780037FBFEF7D6BC94F8E031002B7BF4F8AE46
:109C8800FBF7E3BEDFF85891D9F8000008F040FA76
:109C9800464B1B780022022BC9F800207EF4BEAC8C
:109CA80008F0DEFEFEF7BABC1BF80330002B7EF48A
:109CB800B8ACFEF7CBBDF0EE477A88E6B0EE687A2E
:109CC8006FE63B4A3B4B10681B689847099B9BED26
:109CD800007AD3ED007A384BD7ED006A83ED020A9B
:109CE800364B67EE277A2B4427EE8C7AD3ED007A31
:109CF800334B67EE277AF0EE665AEDEE275A93ED6E
:109D0800006AB1EE467AB4EEE57AF1EE10FA2EDD8D
:109D18002C4B1B78012B02D0192B7BF41EAEDFEDE8
:109D28002A7AB4EEE7DAF1EE10FACCBF0123002369
:109D3800FBF71EBE254BD3ED007AB1EE677AB4EE81
:109D4800C7DAF1EE10FA0FD4B4EEE7DAF1EE10FA52
:109D580088BFB0EE67DA1E4BC7ED00BA1B689342A6
:109D6800BBF6BCADFCF708BFB0EE47DAF3E7B4EEDC
:109D7800E56AF1EE10FA8CBFB0EE657AB0EE467A7D
:109D8800C6E700BF9C460020DB0F4940DB0FC940F7
:109D9800E4CB1641DB0F49C0E4CB16C1DB0FC93F4A
:109DA800DB0FC9BFA820002000000000D82C00202D
:109DB800B8490020CC490020602A0020DC49002056
:109DC800444A00206843002000009642404A002090
:109DD800244A0020A0460020744A0020DC2A0020E3
:109DE800B06E0020069800287FF480AC059858458E
:109DF800B8BFF0EE476A79E4069800287FF454ACBF
:109E080005985845B8BFF0EE476A4DE40698002813
:109E18007FF48EAC05985845B8BFF0EE476A87E4E2
:109E2800069800287FF4D8AB05985845B8BFF0EEDF
:109E3800476AFFF7D1BB45201FF014F8FF201FF039
:109E480011F828481EF0FAFF38461FF00BF8FEF705
:109E580014BC80201DF062F900287DF4FDA8FEF7EF
:109E6800A9BC069800287FF4FDAB05985845B8BFF3
:109E7800F0EE476AFFF7F6BB069800287FF4D0ABF0
:109E880005985845B8BFF0EE476AFFF7C9BB132BD2
:109E980005D1B0EE480A21F0D5FFAAF80000B0EECF
:109EA800480AD5F8143210489847104B1B78132BE2
:109EB800B0EE408A7BF4B2AB21F0C4FFAAF80200EE
:109EC800FBF7ACBBF0EE676A45E6F0EE667A2CE687
:109ED800069800287FF44DAC05985845B8BFF0EEB9
:109EE800476A46E4C8060308187200209C4600200A
:109EF8000B4B002210B4027203F1B404042102E0F7
:109F0800072A09DC9979890702D519798154013220
:109F18009C4203F11403F3D15DF8044B704700BF72
:109F28003C05030810B40D4C04232146002200E030
:109F38008B7913F0010301F1140106D101320A2AC9
:109F4800F6D103705DF8044B704702EB820204EB14
:109F580082025DF8044B1379037070473C050308CF
:109F68000123152122224170427103700371704749
:109F78002DE9F0410B78057BDB43DFB200F11302DA
:109F880000F11D0302F8015F9342FBD1DFF890E076
:109F980000F12701002203F8012F9942FBD1142177
:109FA8000524002647FA04F303F00103002B1E449E
:109FB80014BF4FF019084FF00A0814F0010FF6B259
:109FC80014BFAC464FF0000C0023CA1810FA82F2F6
:109FD8000133434582F814C0F7D15A1E92B20132B8
:109FE800013C8B18621C9BB201D01946DAE716F0C7
:109FF800010F14BF19240A240022991810FA81F1BC
:10A008000132A2420D75F8D113449BB25A1C034485
:10A01800002192B21975AEF800200261BDE8F08106
:10A02800BC2200202DE9F04FDFF890A0BAF80230EA
:10A038000B3383B01FFA83F901F1060B4FF00108C7
:10A048004FF0000C002711F801EB3E464C46012268
:10A05800A4F10B039BB2019105E001339BB2017B94
:10A0680029759C4208D0C518002AF6D1C5180133B5
:10A078009BB29C422A75F6D103190136092F019922
:10A0880083F814C0F6B20CD0092E15D008FA07F3DD
:10A0980013EA0E0F14BF012200220C34A4B20137B8
:10A0A800D6E709F1780959451FFA89F9CAD1AAF8FA
:10A0B80002C003B0BDE8F08F0022EEE7BC2200200A
:10A0C8002DE9F047DFF85C80B8F8043004331FFA54
:10A0D80083FC01F109094FF0010E11F8017B644678
:10A0E8000026231F0EFA06F29BB23A40C2B1B0F81E
:10A0F8000CA0C51801339BB29C4285F814A0F5D179
:10A1080001360434082EA4B2EBD10CF1200C4945D9
:10A118001FFA8CFCE1D10023A8F80430BDE8F087D1
:10A128009246E6E7BC220020436A8269D154436A1A
:10A138000169426B01338B4228BF00234362002A26
:10A148002FD0EFF31181502383F31288436B1A68E1
:10A15800D2072CD470B45E686EB9456A826A95429B
:10A1680017D084691444DC600ED9AA1A5A60856233
:10A17800002280F850201A6842F00102C9B21A6021
:10A1880081F3118870BC70470469A21A5A6086620C
:10A19800EEE7012380F85030C9B281F3118870BC12
:10A1A8007047C26C136843F0800313607047C9B2EC
:10A1B80081F31188704700BF026B10B462B1036C61
:10A1C800C2684469D11A013B615C5DF8044B08BF61
:10A1D80013460364C8B27047016A4369C4685B5C8C
:10A1E8000131A14228BF114601625DF8044BD8B283
:10A1F800704700BF436B13B190F850007047836AF3
:10A20800406A181AB0FA80F040097047416A836AB8
:10A2180099420AD3CB1A416B026961B14968501E51
:10A228000B4483420AD2C01A704702691144CB1A00
:10A23800416B0029F2D1501EC01A704700207047A8
:10A24800036B43B1026C5B6893422FBF981AC068D6
:10A258009B1AC0187047C269036A9A422FBFD01A66
:10A26800C0688018C01A70470A4B30B503F114044F
:10A2780093F900205D78072AC8BF143A811804337F
:10A288000D7313F8025C855413F8012C0A76A34267
:10A29800EED130BDF8E4020803682DE9F041DF692A
:10A2A8001FB13B46BDE8F0411847002A164611DDAC
:10A2B80004460D460E4400E023689B6820469847F4
:10A2C8000028F9D0236815F8011B1B682046984719
:10A2D800AE42F1D1BDE8F0812DE9F0470569C368C8
:10A2E8001D4028D00F4606464FF000484FF00009A1
:10A2F800B5FA85F328FA03F2D2431B3B32611540C5
:10A30800042B16D8DFE803F03129211903007B6AF2
:10A31800002B32D003F1FF3A1FFA8AFAC7F82490CB
:10A328003C6A34B123682046514698476468002C3B
:10A33800F8D1002DDCD1BDE8F0873868716B03686F
:10A3480089B29847002DD3D1F5E77868B16B0368D7
:10A3580089B29847002DCBD1EDE7B868F16B036857
:10A3680089B29847002DC3D1E5E7F868316C0368D6
:10A3780089B29847002DBBD1DDE7F36A1FFA83FA4B
:10A38800CEE700BF30B50446C06C61710368A268AF
:10A3980023F00103036087B0A379009213F004024D
:10A3A8003DD04FF4805213F00203019244D102933E
:10A3B8004FF480630022039311F00103059237D113
:10A3C800049308238D07694648BF04931BF0A8F837
:10A3D8006079E36CA17900F00202002A15BF4FF4FE
:10A3E80040324FF480324FF40034002410F0010F53
:10A3F800586808BF2246CC074CBF024320EA020235
:10A408005A609A6809074CBF42F0080222F0080215
:10A418009A601A6842F001021A6007B030BD13F062
:10A42800020301920BD04FF4005513460295C1E781
:10A43800042304930C23C5E74FF40053B7E70293B2
:10A44800B8E700BF10B50446C06CA160036823F0EC
:10A4580001030360A37986B013F00402009141D090
:10A468004FF4805213F00203019244D102934FF447
:10A47800806362790393D1074FF000030493059337
:10A4880045BF0423049308230C236946920748BF59
:10A4980004931BF045F86079E36CA17900F002029F
:10A4A800002A15BF4FF440324FF480324FF4003485
:10A4B800002410F0010F586808BF2246CC074CBF93
:10A4C800024320EA02025A609A6809074CBF42F028
:10A4D800080222F008029A601A6842F001021A6023
:10A4E80006B010BD13F00203019207D04FF40051DB
:10A4F80013460291BDE74FF40053B7E70293B8E75C
:10A508002DE9F04F013085B0C3B203938E4D8F4FC4
:10A518008F4C904E0A2302933220DFF840921FF0AE
:10A5280089FE4FF4FA7A4FF0100C4FF47A70D9F88C
:10A538000430C3F30803002B40F0C880EFF3118305
:10A54800002B40F0C3802968A26800BF2B6899429D
:10A55800F9D1D7F800E000FB0EF39B1AB3FBFEF32A
:10A5680000FB01314FF0010E0191D9F80430C3F31B
:10A578000803002B40F08E80EFF31183002B40F08E
:10A5880089802B68A16800BF2A689342F9D1D7F85F
:10A5980000B000FB0BF2521AB2FBFBF200FB0323E4
:10A5A800019A9B1AB3F57A7FDFD3BAF1010ABED1BB
:10A5B800039B002B40F0C4804FF47A7ADFF89C911B
:10A5C80050464FF0100CD9F80430C3F30803002BA1
:10A5D80040F09980EFF31183002B40F094802968B4
:10A5E800A26800BF2B689942F9D1D7F800E000FBB8
:10A5F8000EF39B1AB3FBFEF300FB01314FF0010E83
:10A608000191D9F80430C3F308033BBBEFF311837E
:10A6180023BB2B68A16800BF2A689342F9D1D7F8F9
:10A6280000B000FB0BF2521AB2FBFBF200FB032353
:10A63800019A9B1AB3F57A7FE3D3BAF1010AC2D122
:10A64800029B013B02937FF467AF4349434B444865
:10A65800444A0860DA6005B0BDE8F08FEFF311886E
:10A668008CF31288A1682368DB0344BFC6F800E0B6
:10A67800A1682B6832685FFA88F888F31188D7F8E0
:10A6880000801A4400FB08F35B1AB3FBF8F300FBE5
:10A698000233CDE7EFF311888CF31288A1682368A1
:10A6A800DB0344BFC6F800E0A1682B6832685FFA94
:10A6B80088F888F31188D7F800801A4400FB08F35B
:10A6C8005B1AB3FBF8F300FB023369E7EFF311827F
:10A6D8008CF31288D4F808E02368D90303D5012342
:10A6E8003360D4F808E02B683168D2B282F311885D
:10A6F8003A68194400FB02F3A3EB0E03B3FBF2F331
:10A7080000FB01312EE7EFF311828CF31288D4F8A5
:10A7180008E02368D90303D501233360D4F808E09F
:10A728002B683168D2B282F311883A68194400FB69
:10A7380002F3A3EB0E03B3FBF2F300FB01315DE779
:10A7480018461FF0F7FB37E7D46F0020D86F0020BA
:10A7580010E000E0D06F0020FC9F002000ED00E03A
:10A76800EFBEADDE0400FA0538B5434B5A89998926
:10A77800914224BF00225A81198ADA89914224BF62
:10A788000022DA81DA788AB3072A2FD03B493C4D78
:10A7980091F85700012400210A282C709C70D97167
:10A7A8003DD00C2865D0DFED377A8ABB364C9FED5B
:10A7B800370AA278002918BFF0EE407A062A04D892
:10A7C800334901EB820191ED050A217959B3013A28
:10A7D800032A4DD8F7EE007A87EE800A21F032FB83
:10A7E8002388984228BF1846208038BDD97921B1DE
:10A7F80098780428B8BF04209870204890F857002B
:10A808000A280CD00C28CED1DFED227A002ACDD030
:10A81800072ACBD00A282CD1DFED1F7AC6E70A20F9
:10A82800DFED1E7AC1E79B78154A07EE103A1178DA
:10A83800B8EEC77A27EE277A07EE901AF8EEE77A8D
:10A8480067EE877AB4EEE70AF1EE10FA10DDC0EE93
:10A85800077AFDEEE77A17EE903A102BA8BF10237F
:10A86800012BB8BF0123DBB28B4238BF0B461370F4
:10A8780038BDDFED0B7A99E76851002000700020A1
:10A88800AC2C00206F1203398C5300206F12033850
:10A89800F8E402080AD7A3390F506E3A5304E9388E
:10A8A8006F12833A2DE9F047B14FB24E11F04AFDCD
:10A8B800BE421ED2DFF84483DFF84493444625881D
:10A8C80062197DB14A450DD2052D0BD933886188AF
:10A8D800C3F30B03994200F0EF80144625886219F0
:10A8E800002DEFD1716830461436F7F703FBBE42EE
:10A8F800E4D3A14A1378A3F1170102290FD99F497C
:10A9080011F83300002840F00381D8000144497849
:10A9180029B19B4911F83330002B00F02181994B64
:10A928005A78022A40F2EE80002297495A701A7823
:10A938009648022A016000F2E18002EB8201944B02
:10A94800C2EBC10203EB4203998C5A8C914C9142A1
:10A95800236001D300225A848F4B9A78042A00F08E
:10A96800F68032B91A88B2F5F07F84BF4FF4F072DE
:10A978001A808A4DFFF7F8FE2B68894A1A40002A88
:10A9880000F0F180D80700F1DD80590400F1D5808E
:10A998001A0700F1CD809B0400F1C38017F08EFBED
:10A9A80010B9804807F000F88020F7F7D9FA4FF47B
:10A9B8000070F7F7D5FA4FF40030F7F7D1FA4FF4F3
:10A9C8008020F7F7CDFA4FF00070F7F7C9FA4FF08B
:10A9D8008060F7F7C5FA4FF00060F7F7C1FA0FF09B
:10A9E800CDFB00213022704823F037FB206814F09B
:10A9F80005FA6E4B266803F1500102E004339942D0
:10AA08007AD01A78002AF9D19C78D8788442F5D27D
:10AA18006749684B91F804E06748684D5C6B684B80
:10AA28002860C827642111FB0E71DFF8D8E159604E
:10AA3800644F30F8061C644DAEF800100021996090
:10AA4800D960196159619961D96183F8201083F837
:10AA580021103A702E600CB111F0D2FA5B4B9FEDC9
:10AA68005C5A1B885B4A9FED5C6A557B5B4C5C4972
:10AA78005C48086006EE903AF8EEE66A1389C5EE7F
:10AA8800265A07EE103A5389127BC4ED005A07EE96
:10AA9800903AB8EEC77A544BF8EEE77A1D725A72BC
:10AAA80027EE067A67EE867ABDE8F04783ED017AED
:10AAB800C3ED007A11F02EBC63799B077FF40DAFCC
:10AAC800716894F804A03046F7F714FA3388BAEBA3
:10AAD800133F04D01436BE42FFF4F0AE09E7738882
:10AAE8007068AA1FC3F30B039A4204F10601A8BFBA
:10AAF8001A4621F033F8EDE7012289E700221A709F
:10AB0800234B21E7204902EB420201EB82010EE7C9
:10AB1800D8000C186468002C7FF4F8AE1724147061
:10AB2800F4E63248F7F71CFA4020F7F719FA35E748
:10AB38002F48F7F715FA2B682DE72E48F7F710FA84
:10AB48002B6825E72C48F7F70BFA2B681DE79A8A3C
:10AB5800B2F57A7FBFF40DAF4FF47A729A8208E7A4
:10AB680018231370DBE643F400532B600AE700BF99
:10AB7800703B030860370308F42C002004FF020828
:10AB8800DCF90208564B00207E4C0020D03B002008
:10AB9800764B0020684B00208C530020E84C0020A6
:10ABA80009600002F85D002088230020F82C0020AE
:10ABB800144B0020842A0020BE2C0020F86D0020B1
:10ABC800C86E0020A4040020BC230020B821002067
:10ABD800C0C9FB48BC22002017B7D138BC210020CF
:10ABE800F44800203661023DD048002009400002A8
:10ABF80001600002092000020860000202F0030858
:10AC080000000408C041002038B50C4C0C4DAC4283
:10AC180006D2616820461434F7F76CF9AC42F8D3D1
:10AC2800084A094B094C1460002209491A705A70E5
:10AC380008480860BDE838401EF082BD6037030848
:10AC4800703B0308684B0020564B0020764B0020D1
:10AC5800D03B00207E4C0020F0B50C292BD8DFE833
:10AC680001F06F2A2A2A4C2A2A2A2B2A2A2A070084
:10AC7800046AB2F80CE097881668674D24F480548B
:10AC88000462036A4468C16923F4005343EA0E333B
:10AC980021F4E641A84243EA073341EA062100F0DD
:10ACA800B58005F50065A84200F0B0809268446060
:10ACB800C16102640362F0BD046A96899588D2F87E
:10ACC80000E0554F24F480740462036A4468C16943
:10ACD80023F4007343EA062321F07301B84243EAE0
:10ACE800052341EA0E017ED04C4DA8427BD09268E4
:10ACF8004460C161C2630362F0BD046A96899588A5
:10AD0800D2F800E0444F24F010040462036A446857
:10AD1800816923F0200321F0807143EA061321F4AE
:10AD2800E641B84243EA051341EA0E2148D03B4DBB
:10AD3800A84245D092684460816182630362F0BD95
:10AD4800046A9389B2F804E01768334E24F00104CA
:10AD58000462056A4468816943EA0E0321F480317C
:10AD680025F002059BB221F07301B04243EA0503C6
:10AD780041EA070114D0294DA84211D005F54065D4
:10AD8800A8420DD005F58065A84209D005F5806573
:10AD9800A84205D092684460816142630362F0BDB5
:10ADA800D689158A578A23F0080333433D43D6884A
:10ADB80024F4407423F00403ADB233432C43E9E791
:10ADC800D589178AD68823F0800343EA051324F42B
:10ADD8004064558A23F0400344EA870443EA061393
:10ADE80044EA8504A6E7D589178AD68823F4006340
:10ADF80043EA052324F44054558A23F4806344EA43
:10AE0800071443EA062344EA051470E7158A24F474
:10AE1800804444EA851449E7002C0140003401408D
:10AE28002DE9F04FC822002183B07848784CDFF82C
:10AE38000492784D784E794FDFF8FC8123F00DF9B4
:10AE480077487849DFF8F4E1DFF8F4C100221359B4
:10AE5800834200F0C180B3F1804F00F0C980AB425B
:10AE680000F0C880B34200F0C780BB4200F0C68043
:10AE7800734500F0C580634500F0C480434500F089
:10AE8800C380DFF8C0A153457ED00AF5806A5345D8
:10AE980008BF092379D01432C82AD8D15C4C624D36
:10AEA800624E604F04F1C80802E01434A04568D02F
:10AEB800A379002BF9D023794FEA131909F1FF3947
:10AEC800B9F1050F03F00F03EFD835F8190040FA70
:10AED80003F2D207E9D54FF0010A0AFA03F3013B5E
:10AEE800184020F00DFD16F809305149184411EBAF
:10AEF800C002DAD051F83000DFF84CE1217A00F1D5
:10AF080038439B0A1EF8033003F01F0E5B09022B1F
:10AF18000AFA0EFA62D0032B65D0012B03D17B69A4
:10AF28004AEA03037B6193880093B3FA83F3C3F17E
:10AF38001F039BB2DA0800EB820203F00703D2F882
:10AF480020E09B004FF00F0C0CFA03FC2EEA0C0ECD
:10AF5800C2F820E0D2F820E001FA03F343EA0E0336
:10AF6800136269460023022214348DF804208DF8F8
:10AF780005308DF806308DF807301AF089F8A045AD
:10AF880096D103B0BDE8F08F082309EBC3034FF057
:10AF9800010B93F834A00AF01F034FEA5A1ABAF1CA
:10AFA800020F0BFA03F30BD0BAF1030F0ED0DA45F8
:10AFB8007FF471AFD1F814A043EA0A034B616AE742
:10AFC800D1F818A043EA0A038B6164E7D1F81CA002
:10AFD80043EA0A03CB615EE70023D6E7BB694AEA86
:10AFE8000303BB619FE7FB694AEA0303FB619AE736
:10AFF8000123CAE70223C8E70323C6E70423C4E7FB
:10B008000523C2E70623C0E70723BEE72C5D00201F
:10B018003C05030800040040000800400010004000
:10B02800002C014000100240ECFE0208F8FE020865
:10B03800FC5E0020F8E402080040014000140040D3
:10B048000034014000440140340503080149024826
:10B05800FFF742B9CC5D0020004801400149024891
:10B06800FFF73AB9A45D00200040014001490248B9
:10B07800FFF732B97C5D00200004004002494FF020
:10B088008040FFF729B900BF545D002001490248FC
:10B09800FFF722B92C5D0020002C0140014902482D
:10B0A800FFF71AB92C5D0020002C01402DE9F04172
:10B0B80004684A4DA30AAB4272D009D8B3F5801F81
:10B0C8006AD04A3DAB425AD14FF0700E022608E0D2
:10B0D800434DAB4268D00235AB4252D14FF0C00E5F
:10B0E800042647794FEA970C002961D0B0006346DF
:10B0F80085190227D4F80C809F400CEB4503BFB29A
:10B10800384D03F1040C47EA080745F8231045F8C1
:10B118002C20E760EFF31181502282F31288821904
:10B1280005EBC202136973B313620433821905EB8A
:10B13800C202576917B11F6053690433821905EBBE
:10B14800C202976917B11F6093690433821905EB2E
:10B15800C202D76917B11F60D36904330027CAB286
:10B168001F6082F31188304405EBC000036A6BB995
:10B17800E3684FF6FE721340E360BDE8F081BDE876
:10B18800F081BDE8F08105EB0E03CFE7E36843F0FB
:10B198000103E360BDE8F0814FF0480E0126A0E707
:10B1A8004FF0200E00269CE74FF0980E032698E7F4
:10B1B800BF08022306FA03F0BB40DB43E768094DEA
:10B1C8009BB23B4087190CEB470CE3600CF104037E
:10B1D80045F82C1045F823209CE700BF4B001000D1
:10B1E800500010002C5D002030B503685C4D1888B5
:10B1F8005C4CB4FBF2F20139013AAB4294B283B031
:10B2080089B282B266D05848834263D0B3F1804F86
:10B2180060D0A0F5983083425CD000F5806083420E
:10B2280058D0524883425BD000F5806083427DD07D
:10B2380022F4407200F58C3092B283421A80D962AF
:10B248001C850ED0484A93420BD002F540629342C7
:10B2580007D002F58062934203D002F580629342E0
:10B2680001D100221A8601225A611A883C4992B2F9
:10B2780042F001028B421A8062D0B3F1804F61D054
:10B288003B4A934260D002F5806293425ED002F559
:10B29800006293425CD002F5806293425AD002F574
:10B2A8009032934258D002F54062934256D002F54C
:10B2B800806293421ED002F58062934208BF092241
:10B2C80019D002A84FF0012340F8043D19F0D4FD2D
:10B2D80003B030BD254822F07002834292B2A3D158
:10B2E80001201A80D9621C8558611A8892B20243DB
:10B2F8001A80C5E708221F4B03EBC20301A893F885
:10B3080035408DF80440012300228DF805308DF872
:10B3180007308DF8062019F0AFFD1B2CD8D1164B3D
:10B32800019301A819F0A8FD03B030BD01201A80CF
:10B33800D9621C8558611A8892B202431A809CE728
:10B348000022D8E70122D6E70222D4E70322D2E777
:10B358000422D0E70522CEE70622CCE70722CAE777
:10B36800002C014000A24A040034014000100040B3
:10B3780000040040F8E4020819010001204B98423B
:10B388002DD0B0F1804F2CD0A3F5943398422AD019
:10B3980003F58063984228D003F50063984226D0CD
:10B3A80003F58063984224D003F59033984222D065
:10B3B80003F54063984220D003F58063984207D094
:10B3C80003F58063984208BF092202D00020704725
:10B3D80008220C4B03EBC20393F834007047002299
:10B3E800F7E70122F5E70222F3E70322F1E7042257
:10B3F800EFE70522EDE70622EBE70722E9E700BFC2
:10B40800002C0140F8E402082DE9F04F013085B026
:10B41800C3B203930B4602918B4C8C4E002B00F069
:10B428009A8032208A4D8B4FDFF82C921EF002FF53
:10B438004FF4FA7A4FF0100C4FF47A70D9F80430C0
:10B44800C3F30803002B40F0DE80EFF31183002BD9
:10B4580040F0D9802968A26800BF2B689942F9D1C9
:10B46800D7F800E000FB0EF39B1AB3FBFEF300FBDA
:10B4780001314FF0010E0191D9F80430C3F30803EC
:10B48800002B40F08780EFF31183002B40F082807F
:10B498002B68A16800BF2A689342F9D1D7F800B099
:10B4A80000FB0BF2521AB2FBFBF200FB0323019ADA
:10B4B8009B1AB3F57A7FDFD3BAF1010ABED1039B99
:10B4C800002B40F0BD804FF47A7ADFF88C9150461B
:10B4D8004FF0100CD9F80430C3F30803002B75D1D2
:10B4E800EFF31183002B71D12968A26800BF2B6884
:10B4F8009942F9D1D7F800E000FB0EF39B1AB3FB91
:10B50800FEF300FB01314FF0010E0191D9F8043030
:10B51800C3F3080313BBEFF31183FBB92B68A168CE
:10B5280000BF2A689342F9D1D7F800B000FB0BF2AC
:10B53800521AB2FBFBF200FB0323019A9B1AB3F5E4
:10B548007A7FE3D3BAF1010AC4D1029B013B02938B
:10B55800002B7FF466AF05B0BDE8F08FEFF31188DC
:10B568008CF31288A1682368DB0344BFC6F800E0A7
:10B57800A1682B6832685FFA88F888F31188D7F8D1
:10B5880000801A4400FB08F35B1AB3FBF8F300FBD6
:10B598000233D2E7EFF311888CF31288A16823688D
:10B5A800DB0344BFC6F800E0A1682B6832685FFA85
:10B5B80088F888F31188D7F800801A4400FB08F34C
:10B5C8005B1AB3FBF8F300FB023370E7EFF3118269
:10B5D8008CF31288D4F808E02368D90303D5012333
:10B5E8003360D4F808E02B683168D2B282F311884E
:10B5F8003A68194400FB02F3A3EB0E03B3FBF2F322
:10B6080000FB01317FE7EFF311828CF31288D4F845
:10B6180008E02368D90303D501233360D4F808E090
:10B628002B683168D2B282F311883A68194400FB5A
:10B6380002F3A3EB0E03B3FBF2F300FB013118E7AF
:10B6480018461EF077FC3EE710E000E0D06F0020BF
:10B65800D46F0020D86F002000ED00E0204B5B681D
:10B66800C3F3080330B4BBB9EFF31183A3B91D4B7F
:10B678001D4C1868A16800BF1A689042F9D11B4B8D
:10B688001C684FF47A7202FB04F3591AB1FBF4F107
:10B6980030BC02FB00107047EFF31182102383F3D4
:10B6A800128811498C680B6813F4803F104B02D044
:10B6B800012018608C680B49D2B20D68186882F3B3
:10B6C80011880A4B19684FF47A72284402FB01F377
:10B6D8001B1B30BCB3FBF1F302FB0030704700BF0B
:10B6E80000ED00E0D46F002010E000E0D86F0020EB
:10B6F800D06F00202DE9F84F8046FFF7AFFF254EA9
:10B708002549DFF8A0E0254A254D844610274FF447
:10B718007A740120DEF80430C3F30803D3B9EFF3D9
:10B728001183BBB90B68D2F808A000BFD1F800900C
:10B738004B45F7D1D6F800B004FB0BF9A9EB0A0981
:10B74800B9FBFBF904FB0393A3EB0C034345E1D3DB
:10B75800BDE8F88FEFF3118A87F31288D2F808B0A2
:10B768001368DB0344BF2860D2F808B00B68D5F82B
:10B7780000905FFA8AFA8AF31188D6F800A09944F3
:10B7880004FB0AF3A3EB0B03B3FBFAF304FB093343
:10B79800DAE700BFD86F0020D46F002010E000E087
:10B7A800D06F002000ED00E02DE9F04FDFF830C148
:10B7B800474A4849484E494D8046102718F1FF38F6
:10B7C800C0F08480DCF80430C3F30803002B5CD19C
:10B7D800EFF31183002B58D10B68946800BF0868F9
:10B7E8008342F9D1D6F800904FF47A7000FB09FE35
:10B7F800AEEB040EBEFBF9FE00FB03EEDCF80430F2
:10B80800C3F308034FF47A740120FBB9EFF31183F3
:10B81800E3B90B68D2F808A000BFD1F800904B45F7
:10B82800F7D1D6F800B004FB0BF9A9EB0A09B9FB6C
:10B83800FBF904FB0393A3EB0E03B3F57A7FBDD2A8
:10B84800DCF80430C3F30803002BDFD0EFF3118AD0
:10B8580087F31288D2F808B01368DB0344BF286066
:10B86800D2F808B00B68D5F800905FFA8AFA8AF324
:10B878001188D6F800A0994404FB0AF3A3EB0B0344
:10B88800B3FBFAF304FB0933D5E7EFF3118487F32D
:10B898001288D2F808901368D80303D501232B60C7
:10B8A800D2F808900B682868E4B284F31188D6F8B7
:10B8B80000A04FF47A7400EB030E04FB0AF3A3EB29
:10B8C8000903B3FBFAF304FB0E3E97E7BDE8F08FDC
:10B8D80010E000E0D46F0020D86F0020D06F002067
:10B8E80000ED00E030B4EFF31183102282F31288E8
:10B8F8000649074C0A680748013200250A60256096
:10B90800DBB2026883F3118830BC7047D46F002023
:10B91800D06F002010E000E00F4B1B88014643B9B0
:10B928000E4B0F4A1B7810680BB981F00101F6F72E
:10B9380067B90C4B5A691AB118B91A68106058746B
:10B948007047094A18681188084A92FBF1F20121E8
:10B9580002605974704700BFAC6F0020AE6F0020C2
:10B96800B06F0020B46F0020CC6F002020A107002A
:10B978001D4B70B59C68E36C226BDD69C2B1636BCB
:10B988002BB12B0702D5E36C08221A6270BD2A0678
:10B99800F7D5A26A616A8A421FD0511CA069A162C8
:10B9A800825C2069E66C81423285EAD3A362E8E7CB
:10B9B800A906E4D5E26A1AB1988C80B29047DEE70E
:10B9C800E1699B8C6069DBB24E1CE6614354E16916
:10B9D800E368994228BFE261D1E7E26C136823F07B
:10B9E80080031360CDE700BFB83500201D4B70B54C
:10B9F8005C68E36C226BDD69C2B1636B2BB12B070A
:10BA080002D5E36C08221A6270BD2A06F7D5A26A2D
:10BA1800616A8A421FD0511CA069A162825C2069B8
:10BA2800E66C81423285EAD3A362E8E7A906E4D549
:10BA3800E26A1AB1988C80B29047DEE7E1699B8C84
:10BA48006069DBB24E1CE6614354E169E3689942E0
:10BA580028BFE261D1E7E26C136823F0800313602A
:10BA6800CDE700BFB83500201D4B70B51C68E36CEE
:10BA7800226BDD69C2B1636B2BB12B0702D5E36C76
:10BA880008221A6270BD2A06F7D5A26A616A8A423C
:10BA98001FD0511CA069A162825C2069E66C8142BA
:10BAA8003285EAD3A362E8E7A906E4D5E26A1AB1C7
:10BAB800988C80B29047DEE7E1699B8C6069DBB2C5
:10BAC8004E1CE6614354E169E368994228BFE2618C
:10BAD800D1E7E26C136823F080031360CDE700BF61
:10BAE800B835002070B4EFF31186502383F3128821
:10BAF800436B1A68D20720D45D686DB9446A826ABC
:10BB0800944217D081691144D9600ED9A21A5A609B
:10BB18008462002280F850201A6842F00102F1B2D3
:10BB28001A6081F3118870BC704701698A1A5A60DB
:10BB38008562EEE7012380F85030F1B281F3118875
:10BB480070BC704703685B6A03B11847704700BF51
:10BB580003681B6A03B11847704700BF2DE9F04F0F
:10BB6800B0F908500D81EDB2442D8BB00C46164645
:10BB780000F0138207462FD9812D00F0528200F27F
:10BB88008180542D00F0AE8040F29A816E2D00F035
:10BB9800D181802D40F0B280B64B1D780B3D15F059
:10BBA800FF0512D0B44F00220A2621683B88481CA2
:10BBB80020600E702168FF2B02F10102A8BFFF234D
:10BBC800481CAA4220600B70EFDB01231A46184676
:10BBD80062810BB0BDE8F08F052D00F0CC811ED836
:10BBE800022D77D040F23181032D00F09381042D8E
:10BBF80040F084802A46A1492046F6F717FC002128
:10BC08002046F6F743FC216800204A1C01232260E5
:10BC180008701A46184662810BB0BDE8F08F242DD3
:10BC280056D040F2CA80282D00F0BF81382D65D14A
:10BC38000968934A0123481C20600B70216805207D
:10BC4800CD182560087021680A20CD182560087075
:10BC580021680020CD182560087021681078CD185B
:10BC68002560087021685078CD1825600870216813
:10BC78009078CA1822601A460870184662810BB07C
:10BC8800BDE8F08FA02D11D040F2B580B82D00F09E
:10BC9800C681FE2D32D17B4D05F1080635F8021B11
:10BCA8002046F6F7F3FBAE42F8D18EE7764B08460E
:10BCB8001968F6F7D3FB754B20461968F6F7CEFBE3
:10BCC800734B19682046F6F7C9FB01231A467EE72D
:10BCD800704BF6E7042270492046F6F7A7FB0123CC
:10BCE8001A46CAE70B6800205A1C0A6018700968CF
:10BCF8000123CA1822601A460870BEE72146284662
:10BD080003F09EFB00287FF460AF742D00F0F580EF
:10BD1800772D0CD13B687A689A421BBF5A1C3A604F
:10BD2800014619785D4A20461CF0AAFA4DE7F52D20
:10BD380000F0D1817A683E68292DA2EB060300F055
:10BD4800748240F25182392D01F00082532D40F067
:10BD58008582721C3A603178032900F2CC844A1E2D
:10BD68004F4D5048D2B202EB420205EB420201703D
:10BD7800557900293FF429AF013BDBB2AB4240F0D3
:10BD8800BA84821C00231360536013725DB10135BD
:10BD98003B682844013A01333B6013F8011C02F860
:10BDA800011F9042F7D1404B1B78002B3FF40DAF99
:10BDB80019F090FE01231A465FE7202D9ED10B68EB
:10BDC8003A4D591C6A7821601A7023682A78591CE0
:10BDD80021601A702368AA78591C21601A70298971
:10BDE8002046F6F753FB23686A79591C21601A70BC
:10BDF8002168A87909E7822D80D10B682C4A2D4D3E
:10BE080011782A4A581C2060197011892046F6F7C3
:10BE18003DFB294B22681B88FF2B02F10101A8BFBB
:10BE2800FF2321601370A96881F3100189B22046AD
:10BE3800F6F72CFB296801F30F0189B22046F6F7C3
:10BE480025FB1E4B21681878DFE6012D7FF456AFDD
:10BE58000B680022591C21601A7023685A1C226042
:10BE68001D70216824204A1C22602B462A4608702F
:10BE780003E700BF4A460020382E00205B4B002015
:10BE8800514B0020A0460020ACF7FF1FB0F7FF1F62
:10BE9800B4F7FF1FE84C0020A807030861750208E3
:10BEA80078E50208345A0020F8350020283A0020A6
:10BEB800BA460020004600200C4600201A3900200F
:10BEC800522D7FF41BAF0A68B14B501C0321206030
:10BED80003F10C061170062001212268551C25600B
:10BEE80011702268B34202F101012160107000F064
:10BEF800D2809979D8790633EFE73B687A689A4215
:10BF08001BBF5A1C3A6001461978A24A20461CF009
:10BF1800B7F95AE60B685A1C0A601D700B680222B2
:10BF2800591C21601A7021680123CA1822601A4618
:10BF38000D70A2E6984B0A681B88984DFF2B02F1FA
:10BF48000101A8BFFF2321601370A96881F31001C4
:10BF580089B22046F6F79AFA914B20461988F6F7E7
:10BF680095FA296801F30F0189B22046F6F78EFA8F
:10BF780001231A4681E60B228A492046F6F756FA2B
:10BF8800082289492046F6F751FA072287492046B0
:10BF9800F6F74CFA01231A466FE6002A3FF415AE6D
:10BFA800834B136001231A4667E60B68DFF830827B
:10BFB800804E591C022221601A70236806275A1CD9
:10BFC80022601F7023680A22591C21601A70236896
:10BFD80001255A1922601D70B8F800102046F6F79E
:10BFE80055FAB8F802102046F6F750FA23685A199D
:10BFF80022601F7023685022591921601A70236823
:10C008000022591921601A7031882046F6F73EFA45
:10C0180071882046F6F73AFA2B462A462DE6664BF3
:10C028004FE6664B1E780A3E16F0FF063FF4CDAD8C
:10C03800634B644F1E4403F101080A2314E0502B9C
:10C0480000F0A380002529462268501C2060204665
:10C058001370F6F71BFA29462046F6F717FAB0458B
:10C068003FF4B3AD18F8013B0A2BE8D1564A95685E
:10C07800116805EB85054FF6FF726D009542A8BF64
:10C0880015469142A8BF114625EAE57521EAE171F6
:10C09800ADB289B2D8E74D4B21681A78481C2060A8
:10C0A8000A70002A3FF491AD013AD2B2444902EB3A
:10C0B800420201EB42025579002D3FF486AD01356D
:10C0C8001D440133226813F8011F501C9D42206053
:10C0D8001170F7D179E53B687A689A4241F0468059
:10C0E8003B4BFF221A704FF000093A4D08F08EFEC4
:10C0F80049462022384885F8009021F0AEFF8DF897
:10C1080004909DF80430072B01F29580DFF8D48065
:10C11800314F4A469DF8043003EB430308EBC30351
:10C128005B7CE3B19DF8043003EB430308EBC303E6
:10C1380020215B699BB19DF8043003EB430308EBB6
:10C14800C303586947F82200F5F796FA2B7857F891
:10C158002300F5F74FFD2A780132D2B22A709DF8F4
:10C1680004300133DBB28DF804309DF80430072B1E
:10C17800D0D92368591C21601A70002E3FF425ADD0
:10C18800164B336001231A4677E5BD68396870E7B6
:10C198007CE50208418102080C4600200046002088
:10C1A80014390020B0070308BC070308F42A030861
:10C1B8001DF40008282E0020503600204A46002092
:10C1C80078E502082C2E0020F42D0020345A002097
:10C1D800D422002047420020C4580020F9C5010895
:10C1E800A82C0020CC520020212D37D13346721CB8
:10C1F8003A60184D13F8022B6A703B6073782B7005
:10C20800F31C3B60B378AB703846F6F7FDF83B6833
:10C2180028811A46591C396012F8021B69713A6064
:10C228005B78AB7101231A4627E5731C3B603378B2
:10C238000A2B00F0C387502B40F0F0853846F6F7FC
:10C24800E3F8054D28803846F6F7DEF801236880C4
:10C258001A4612E5283A0020282E00200B3DEF2D23
:10C2680000F2498201A151F825F000BF45D000082D
:10C27800FFC60008FFC60008FFC60008FFC6000882
:10C28800FFC60008FFC60008FFC60008FFC6000872
:10C29800FFC60008FFC60008FFC60008FFC6000862
:10C2A800FFC60008FFC60008FFC60008FFC6000852
:10C2B800FFC60008FFC60008FFC60008FFC6000842
:10C2C800FFC60008FFC60008FFC60008B5CF000873
:10C2D800FFC600083BD10008FFC6000819D10008B6
:10C2E800FFC60008FFC60008FFC60008F1D0000816
:10C2F800FFC600087BD00008FFC6000883CF0008EF
:10C30800FFC600085DCF0008FFC600084BCF000835
:10C31800FFC60008F7CE0008FFC6000851CE000887
:10C32800FFC60008FFC60008FFC60008FFC60008D1
:10C33800D3BB0008FFC6000835CE0008FFC60008BA
:10C34800FFC60008DDCE0008FFC60008DBCD0008E8
:10C35800FFC60008FFC60008FFC60008FFC60008A1
:10C36800FFC60008FFC60008FFC60008FFC6000891
:10C378009DCE0008FFC600088DCD0008FFC6000846
:10C38800FFC6000853CD0008FFC60008FFC6000816
:10C39800FFC60008FFC60008FFC60008FFC6000861
:10C3A800FFC6000891CC0008FFC60008D9CB0008DA
:10C3B800FFC600082FCB0008FFC600088DCA00087A
:10C3C800FFC6000865CA000847CA0008FFC600087B
:10C3D800FFC60008FFC60008FFC60008FFC6000821
:10C3E800FFC60008FFC60008FFC60008FFC6000811
:10C3F800FFC60008FFC60008FFC60008FFC6000801
:10C40800FFC60008FFC60008FFC60008FFC60008F0
:10C41800FFC60008FFC60008FFC60008FFC60008E0
:10C42800FFC60008FFC60008FFC60008FFC60008D0
:10C43800FFC60008FFC60008FFC60008FFC60008C0
:10C44800FFC60008FFC60008FFC60008FFC60008B0
:10C45800FFC60008FFC60008FFC60008FFC60008A0
:10C46800FFC60008FFC60008FFC60008FFC6000890
:10C47800FFC60008FFC60008FFC60008FFC6000880
:10C48800FFC60008FFC60008FFC60008FFC6000870
:10C49800FFC60008FFC60008FFC60008FFC6000860
:10C4A800FFC60008FFC60008FFC60008FFC6000850
:10C4B800FFC60008FFC60008FFC60008FFC6000840
:10C4C800FFC60008FFC60008FFC60008FFC6000830
:10C4D800FFC60008FFC60008FFC60008FFC6000820
:10C4E800FFC60008FFC60008FFC60008FFC6000810
:10C4F800FFC60008FFC60008FFC60008FFC6000800
:10C50800FFC60008FFC60008FFC60008FFC60008EF
:10C51800FFC60008FFC60008FFC600081BCA0008BF
:10C52800FFC6000805CA0008FFC60008FFC60008C5
:10C53800FFC60008FFC60008FFC60008FFC60008BF
:10C54800FFC60008FFC60008FFC60008FFC60008AF
:10C55800FFC60008FFC60008FFC60008FFC600089F
:10C56800A9C90008FFC6000871C90008FFC600086D
:10C5780095C800087BC800085FC80008FFC6000807
:10C5880045C80008FFC600081DC80008FFC6000807
:10C59800C3C70008FFC6000895C70008FFC6000803
:10C5A800FFC6000873C7000845C7000831C7000860
:10C5B80009C70008E1C60008BFC60008FFC6000892
:10C5C800FFC60008FFC60008FFC60008FFC600082F
:10C5D800FFC60008FFC60008FFC60008FFC600081F
:10C5E800FFC60008FFC60008FFC60008FFC600080F
:10C5F800FFC60008FFC60008FFC60008A5C6000859
:10C60800FFC60008FFC600084DC60008FFC60008A0
:10C61800FFC60008FFC60008FFC60008FFC60008DE
:10C62800FFC60008FFC6000835C60008BE4B1B78C9
:10C63800DB0760D403F010FFFEF734F901231A4634
:10C64800FFF71BBB731C3B6033780F2B53D8B21C0E
:10C658003A60C3EBC303B54A7178D154F11C396011
:10C668001344B2785A70321D3A60F2789A70721D8B
:10C678003A603279DA70B21D3A6072791A71F21D35
:10C688003A60B2795A7106F108023A60F2799A7101
:10C6980010F08EFE01231A46FFF7EFBA3846F5F779
:10C6A800B3FEA34DE8813846F5F7AEFE0123A88115
:10C6B8001A46FFF7E2BA3846F5F7A6FE9D4D2882DE
:10C6C8003846F5F7A1FE68823846F5F79DFE012346
:10C6D800A8821A46FFF7D1BA3346721C3A6013F89B
:10C6E800020B3B60F31C71783B60B2780CF0C2FE21
:10C6F80000287FF46AAA4FF0FF331A46FFF7BDBA45
:10C708003346721C3A608C4A13F8021B11703B6066
:10C71800874A73789370F31C3B60884BB2789A70A1
:10C7280001231A46FFF7A9BA854B864918684E2295
:10C738001FF014FA01231A46FFF79FBA3246731CFA
:10C748003B60814B12F8021B19703A6072785A707C
:10C75800F21C3A60B2789A703846F5F755FE7B4A73
:10C768000123D0801A46FFF788BA3846F5F74CFE01
:10C77800764D28803846F5F747FE68803846F5F745
:10C7880043FE0123A8801A46FFF777BADFF8CC8169
:10C7980098F80030002B3FF418AA6D4E0025384653
:10C7A800F5F732FE12F0C6FD98F80030A6EC010A43
:10C7B80001359D42F3DBFFF708BA0D2B9BD1731CA3
:10C7C8003B603578072D96D8DFF8948138460C26DB
:10C7D800F5F71AFE06FB05F608EB0605A8803846AD
:10C7E800F5F712FEE8803846F5F70EFE3B6828811B
:10C7F8001A46591C396012F8021BA9723A605B7814
:10C80800EB723846F5F7E8FD012348F806001A46AA
:10C81800FFF733BA731C3B603078060600F10E85CB
:10C82800414B1B78DD073FF5D0A9032828BF00201E
:10C8380003F0DCFD01231A46FFF71FBA3A4B1B78B9
:10C84800D8073FF5C2A903F0FBFDFEF72BF801233B
:10C858001A46FFF712BA344B1B78DA073FF5B5A929
:10C868003C490A78012342F004020A701A46FFF78D
:10C8780004BA2D4B1B78D9073FF5A7A9364A4FF4C0
:10C88800C871012311801A46FFF7F7B9092B7FF702
:10C8980032AFDFF8D0803346721CD8F800503A60C7
:10C8A80013F8022B2A703B607378AB70F31C3B6063
:10C8B800B378642BA8BF6423321D6B713A60F37898
:10C8C800642BA8BF6423721DAB713A603379EB7196
:10C8D800B31D3B607379642BA8BF6423F21D2B72D0
:10C8E8003A60B379EB7006F108033B60F3792B717A
:10C8F8003846F5F789FD7A683B686881D11A0029BE
:10C908000CDD591CD8F800003960521A002A197831
:10C91800417203DD9A1C3A605B7843700DF02EFC7F
:10C9280001231A46FFF7A9B92E5A002068440020AF
:10C93800B82C00208C53002068510020C82C0020FF
:10C94800684B002070FB0208B02C0020FC4A002035
:10C95800544A0020142B0020EE3B00204A460020B9
:10C9680074430020D03B0020BA4B1868F31C0246E1
:10C978002136991E396013F8031C1170591E39604D
:10C9880013F8021C51703B6013F8011C91700333BB
:10C99800B34202F10302ECD112F09CFBFFF715B988
:10C9A800C3F34705122D3FF6A6AEBDB10AAB0DF194
:10C9B800020803EB45094646A9F126093846F5F76A
:10C9C80023FD26F8020FB145F8D1A34B38F8022F02
:10C9D80023F8022FB045F9D1112D09D89F4A6B00D1
:10C9E800023B13440021223223F8021F9A42FBD152
:10C9F8009B49012213460A70FFF73FB9994D00235E
:10CA080038462B60F5F7E8FC012328601A46FFF743
:10CA180034B93346721C3A6013F8025B3B60F31C6E
:10CA280070783B60B178002D00F04984012D7FF4C7
:10CA3800CCA809F0D1FC2B462A46FFF71EB98A4B31
:10CA48001B7813F001017FF456AE731C3B603078FD
:10CA580009F004FC01231A46FFF70FB93346721C8C
:10CA68003A60824A13F8021BD1703B60804A73789F
:10CA78005371F31C3B607F4BB278DA7001231A467E
:10CA8800FFF7FBB83846F5F7BFFC3846F5F7BCFCAE
:10CA98003846F5F7B9FC3846F5F7C2FC3B686D4DEA
:10CAA8001946581C2A68386011F8020B82F82C00C5
:10CAB8003960597882F83610D91C39609B7882F829
:10CAC80037303846F5F7ACFC3846F5F7A9FC384658
:10CAD800F5F7A6FC38462E68F5F796FC70873846B9
:10CAE8002E68F5F791FC3B687A683087D11A0129DE
:10CAF8000ADD591C2A6839601B7882F82E303846BE
:10CB0800F5F78EFC3B687A68D31A032B09DD3846A3
:10CB18002E68F5F779FC708638462E68F5F774FCB0
:10CB2800B086286838E7731C3B604A4DDFF85481AB
:10CB3800337888F8053038462E68F5F765FC308478
:10CB480038462E68F5F760FC7A683B68F083D11A9E
:10CB5800072915DD3846F5F757FCA8F80A003846C6
:10CB6800F5F752FCA8F80C0038462E68F5F74CFC8F
:10CB7800708438462E68F5F747FC3B687A68B084BD
:10CB8800D11A03290BDD3846F5F73EFCA8F80E004C
:10CB98003846F5F739FC3B687A68A8F81000D21ACD
:10CBA800002A05DD591C2A6839601B7882F826306E
:10CBB800FDF7DAFD14F01EFA2F4B1B68002B00F06E
:10CBC8006783286811F06CFF01231A46FFF755B8F0
:10CBD8003346721C3A60DFF8AC8013F8022B88F8F1
:10CBE80002203B60254A73781370F31C3B60244D88
:10CBF800B3782B71331D3B60F378092BA8BF092349
:10CC08003846AB70F5F700FC3B687A682880D11A83
:10CC1800012905DD3846F5F7F7FB3B687A68E881B6
:10CC28009A4207D05A1C3A601B78003318BF012378
:10CC380088F80730FDF798FD3B687A689A423EF419
:10CC4800C4AF5A1C3A601B78EB7001231A46FFF7F1
:10CC580014B800BF684B0020C6570020C8570020F2
:10CC6800EC570020503600202E5A0020B82C002007
:10CC7800A83B0020C82C0020DC2C0020AC2C002075
:10CC88008C530020685100203846F5F7BDFB054657
:10CC98001CF026FEFF283EF498AF0AA9002301F8ED
:10CCA800263DEE080DF101008DF8013001361CF02B
:10CCB800F7FD9DF80130F6B205F00705B34205F11E
:10CCC800010503D19DF80230AB4203D02946304616
:10CCD8001CF0F2FD3B687A68D21A012A7EF775AF1C
:10CCE8005A1C0AA83A6000221D7800F8252D1CF06D
:10CCF800CBFD9DF80330AB420AD0C04B1B683BB15B
:10CD08009A79AA4204D31B681B690BB12846984735
:10CD18003B680AA85A1C3A6000221D7800F8242DA6
:10CD28001CF0A6FD9DF80430AB423EF44EAFB34B69
:10CD38001B68002B3EF449AF1B685B69002B3EF46F
:10CD480044AF28469847FEF740BFAD4B1B78012BF0
:10CD58003EF63BAF731C31463B60AA4D11F8023BCF
:10CD6800AB70F31CD21A3960012A96F801E03B60D7
:10CD780040F399823846F5F747FB012328801A4685
:10CD8800FEF77BBF731C3B6096F80080B8F1110F6B
:10CD98003FF6B1ACB31C3B609B4D737805F8183077
:10CDA8003846F5F731FB40F6CA039842A8BF184643
:10CDB80040F2EE23984205EB4805B8BF1846012318
:10CDC800A0F2EE211A46192091FBF0F16970FEF7E6
:10CDD80054BF731C3B608D4B3278DFF85C821A704D
:10CDE8000023C8F800303846F5F7F6FA3A68D8F85C
:10CDF80000308749874D0343501CC8F8003038601D
:10CE080013780B723846F5F7FFFA28603846F5F7BD
:10CE1800FBFA68603846F5F7F7FAA8603846F5F780
:10CE2800F3FA3846F5F7F0FAFEF7CFBE3346721C30
:10CE38003A60794A13F8021B91703B60737853701B
:10CE480001231A46FEF719BF0722B3FBF2F2C2EB21
:10CE5800C2015B1A7FF44FACD2B202F1FF385FFA1D
:10CE680088F8002A3EF4B1AEDFF8B0A108F1010855
:10CE78009946731C3B6096F90010684B002593F99E
:10CE880002208A4203F1080300F0AF810135062D24
:10CE9800F5D130E43346721C3A60614D13F8022B29
:10CEA8002A713B6073786B713846F5F7ADFA3B68C9
:10CEB80028805A1C3A601B78AB713846F5F7A4FAFB
:10CEC8003B6868805A1C3A601B78EB7101231A464C
:10CED800FEF7D3BE534B06F1080201363E6016F842
:10CEE800011C03F8011FB242F7D1FEF76EBE731C96
:10CEF8003B6033780E2B3FF6FEABB21C3A6070787D
:10CF080003283FF6F8AB4849062202FB03F28B18C8
:10CF1800F51C58713D60B0788854321D3A60F2783B
:10CF28005A70721D3A6032799A70B21D3A607279FD
:10CF3800DA70F21D3A60B2791A7101231A46FEF7C7
:10CF48009CBE731C3B60324B32785A7501231A46DB
:10CF5800FEF793BE721C3A6035781F2D3FF6CBABB7
:10CF6800052B7FF4C8AB3846F5F736FA2F4B43F854
:10CF780025001CF0E5FBFEF728BE2C4D05F1400608
:10CF88003846F5F741FA3B68A5F88000591C1A465F
:10CF9800396012F8021B85F882103A605B7885F8D0
:10CFA80083300435AE42EBD1FEF70FBE731C3B60F5
:10CFB8003578132D3FF69FABB31C3B6070781BF0A0
:10CFC80099F900283FF497AB194B027803F825200C
:10CFD800F21C3A6003EB8503B2785A70321D3A604E
:10CFE800F2789A70721D3A6012493279DA700868DC
:10CFF8000DF052F801231A46FEF73FBEF06E0020EE
:10D00800B34C0020B64C002090590020F42C00208E
:10D0180010570020DC350020D42C0020F85D0020BB
:10D02800144B00200F5700205C360020C437002026
:10D03800F82C0020684B0020E84C0020A349102B56
:10D048004FF0000228BF10230A604A608A60CA6055
:10D058000A74002B3EF4B9AD3A6801391344013221
:10D068003A6012F8010C01F8010F9342F7D1FEF76C
:10D07800ACBD731C964D3B6033782B723846F5F780
:10D08800C3F9A8833846F5F7BFF928833846F5F77A
:10D09800BBF93A686883531C3B601278EA747A6873
:10D0A800D31A032B00F3D5803B68D11A05290EDD6E
:10D0B8005A1C3A601B78EB723846F5F78DF93B68D5
:10D0C800E8605A1C3A601B782B743B687A68D21A5D
:10D0D800002A7EF77AAD5A1C3A601B7885F8213011
:10D0E80001231A46FEF7C9BD731C3B6079493078A5
:10D0F8000870D21A002A7EF768ADB31C3B607278BC
:10D10800003218BF012201234A701A46FEF7B5BD46
:10D118003846F5F779F9704D28603846F5F774F90F
:10D1280068603846F5F770F90123A8601A46FEF7DB
:10D13800A4BD6A4D00232B603846F5F74DF92A68DF
:10D14800012302432A601A46FEF797BD731C3B6011
:10D1580033780A2B38D03846F5F762F93846F5F7B0
:10D168005FF93846F5F75CF9FEF72FBD5A1C1946EA
:10D178003A605B4811F8022B027039605B784370A3
:10D18800042A06D9FF2A3EF4AEAF21680020FEF734
:10D198003CBD54490978994203D8022AF5D1FF2B9E
:10D1A800F3D122680123D11821601370002E3EF4B8
:10D1B8000CAD4D4A32601A46FEF75FBD3846F5F7AA
:10D1C80023F94A4DFFF73EB8B31C3B60484B7278D1
:10D1D8001A70F21C3A60B2785A70321D3A60F278CE
:10D1E8009A7001231A46FEF748BD0AEBC50B38466C
:10D1F8008BF80210F5F708F93B682AF835001A464B
:10D20800591C396012F8021B8BF803103A605A78DF
:10D218008BF80420DA1C3A609A788BF806201E1DD9
:10D228003E6009F10109DB788BF80530C8457FF4C9
:10D2380020AEFEF7CABC4A46FEF79BBF00F07F004F
:10D24800032828BF002009F0E3F801231A46FEF757
:10D2580014BD3846F5F7D8F8A8843846F5F7D4F859
:10D268003B687A68E884D11A03297FF71EAF1A460B
:10D27800591C396012F8021BA9773A605B7885F867
:10D2880020303846F5F7C0F83B687A6868840CE7C0
:10D29800184B194A19481A491A60012302600A6092
:10D2A8001A46FEF7EABC174BB0781988012311FB20
:10D2B8000EF11A4691FBF0F12980FEF7DEBC11F061
:10D2C80081FD01231A46FEF7D8BC00BF942C00202C
:10D2D80010570020F42C0020DC350020E84C0020FA
:10D2E800D42200204A46002035F40008A82C00204B
:10D2F800514B002010490020D10500086449002046
:10D30800CC490020222B00202DE9F04F2DED028B77
:10D31800984B994A1C7893B000F59C41203181467E
:10D3280007911160002C00F07886944A12689042A8
:10D3380040F28A80924A93491768934DDFF888B281
:10D348000592013C03911C7007F48057002F40F0B0
:10D358008880039B5B7D002B40F03386059B1B6810
:10D368001E0401F1F780894B99459BF8023000F2C1
:10D378000285002B40F00385854B0693059B1F68AB
:10D3880017F4805940F0F685039BB5F906605B8B6E
:10D398009E42B4BF002601267E4B1B6813F08053C3
:10D3A80069D0069A127812F001026AD003987A4975
:10D3B800408C91ED037A049107EE900AF8EEE77A33
:10D3C800B4EEE77AF1EE10FA81F27581002E60D1A1
:10D3D800724C94F8A01000295BD17148714900681B
:10D3E80090F82D0000240C604C608C606E49002879
:10D3F80050D10870002A51D0F8064FD56B4A1278E0
:10D40800D1064BD4B9F1000F48D1002B46D17A028E
:10D4180044D4674B1B78002B01F0FF86654B9B7843
:10D42800002E41F0AC873BB1634A644B12681B681D
:10D438009B1A002BC1F29B871020584C05F0F8FB73
:10D44800012384F8A13029E04D4B4E4A1F6805930B
:10D4580007F4805703924C4DDFF86CB1002F3FF46E
:10D4680078AF00214B48F5F7F7F900287FF471AF42
:10D4780007F008FD6DE77C0293D4069A127802F053
:10D488000102464C002184F8A01043490491002E63
:10D49800A3D0454901200870002AADD1484B1A781D
:10D4A800002A50D10399B5F900E0488B898BB5F96A
:10D4B80002407045B4BF8027002747F040037145FC
:10D4C800D8BF3B469B0843F08007A042B8BF3B4605
:10D4D80043F04007A142C8BF3B469B08B5F904404A
:10D4E800B5F9067043F0800EA042B8BF734643F00A
:10D4F800400EA142C8BF73469B0843F0800E274CDC
:10D508008742C8BF734643F0400E94F8A2C08F42CA
:10D51800B8BF73469C4501F0C782A4F8A42084F8DC
:10D52800A620234984F8A2300F78002F01F0288222
:10D538005F2B01F093826F2B01F01981069B1B78FA
:10D54800DE0741F1DD80059B1B6803F00403002B17
:10D5580040F01C860DF140081A4C0022C8F804203F
:10D5680004F15009109240F6330A192740F2833625
:10D578002FE000BF344200202C3E00203042002023
:10D588008C51002010570020EC380020404B4C00F4
:10D598002E5A00200C2B0020BC460020D822002048
:10D5A800684B00206C2A002088220020142B0020C1
:10D5B800A4040020D42C0020D46F0020E82D0020E3
:10D5C8002D6E0020F82C0020C86E002004344C4535
:10D5D80020D0A278E3789A4217FB0261F6D26278EB
:10D5E800043217FB036335F912205245A8BF52468F
:10D5F800B2F5617FB8BF4FF461728A42E6DD9A42A4
:10D60800E4DC21782429E1D840460434F5F714F9FC
:10D618004C45DED1624A634B177898E8030083E8EB
:10D628000300002F00F03B855F4B08935D48012104
:10D63800F5F712F9002840F0AB829BF80330002B75
:10D6480040F0A682594B0793594C23881EB226F006
:10D6580001061FFA86F84345A4F8008000F0D98730
:10D66800544E4FF002090E2014274FF0FF0A86F897
:10D678000090777086F802A005F0DAFA4946494822
:10D68800B4F80080F5F7E8F8002841F0B38128F0F5
:10D6980002039BB2434523800BD0464B1421FF2243
:10D6A80002260E201E7059709A7005F0C1FAB4F85F
:10D6B8000080414B414A197850680A9318F0030FCB
:10D6C80008BF81F00201C1F340010992F4F798FA0A
:10D6D80024213448F5F7C0F830B9069A13785E0764
:10D6E80044BF23F004031370079B1B6813F00A0F51
:10D6F8001AD006212B48F5F7AFF8002800F0AC87C0
:10D708002388580641F1B98007212648F5F7A4F87F
:10D7180050B12B4B2B4AB3F904302B4982FB03023F
:10D72800DB17C3EBA2030B800C211E48F5F794F816
:10D738002288002800F04C8242F480739A422380A9
:10D7480009D01C4B02201421FF2218700E2059709A
:10D758009A7005F06DFA1D4B1B78082B00F0448277
:10D768000E2B00F04182059B1B68590561D5184BAB
:10D778001B79002B00F0258114210A48F5F76CF875
:10D78800002840F023810BF00FFB012005F032F94F
:10D7980000284ED0DFF83C9000264FF0CC0A1EE05F
:10D7A800BD6E00200C2B0020D03B0020203A00202A
:10D7B80016390020783700209F6F0020A06F0020C6
:10D7C8006C43002067666666E62D0020F42C002076
:10D7D800AC46002070690020DEB2022E29D80AFB70
:10D7E80006F8731C59F80870002FF5D1C378D14A90
:10D7F80090F9020052F82330019703220092012188
:10D808003A4604F0C9FC034606EB460000EB00105C
:10D81800079353B1394609EB8000CC2220F01DFC58
:10D82800079B49F808300136F6B218F065FD002864
:10D83800D3D1069B1E7816F0010600F02B82BE4B52
:10D8480001221A70089BB5F906101B68BB485A8953
:10D8580001279142077080F20382B94B4FF07E5244
:10D868001A60B84A039BB5F900E01F8B92F904309F
:10D87800107892F801C0002BAEEB070314BF012209
:10D888004FF0FF32002BB8BF5B42B3F5FA7FA8BF59
:10D898004FF4FA73984280F2E0811B1A07EE903A2F
:10D8A800F8EEE77A049BBE45C3ED007A03DAF1EEA1
:10D8B800677AC3ED007AB5F902E0AEEB0703002BF7
:10D8C800B8BF5B42B3F5FA7FA8BF4FF4FA7398422A
:10D8D80080F2C0811B1A07EE903AF8EEE77A049BB3
:10D8E8007745C3ED017A03DDF1EE677AC3ED017A7E
:10D8F800B5F90400C31B002BB8BF5B42B3F5FA7F30
:10D90800A8BF4FF4FA736345CCBFA3EB0C03002305
:10D9180002FB03F307EE903A049A059BF8EEE77AC8
:10D92800B842C2ED027ABCBFF1EE677AC2ED027A64
:10D938001A6812F4805200F06A81B1F5FA6F824BCE
:10D94800A8BF4FF4FA61B1F57A7F1878B8BF4FF4E1
:10D958007A71A1F57A71002840F072817B4D7C487C
:10D9680085FB013ECB17C3EB6E1303F1010E6FF07D
:10D97800630C30F91EE030F913000CFB0313AEEB17
:10D98800000103FB01F385FB0315DB17C3EB6513EC
:10D9980003441BB207EE903A049BB8EEE78A83ED86
:10D9A800038A002A40F0368423885B0627D4002E99
:10D9B80040F0B3800CF0C3FD13B0BDEC028BBDE8A2
:10D9C800F08F069B1B78DA077FF5DDAE4FF40F70FA
:10D9D80019F0A4FB00283FF42CAF04F0C5FB4FF46A
:10D9E8000F7019F03DFB00283FF423AF04F0BCFB97
:10D9F8004FF40F7019F034FB0028EED119E7554B9E
:10DA0800554AB3F904305549DFED556A09889FED49
:10DA1800557A82FB0302DB17C3EBA2035B1A1BB226
:10DA280007EE903AF8EEE77A67EEA67A77EE876A1D
:10DA3800BDEEE66A16EE103A2033402B40F25887C6
:10DA4800DFED496ABDEEE77A17EE103A2033402B36
:10DA580000F21B879FED457AF4EEC77AF1EE10FAD3
:10DA680041F3B482DFED425A9FED426A01E0F0EEE5
:10DA7800477AF4EEC67AF1EE10FA37EEE57AF6DC7C
:10DA8800DFED3D7AB4EEE77AF1EE10FA41F1A282C9
:10DA9800DFED375A9FED396A01E0B0EE677AB4EEF0
:10DAA800C67AF1EE10FA77EE257AF6D49FED2D7A44
:10DAB800F4EEC77AF1EE10FA00F315869FED307A8E
:10DAC800F4EEC77AF1EE10FA44BF9FED2B7A77EEA9
:10DAD800677A67EEA75A9FED2B5A9FED2B6A9FED49
:10DAE8002B7AA5EE856A27EEA55AA5EE867AE5EE8D
:10DAF800077A049A92ED016AD2ED005A27EEC67AA7
:10DB080065EEA77AA5EEA67AE6EE267A82ED007A89
:10DB1800C2ED017A002E3FF44DAF0A9B1978099B9C
:10DB280001F001011868F4F76BF813B0BDEC028B33
:10DB3800BDE8F08F20F802082F5A0020C0210020ED
:10DB480064220020B02C0020682E00201F85EB5195
:10DB5800D43B00206C43002067666666E62D0020F3
:10DB680035FA8E3CDB0FC93F00000000DB0F49404F
:10DB7800DB0FC940E4CB1641DB0F49C0E4CB16C12B
:10DB8800DB0FC9BF92E741B99730083C15A82ABEF8
:10DB9800BC4B07931B689F077FF556ADBA4CB4F88A
:10DBA800008018F0010F7FF472AD48F0010398452A
:10DBB80023803FF46CADB54B022214211A700E205D
:10DBC800FF2259709A7005F033F8B4F800805EE5CA
:10DBD80022F480739BB29A4223807FF4B2ADAC4B9F
:10DBE8001B78082B7FF4BCAD228822F040039BB23F
:10DBF8009A4223803FF4B7ADA44B02201421FF22A0
:10DC080018700E2059709A7005F012F8ABE5039B56
:10DC1800588B8142C0F20984B1F5FA6FD4BFC0EBCA
:10DC28000101C0F5FA614FF47A7303FB01F1994BD6
:10DC38001D78C0F5FA60B1FBF0F1002D3FF48EAE0F
:10DC48005B78954801FB03F380FB0301DB17C3EB0B
:10DC5800611183E6DFED917A41E6DFED907A21E606
:10DC6800B1F5FA6F80F2E483187A8B1A03FB00F39C
:10DC7800C2F5FA6293FBF2F3C3F1640307EE903A3C
:10DC8800F8EEE77A9FED867A864B67EE877AC3EDE2
:10DC9800007AE6E5844B1B780793002B7FF4D2AD1E
:10DCA800DFF838A2DFF838921AF8030C99F80080E8
:10DCB8005146AAF103070CF0BFF9002800F0BE8313
:10DCC800079BB8F1000F53D107F1080178790CF0E0
:10DCD800B3F9002841F0DB817449B87A0CF0ACF94B
:10DCE800002800F0BF83B8F1020F41F0E7817049C6
:10DCF800F87B0CF0A1F9002841F0E3816D49387DEB
:10DD08000CF09AF9002800F0BF83B8F1040F41F035
:10DD1800DB816949787E0CF08FF9002841F0D781C2
:10DD28006649B87F0CF088F9002800F0BF83B8F185
:10DD3800060F41F0A981624997F823000CF07CF99D
:10DD4800002840F04A875F4997F828000CF074F9DA
:10DD5800002800F0BF83B8F1080F40F04F875A49F8
:10DD680097F82D000CF068F900283FF46BAD0923F3
:10DD78001A4600F034BF13B901238BF80230534B15
:10DD880006931B201F789BF821600CF07FF9012E69
:10DD980007F00109824600F05D8607F0020304934C
:10DDA8009BF82030DFF83C81494C052B00F2D580E8
:10DDB800DFE813F0C500BA00060003010501F8000A
:10DDC800012E04BF05238BF82030B9F1000F12D0C3
:10DDD800039BB8F80000B3F918100022134661F34A
:10DDE8000F0361F31F4361F30F0260F31F422B60BF
:10DDF80003236A600493374FDBF814203B689A4288
:10DE080080F02B8547F230520323CBF81C208BF887
:10DE18002030238843F00203238007F033F83A6860
:10DE2800DBF81C3013440422CBF818308BF8202080
:10DE3800012E40F08A863B68DBF818209A4280F071
:10DE48008C80254B187820B90CF020F9002840F078
:10DE58008480238823F0020323803A68B8F80230CC
:10DE6800642101FB03234FF480600022CBF81030BB
:10DE78008BF820208BF803201CF044FF9BF82030FF
:10DE880093E700BF203A0020163900207837002099
:10DE9800F42C0020682E00201F85EB5100000000A4
:10DEA8000AD7233C642200202F5A00205037002034
:10DEB800553700205A3700205F370020643700208C
:10DEC800693700206E370020733700202E5A002053
:10DED800EC6E0020D46F0020A404002046370020F8
:10DEE80080000020144B00200CF0FCF8012808D119
:10DEF800B84FB8F802303A68642101FB0323CBF825
:10DF08001030BAF1000F03D098F80630002B4BD12F
:10DF1800012E22D0AF4FDBF810203B689A42C0F0A8
:10DF2800098601238BF82030012E3BD098F8073062
:10DF3800012B67D011F08EFF9BF8203035E7B9F13F
:10DF4800000FD1D14FF48060BAF1000F00F0818347
:10DF58001CF0F0FE0023CBF81030049B002B3FF49C
:10DF68000DAA184604F064FE059B1F6817F4805933
:10DF78003FF40AAA1D219848F4F76EFC00287FF4A4
:10DF880003AA964A039BD2881B8BB5F90660991A97
:10DF98008E4240F3E28513449E42B4BF0026012618
:10DFA800FFF7FAB98B4F58E711F054FF03224FF4EB
:10DFB8007A738BF82020CBF81C30864F29E7854FE1
:10DFC80036E7039A013BD27D35F91330002A40F039
:10DFD8005783A3F57A73B3F57A7FA8BF4FF47A73A2
:10DFE80023EAE37307EE903A9FED7D7AF8EEE77A3D
:10DFF80067EE877A7B4AFCEEE77A17EE903A138051
:10E00800FFF7B1B911F026FF032240F6B8338BF8B9
:10E018002020CBF81C306F4FFBE6734F3B78002B6A
:10E0280000F0E587714BDFF8D881DFF8D8B1DFF869
:10E03800D8A1039345465E46049099460EE019F828
:10E0480004109847032C28DC88B93B782AF8020F7B
:10E0580001349C4205F1040580F20A81072CE1B2E3
:10E068003046DBF80430EADD984700B2EDE738F8CF
:10E0780024206B88801A4FF47A719B1A01FB00F0F8
:10E0880040F6CA0290FBF3F00844904240F2EE23B7
:10E09800A8BF10469842B8BF184600B2D5E7DFF8C7
:10E0A8006CA1DFF86C81524C0AF15A064FF0010955
:10E0B80051461AF8010C0BF0BFFFF8B19AF80400AA
:10E0C8009AF802309AF803E000EB400104EB810172
:10E0D800013BD1F8B42003EB4303434493420DD0F2
:10E0E80094F8E02081F8B0E009FA00F022EA000094
:10E0F800C1F8B430C1F8B87084F8E0000AF1060A33
:10E10800B245D5D13B4B08931946324A3A4B3B4C62
:10E1180009681B78D2F8009009910793A4F1B00A16
:10E12800002663685BB31F784FB3A268A9EB0202AD
:10E13800002A0ADB9AF8E0200121B14022EA010214
:10E1480009F5FA718AF8E020A160079ABAB1227835
:10E1580059780432D2B2002940F0B382039935F9D4
:10E168001220098B01F1C800824240F3B5849AF865
:10E17800E0109A7841FA06F3D90740F1298501366B
:10E18800042E04F10C04CCD1FFF750BA184C94F8C3
:10E19800AA3053B1069B1B78D80706D5039BB5F95F
:10E1A80006205B8B9A4200F3E88411210A48F4F7B1
:10E1B80053FB002800F06D8294F8AE302BB994F828
:10E1C800A83013B93223A4F8AC30012384F8AE3058
:10E1D800FFF7C0B9D46F00200C2B0020FC4A0020A8
:10E1E800AAF1823F1439002044590020105700201A
:10E1F800D8220020D03B0020C138002088230020EE
:10E208005C590020203E0020D62200205D360020E8
:10E2180090E502081D21B648F4F71EFB00283FF4DC
:10E22800C3AB9BF80330002B7FF4BEABDFEDB17AB4
:10E23800B14938EE678AC7F5FA63FDEEC87A1BB2B2
:10E24800CDED037ABDF90C20120381FB0201D21730
:10E25800C2EBA11203FB02F343F30F333B4407EE77
:10E26800903A049BF8EEE77AC3ED037AFFF79CBB7C
:10E27800DDF81090A14A059211469F4A096842F2BA
:10E28800010AA2FB092B11EA0A0A4FEA9B1B00F0BC
:10E29800FC819B4D9B489C4C9C4A95F800E000787B
:10E2A80084F800E01070BEF1000F04D0974A92F88D
:10E2B80000E08EF0010E964C0F2084F82400002B0D
:10E2C80000F06B83934B0C931B780B931E463B78A3
:10E2D800039F914AB7F824C0DFF870820A903D4640
:10E2E800FF8C09973746A2FB0662520802EB4202EE
:10E2F8002D8B0E95BA1A94F825500495D2B201F4D4
:10E3080080510892854DCDF834900BF59672DDF862
:10E3180010900F91CDF810E004F128060020069225
:10E328006746A646049A002A00F03A823EF9101081
:10E338001FFA81FCBC454FEA400203D3099CA4455F
:10E3480040F2728258F820108B4580F03282A95E24
:10E35800BAF1000F40F0478201309842A95206F105
:10E368000606DFDB0A996E4A8EF824100F29484604
:10E378000CBF01210021DDF834908EF825001170C2
:10E3880000F01183DFF8C8B1664E674F34883868EB
:10E39800DBF80810DBF80420CBF80C0044F0040488
:10E3A800401A9042574F3480584C4FF0010188BFB3
:10E3B80000223970217088BF8BF82120002B00F0D3
:10E3C8000783059A03991768584EB1F824C0B1F825
:10E3D80018E0524817F48057344640F01D833946F8
:10E3E8000EE0627802EB820202EB820202F2EE2277
:10E3F80092B201318B4220F8022B04F102040ED0B4
:10E4080016F81120002A00F01382022AE9D00131FF
:10E41800028820F8022B8B4204F10204F0D10C9AF6
:10E42800137801331370FEF791BF1146FFF7FFBB56
:10E438001B7AC3F1640307EE903A21E40AF105015F
:10E4480078790BF0F9FD00283FF446ACB8F1010FDC
:10E4580040F01D8607F10D01B87A0BF0EDFD00289C
:10E4680040F02C863249F87B0BF0E6FD00283FF49B
:10E4780045ACB8F1030F40F024862E49387D0BF0E7
:10E48800DBFD002840F020862B49787E0BF0D4FD78
:10E4980000283FF445ACB8F1050F40F0188627492D
:10E4A800B87F0BF0C9FD002840F0EE85244997F8A5
:10E4B80023000BF0C1FD00283FF445ACB8F1070F6D
:10E4C80040F08B831F4997F828000BF0B5FD002812
:10E4D80040F094831C4997F82D000BF0ADFD0028FF
:10E4E8003FF4B0A9B8F1090F3FF4ACA93FE400BF6D
:10E4F8000C2B002000007A44D34D62108C51002070
:10E50800FC3D0020A8040020C1380020A9040020F8
:10E51800D8220020F1580020ABAAAAAAEC38002083
:10E52800152B0020EC6E0020D46F0020905900209D
:10E53800553700205A3700205F3700206437002005
:10E54800693700206E37002073370020F458002008
:10E55800C86E0020CF4CD4F88830A9EB0303002BF9
:10E56800FEF601AFCC4A94F88C30517C079AC4F877
:10E5780088200133C94A039E32F81120B17D03F087
:10E588000F0384F88C30234492B292FBF1F283F8A3
:10E59800902094F8901094F8912094F8923094F880
:10E5A8009C000A4494F89310134494F89420194456
:10E5B80094F895300A4494F89610134494F89720E8
:10E5C800194494F898300A4494F89910134494F82C
:10E5D8009A20194494F89B300A44134494F89D10E7
:10E5E80094F89F20184494F89E3001440B441A4430
:10E5F80042F30B12642AF17DA8BF642213B209B159
:10E60800C2F1640307EE903A9FEDA57AF8EEE77A37
:10E61800EEE40221A348F4F71FF900283FF437A8D5
:10E62800268018F0020F7FF444A848F002034345FF
:10E6380023803FF43EA89C4B022214211A700E201E
:10E64800FF2259709A7004F0F3FAB4F80080FFF7CB
:10E6580030B81CF057FB7DE4228822F040039BB2BF
:10E668009A4223803FF450A88F4B02201421FF22A6
:10E6780018700E2059709A7004F0DAFAFFF744B84F
:10E68800C3F53B6308331BB2A3E4884A92F800E061
:10E6980009E694F8A830002B3EF45CAF069B1B7883
:10E6A80013F001037EF456AF012284F8A83084F8F1
:10E6B800A920FEF74FBF774C012184F8A010FEF780
:10E6C800E8BE012900F045849AF8E0200123B34010
:10E6D80001361343042E8AF8E03004F10C047FF469
:10E6E80020ADFEF7A3BF9FED7E7A77EE677AFFF73E
:10E6F800F0B9069B6E4A1B781060DB0700F14B826D
:10E7080094F8A60000287EF41EAFB4F9A430322B8A
:10E718007EF719AF94F8A2200121572A84F8A61091
:10E7280000F0B884059B1B6813F0040302D05A2A32
:10E7380000F043855D2A00F008855B2A00F02E85ED
:10E748005E2A00F02F85562A00F04E85972A00F0A1
:10E758005A85A72A40F0C6845649059B0A781B6843
:10E7680042F004020A7003F00403FEF7F0BEB2F5AB
:10E77800FA7FFEF6E8AE94F8A620002A7EF4E3AE0F
:10E78800069B1B780121DF0784F8A61000F1A284FC
:10E7980006F076FF059B1B6803F00403FEF7D7BE5F
:10E7A800002F3FD058F820108B454FEA4002FFF465
:10E7B800CEAD4149404C895C04EB020C002900F0C5
:10E7C8000C81022947D19CF8011001EB810101EB72
:10E7D800810101F2EE2189B2032833DD09B2BAF1D1
:10E7E800000F3FF4B9AD089C26F81410B9F1000FDA
:10E7F80003D10B9C022C7FF6AFADB6F8029031889E
:10E80800B6F804C049448C442C490FFA8CFC81FBAF
:10E818000C412B4CA1EBEC7124F802C009B24FF06B
:10E82800010999E539464200069C48F820408FE5E1
:10E83800CAB2022A04D9032A7FF4E9AD6246D8E5B0
:10E848007246D6E5012404FA00FC0A9C24EA0C046A
:10E8580009B20A947CE5A95ABEE71A4B1B78002B2B
:10E868007FF4D0AAB9F1000F3FF4CCAA012E7FF4AF
:10E8780074AB9BF82030FFF798BA43F040029342FC
:10E8880022807FF4F1AEFEF73FBFDFED0F7AFFF78E
:10E8980030B900BFD8220020DC6F0020F86F0020BC
:10E8A80014AE23410C2B002078370020C1380020FB
:10E8B800EC2D0020142B002090590020565555555A
:10E8C800482300207822002000000000E4CB1641F5
:10E8D800DB0F49C0DB0FC940E4CB16C1DB0FC93FD2
:10E8E800DB0F494092E741B99730083C15A82ABE8A
:10E8F800F4EEC77AF1EE10FA40F37D835FED0B5A20
:10E908001FED0E6A01E0F0EE476AF4EEC66AF1EE1A
:10E9180010FA36EEE57AF6DC5FED136AB4EEE67AC5
:10E92800F1EE10FA40F16A835FED165A1FED166A90
:10E9380001E0B0EE667AB4EEC67AF1EE10FA77EE40
:10E94800256AF6D41FED1B7AF4EEC76AF1EE10FAC9
:10E9580040F39E801FED1E7A77EE666A66EEA65A31
:10E968001FED205A1FED206A1FED207AA5EE856A5B
:10E9780026EEA55AA5EE867AE5EE076AFFF762B895
:10E988003946C248F3F768FF00283FF4B2AE84F86E
:10E99800A77006F075FEFEF7D1BDBD49BD4A0C91C2
:10E9A800BD4D012111701B21B8480493F3F754FFA2
:10E9B800049B00287FF4E6ACDFF8FCB2B74FDBF825
:10E9C8000C203B68CBF808309B1AC82B00F2358323
:10E9D800059B1F6807F4805721E5C1B2022940F260
:10E9E800B68203297FF437AF0E990F9C002C08BF1D
:10E9F8003946F1E628F0010292B2424522803FF4FE
:10EA080010AE0E2086F80090777086F802A004F009
:10EA18000FF9B4F8008004E600210FE0627802EBF9
:10EA2800820202EB820202F2EE2292B201318B42A2
:10EA380020F8022B04F102043FF4F1AC16F811207F
:10EA48001AB1022AEAD00288F0E7CAB2032AFAD831
:10EA58007246EBE700230493FFF7A2B9B2F5FA7FF9
:10EA6800FEF671AD94F8A630002B7EF46CAD069BD3
:10EA78001B78012113EA010084F8A61000F0C18276
:10EA880006F000FA059B1B6803F00403FEF75FBD60
:10EA98009FED837AF4EEC76AF1EE10FA44BF9FED5A
:10EAA800817A77EE666A59E77F4A80491068B4F937
:10EAB800A420C76981FB07018911FF17781A00F59F
:10EAC800FF407F3082423EF72CADC91B0A4412B288
:10EAD800A4F8A420FEF725BDC8398A4240DA9AF87E
:10EAE800E0109A7841FA06F3DB073FF548AB52424B
:10EAF80001200A9204F080F97B1E0A9A162B00F274
:10EB08001B81DFE813F0A401BA018B01E301D001F6
:10EB1800F701760161014A0133011C011901E30182
:10EB28000901F70176016101F300DD00AC000C0278
:10EB380094007E0011F08EF9032240F6B8338BF86A
:10EB48002020CBF81C30FFF764B93A68DBF81C309A
:10EB58001344CBF81830FFF700BA0126FEF71CBCA7
:10EB68009AF8E0300122B24023EA020309F5FA726A
:10EB78008AF8E030A260FFF702BB00214348F3F7B0
:10EB88006BFE00287FF411AB322384F8AA00A4F8A6
:10EB9800AC30FFF70ABB464B1B78002B3EF4D3ACD6
:10EBA8009BF80330002B7EF4CEAC94F8A7300133E9
:10EBB800DBB2032B84F8A7307EF6C5AC3D4B5B78FF
:10EBC80013B9002E7EF4BFAC06F05CF9FEF7B6BCB4
:10EBD800002A0CBF012002208BE707231A4602EB0C
:10EBE8008202174489F80030B97878781AF064FE00
:10EBF800069B1E7806F00106FEF724BE08231A4677
:10EC0800EDE7DAF8E400DFF8B48090F8361098F809
:10EC1800023011446429A8BF642121EAE17180F817
:10EC28003610002B40F0608310F054FA4CE5DAF807
:10EC3800E400DFF8888090F8371098F80230114423
:10EC4800FE29A8BFFE2121EAE17180F83710002BC8
:10EC5800EAD016200BF078FADAF8E400E4E7DAF8FC
:10EC6800E400DFF8588081781144C829A8BFC8217A
:10EC780021EAE171817098F80230002BD4D0142079
:10EC88000BF062FADAF8E400CEE700BF0C2B0020A4
:10EC9800F1580020152B0020EC380020D46F0020FC
:10ECA800DB0FC9BFDB0F49C0CC3B0020D34D62103E
:10ECB800C1380020D42C0020C86E0020B64C00209B
:10ECC800DAF8E400DFF8848641781144C829A8BF3F
:10ECD800C82121EAE171417098F80230002BA3D0D5
:10ECE80013200BF031FADAF8E4009DE7DAF8E400D3
:10ECF800DFF8588601781144C829A8BFC82121EA3D
:10ED0800E171017098F80230002B8DD012200BF0C1
:10ED18001BFADAF8E40087E7DFF83086099898F8F4
:10ED28000230417911446429A8BF642121EAE171C4
:10ED38004171002B40F0BC82DAF8E40074E7DAF89D
:10ED4800E400DFF80886017A98F802301144C829EF
:10ED5800A8BFC82121EAE1710172002B3FF464AF1A
:10ED68000B200BF0F1F9DAF8E4005DE7DAF8E400DB
:10ED7800DFF8D885C17998F802301144C829A8BFAE
:10ED8800C82121EAE171C171002B3FF44DAF0A207F
:10ED98000BF0DAF9DAF8E40046E7DAF8E400DFF82D
:10EDA800AC85817998F802301144C829A8BFC821D8
:10EDB80021EAE1718171002B3FF436AF09200BF095
:10EDC800C3F9DAF8E4002FE7DAF8E400DFF87C8525
:10EDD800417998F802301144C829A8BFC82121EA0E
:10EDE800E1714171002B40F07182112F7FF43BAF2C
:10EDF8001AE7DAF8E400DFF85485017998F8023068
:10EE08001144C829A8BFC82121EAE1710171002B6A
:10EE180040F05482102F7FF457AF05E70999DFF8C7
:10EE28002C850F791744642FA8BF642727EAE77752
:10EE38000F710BF0A3F998F80230002B3FF47CAF68
:10EE4800032039460BF080F9DAF8E400ECE609987B
:10EE5800DFF8F88401781144FA29A8BFFA2121EAD9
:10EE6800E171017098F80230002B3FF465AF012082
:10EE78000BF06AF9DAF8E400D6E60998DFF8CC84F2
:10EE8800817811446429A8BF642121EAE171817065
:10EE980098F80230002B3FF44FAF02200BF054F9E2
:10EEA800DAF8E400C0E60998DFF8A084C17998F898
:10EEB8000230114481F30801C171002B3FF43CAFCB
:10EEC80005200BF041F9DAF8E400ADE6099BDFF81C
:10EED8007C84997998F8020011446429A8BF6421B8
:10EEE80021EAE1719971002840F0F8810D2F7FF433
:10EEF80015AF21E7DAF8E400DFF85084C17898F814
:10EF080002301144C829A8BFC82121EAE171C170A3
:10EF1800002B40F0ED810F2F7FF4ECAE84E60998CA
:10EF2800DFF8288441781144B1F5967FA8BF4FF4E3
:10EF3800967121EAE171417098F80230002B3FF494
:10EF4800FBAE15200BF000F9DAF8E4006CE60E9938
:10EF580042E435F912209978B2F5617F4FF496634F
:10EF680093FBF1F33ADB40F633019142A8BF114617
:10EF78000C2FA1F5617191FBF3F100F00D81182FB1
:10EF88007FF4A2ABC9B2C8290B46A8BFC823DAF8D8
:10EF9800E400C27DDFB297423FF496AB9A1ADFF8DD
:10EFA800AC83C77548BF0732D71098F802300137CD
:10EFB800FFB23BB9002F3FF487AB384603F01CFF84
:10EFC800FFF782BB18200BF0BFF8F3E7B0EE677AC3
:10EFD800FEF756BDF0EE477AFEF768BD0C2F00F03D
:10EFE800C380182F7FF470AB00210B46CFE7C44ACB
:10EFF8000392FFF73FB9B0EE667A8DE4F0EE476A08
:10F00800A0E4C04B1B6813F4003340F0CF801846CF
:10F01800BD490E5C0F2E00F10C001CD00133152BDE
:10F02800F7D1059B1B68FA3A0021A4F8A42003F045
:10F03800040384F8A610FEF78ABAB44A059B1F6831
:10F04800138823F004031380012307F480578BF8F7
:10F058002130FFF7E4B9AE4FD7F800E05800BEF111
:10F06800000F07D0C61801EB86069EF801E07678F7
:10F078007645D6D21844A74EA74B01EB8001002055
:10F08800396030801860CCE706231A46A7E50123CB
:10F098001A46A4E5A14BA2491A684FF47A73B3FB48
:10F0A800F2F3C3EB431203EB8202059B1B68D20009
:10F0B800A1F8B42003F00403FEF749BA02231A4664
:10F0C8008DE503231A468AE504231A4687E50523B6
:10F0D8001A4684E5059B93491B680A6003F00403FC
:10F0E800FEF735BA0021BB2A109100F0C380B72A79
:10F0F80000F0BC80BE2A00F0B780BD2A00F09D80D9
:10F108009E2A00F0CF809D2A00F0C580AE2A00F02C
:10F11800BB80AD2A00F0B180EF2A00F05881FD2AAB
:10F1280000F05281FB2A00F04C81FE2A00F0468153
:10F13800F72A00F035817B2A7EF405AA4FF4FA619C
:10F14800022007F08BF8FEF7FEB9774B002201206A
:10F158007649774C0B60227003F04EFE059B1B68C6
:10F1680003F00403FEF7F3B900273946704B0A9100
:10F178005B78BB423FF4A8AADFF8D081384607F095
:10F1880047F998F802300A991BB1C9B20C200AF065
:10F19800DBFF0137FFB20DE7CFB2E7E7654B01228E
:10F1A8000220D5E7644B02220320D1E7634B1B788A
:10F1B800032B00F0F08003462AE794F8A820002AE1
:10F1C80040F0CF8094F8AA3083F0010384F8AA3085
:10F1D800002B40F0BD800C2003F02AFD059B1B6826
:10F1E80003F00403FEF7B3B90DF0ACF8F2F7F6FE3E
:10F1F8000DF090F8FBF756FB012003F0FDFD94F8A5
:10F20800A220FFF7A3BA059B4D4A1B684FF4C871AB
:10F21800118003F00403FEF79AB9002E3EF40CA9FE
:10F22800484C94F8A130002B3EF438A903F0E4FCD4
:10F23800002384F8A130FEF731B94FF6FE73424A35
:10F24800D0899689014433449381D1810DF07AF8AD
:10F25800F2F7C4FE0DF05EF8FBF724FB012003F083
:10F26800CBFDB4F8A420DCE60223E8E70B464FF612
:10F27800FE71E4E70B460221E1E7FF2100201CF0C4
:10F288001FFC94F8A22047E7012100201CF018FC7D
:10F2980094F8A2203DE70021FF201CF011FC94F80F
:10F2A800A22033E701201CF00BFC94F8A2202AE7E7
:10F2B8000E200AF049FFDAF8E400B5E410200A92BB
:10F2C8000AF042FFDAF8E4000A9AA3E511200A924C
:10F2D8000AF03AFFDAF8E4000A9A86E50D200A9265
:10F2E8000AF032FF0A9A01E617200AF02DFF23E5FB
:10F2F8000F200A920AF028FFDAF8E4000A9A0AE6D0
:10F3080010570020503600208CF40208EC6E0020C4
:10F318005C220020B0220020B42200207C51002072
:10F3280000700020EC2D0020764B0020684B002058
:10F33800564B0020C44B0020124C00201A390020E4
:10F34800EE3B0020D8220020B82C0020B64C00202C
:10F358000B2003F06DFC059B1B6803F00403FEF70C
:10F36800F6B884F8A80084F8A910FEF7F0B8194C8C
:10F3780005F088FD002384F8A130FEF78FB8002B34
:10F388003FF44EAF1449154A09684FF47A7000FBF0
:10F398000313136044E703F02FFCB4F9A42040E6FC
:10F3A8000021042006F05AFFB4F8A4300022963B4E
:10F3B800A4F8A43084F8A620FEF7C5B800210320DD
:10F3C800F0E700210220EDE700210120EAE7002113
:10F3D8000846E7E7D8220020D46F0020E82D002057
:10F3E80038B50B4C23688BB15A68821A002A054637
:10F3F80004DA0CE05A68AA1A002A07DB9A68226025
:10F4080018461A6890472368002BF3D138BD38BDD9
:10F41800483E002008B510F00FF8024B024ADA60A7
:10F42800FEE700BF00ED00E00400FA05024A034BC6
:10F43800127819781AF070BAD4220020D522002048
:10F448002DE9F04F2DED028BA0F10A0389B00C468F
:10F45800E72B00F24386DFE813F01C014106410662
:10F46800410641064106410641064106410641065C
:10F47800410641064106410641064106410641064C
:10F48800410641064106410641065F05410641061F
:10F49800410623054106410641063A064106AC05E8
:10F4A800410693054106870541067E054106140677
:10F4B80041060006410641064106F905F1054106E7
:10F4C8003303410641062C03410604034106410665
:10F4D8004106F1024106410641064106D2024106B3
:10F4E800FC00410629046501410641064106410622
:10F4F8004106410641062D014106FB034106C703AB
:10F5080041065403410640034106410641064106AF
:10F518000005C504BE048D04E80041064106370213
:10F528002D024106F601DA0141064106410641066F
:10F53800CF0141064106AE014106410641069F0141
:10F548008801BE027C024106410641066D02410661
:10F5580041066D0441064106410641064106410641
:10F56800410641064106410641064106410641065B
:10F57800410600054106410641064106410641068D
:10F58800410641064106410641064106410641063B
:10F59800410641064106410641064106410641062B
:10F5A800410641064106410641064106410641061B
:10F5B800410641064106410641064106410641060B
:10F5C80041064106410641064106410641064106FB
:10F5D80041064106410641064106410641064106EB
:10F5E80041064106410641064106410641064106DB
:10F5F80041064106410641064106410641064106CB
:10F6080041064106410641064106410641064106BA
:10F6180041064106410641064106410641064106AA
:10F6280041064106410662043804B34E337853B1AB
:10F63800B24F002537F8021F2046F2F727FF33782C
:10F648000135AB42F6DC012009B0BDEC028BBDE808
:10F65800F08FA94E3378002BF5D0A94F0025B84676
:10F66800236817F81520591C21601A7098F80110A2
:10F6780001EB810101EB810101F2EE2189B2204603
:10F68800F2F704FF33780135AB4208F10208E7DCF2
:10F69800D9E79C4D28461BF089FC0028D3DD2B4672
:10F6A8000544226813F8011B501C9D42206011700C
:10F6B800F7D1C8E71AF014F9FF28054600F0F985D4
:10F6C80008A9002601F8116D0DF10E008DF80E60E5
:10F6D8001AF0E6F808A800F8106D1AF0D5F808A88E
:10F6E80000F8086D1AF0C4F823685A1C22601D70CF
:10F6F80023689DF80E20591C21601A7023689DF814
:10F708000F20591C21601A7023689DF81020591C7D
:10F7180021601A7023689DF81820591C2160012067
:10F728001A7091E70B68784E01255A1C0A601D7003
:10F738000B68B278591921601A7003F01FFD23680D
:10F74800724A73495F1927601870B1F90010B2F94D
:10F758000000F3F715F823685A19226018703188E9
:10F768002046F2F793FE28466EE70A68694B6A4915
:10F778001878551C2560107022685878551C25602B
:10F78800107022689B78501C206013702046C9882E
:10F79800F2F77CFE012057E75F4D08462988F2F70B
:10F7A80075FE69882046F2F771FE2046A988F2F7AF
:10F7B8006DFE012048E7594D05F16006A9882046ED
:10F7C800F2F764FEE9882046F2F760FE29892046B0
:10F7D800F2F75CFE2368AA7A591C21601A70236824
:10F7E800EA7A591C21601A7055F80C1B2046F2F76A
:10F7F80035FEB542E2D126E7494952232268501C1A
:10F808002060137011F8013F002BF7D11BE7454822
:10F8180000232268056803EB4301561C6D5C2660D3
:10F828001570026825680A446E1C527826602A7092
:10F83800026825680A4401339278691C0A2B216002
:10F848002A70E6D1FFE6384D0B682A68591C1278F1
:10F8580021601A702B6822689978531C2360002352
:10F8680011702A6821681A4401335279481C032B05
:10F8780020600A70F5D123682A68591C127A216021
:10F888001A7023682A68591CD27821601A70236874
:10F898002A68591C127921601A702B6820465989E8
:10F8A800F2F7F4FD2A682368527A591C21601A700D
:10F8B8002A680BE100212046F2F7D0FD20460021FE
:10F8C800F2F7E4FD0120BFE6184D08462988F2F753
:10F8D800DDFD69882046F2F7D9FDB5F90430144AF0
:10F8E800D91782FB0323C1EBA301204689B2F2F7A3
:10F8F800CDFD0120A8E600BF203E0020EA38002008
:10F9080090590020942C0020B64C0020222B002077
:10F91800242B0020B02C0020FC4A00207443002037
:10F92800D8E50208684B0020D03B00206C4300203B
:10F93800676666669D4D0846298AF2F7A7FD698ABB
:10F948002046F2F7A3FD2046A98AF2F79FFD012081
:10F958007AE6DFF890E20027FEB2714600232268BB
:10F96800501C206016702268501C2060137022689A
:10F9780011F8010F0133551C062B25601070EED1CC
:10F988000137062F0EF1060EE6D1894900232268B9
:10F99800501C206017702268501C20601370226869
:10F9A80011F8010F0133551C0B2B25601070EED197
:10F9B8002368804A581C0721206019702368002199
:10F9C800581C20601970236892F8F020591C216097
:10F9D80001201A7038E60B68774A78491078784A17
:10F9E8005D1C2560187023688978581C2060197080
:10F9F80023689278591C216001201A7024E60B684C
:10FA0800704D591C2A7921601A7023686A79591C2B
:10FA180021601A7029882046F2F738FD2368AA79F0
:10FA2800591C21601A7069882046F2F72FFD236857
:10FA3800EA79591C216001201A7005E60B68002537
:10FA48005A1C0A60204629461D70F2F707FD294610
:10FA58002046F2F703FD20462946F2F7FFFC012075
:10FA6800F2E50B68584A594D1178594A581C2060DC
:10FA7800197011682046F2F7F1FC2368554A591CA1
:10FA8800127A21601A7029882046F2F7FFFCA988AB
:10FA98002046F2F7FBFC29892046F2F7F7FC002103
:10FAA8002046F2F7F3FC20460021F2F7EFFC012094
:10FAB800CAE5084608224749F2F7B8FC0120C3E521
:10FAC8000B68454A581C9178206019702368527851
:10FAD800591C216001201A70B6E50B68374A3F4966
:10FAE800D078374A5D1C2560187023684979581CFE
:10FAF800206019702368D278591C216001201A707F
:10FB0800A2E500212046F2F7C1FC00212046F2F7C9
:10FB1800BDFC00212046F2F7B9FC2368304D0026D1
:10FB28005A1C22601E7023682A68591C92F82C20DF
:10FB380021601A7023682A68591C92F836202160BF
:10FB48001A7023682A68591C92F8372021601A70A5
:10FB580023685A1C22601E7023685A1C22601E707B
:10FB680023685A1C22601E702B682046598FF2F7B2
:10FB78008DFC2B682046198FF2F788FC23682A68C9
:10FB8800591C92F82E2021601A7023685A1C226092
:10FB98001E702B682046598EF2F778FC2B68204699
:10FBA800998EF2F773FC01204EE500BF8C530020BC
:10FBB800A7380020C437002068510020B82C002046
:10FBC800C82C0020144B0020F42C0020DC35002029
:10FBD800E84C002010570020D42C0020A83B00201F
:10FBE800684B002083380020B54E0B687279B54DFC
:10FBF800591C21601A702B682046198CF2F746FCB4
:10FC08002B682046D98BF2F741FC71892046F2F720
:10FC18003DFCB1892046F2F739FC2B682046598C07
:10FC2800F2F734FC2B682046998CF2F72FFCF18907
:10FC38002046F2F72BFC318A2046F2F727FC2A6887
:10FC4800236892F82620591C216001201A70FBE4D1
:10FC58009B4EF378002B00F01E830B680822591C7A
:10FC680021601A7023680122991821601A7023688C
:10FC7800954D591C2A7921601A702368AA78591C55
:10FC880021601A7029882046F2F700FCE98920468D
:10FC9800F2F7FCFB2368F279591C21601A7023687B
:10FCA800EA78591C216001201A70CDE40B68002500
:10FCB8005A1C0A601D700B685A1C0A601D700B687C
:10FCC8005A1C0A6029461D70C2E6804B03F1700574
:10FCD80022681978501C2060117022685978501CCD
:10FCE8002060117022689978501C20601170226879
:10FCF800D978501C2060117022681979501C206036
:10FD0800117022685979501C206011702268997905
:10FD18000733501C9D4220601170D9D193E46C4D7B
:10FD28000846E989F2F7B2FB2046A989F2F7AEFB4B
:10FD3800012089E40B68674F591C3A7821601A70D2
:10FD48003B78002B3FF47FAC0025EEB230460DF037
:10FD5800E5FF23684278591C216030461A700DF07F
:10FD6800DDFF01892046F2F791FB3B780135AB4274
:10FD7800EBDC68E4584D594E9FED598ADFF88C81C9
:10FD8800DFED588A05F120070EE0FCEEE77ACDEDAD
:10FD9800017ABDF8041020460435F2F777FBAF422C
:10FDA80006F118063FF44FAC717C0029F3D04E4B96
:10FDB800D5ED007A1B78012BE7D14C4B1B68DB048F
:10FDC80040F16182F5EE407AF1EE10FA40F08A8255
:10FDD80040F2DC51DFE7084610224549F2F726FBDE
:10FDE800012031E4434B9B8AB3F5006F00F25F8238
:10FDF800B3F5806F00F27482B3F5007F34BF01273A
:10FE080002273D4D05F10C0655F8041B91FBF7F14F
:10FE1800204689B2F2F73AFBAE42F5D1374D384F5A
:10FE280005F10C06B5EC010AD7ED087A80EE270A31
:10FE38001CF008F881B22046F2F728FBB542F1D150
:10FE4800304D05F10C0655F8041B204689B2F2F72F
:10FE58001DFBAE42F7D1FFF7F6BB00258146DFF860
:10FE6800B080DFF8B0B00595049506950795012197
:10FE78004FF6FF7A05E001350B2D00F04F8118F998
:10FE8800011F4F1C4AFA05F3F5D0DE07F3D5BBF87E
:10FE980000302B41D807EED506A8F2F7CDFCEAE7EB
:10FEA800194D08462988F2F7F1FAA9882046F2F791
:10FEB800EDFA20462989F2F7E9FA0120FFF7C4BBD9
:10FEC80068510020684B00208C53002068440020B3
:10FED800B82C00204A460020DC2A0020CC52002002
:10FEE8000000404200E08244B05300208C510020C2
:10FEF800CC2A0020842A0020BC2A0020805100201F
:10FF0800007000202C4B0020DC350020DB9B914149
:10FF180008E60208163900209F4D05F1500628789A
:10FF280018F002FA2368027A591C21601A702368B3
:10FF38006A78591C21601A702368AA78591C2160B4
:10FF48001A702368EA780435591CAE4221601A7089
:10FF5800E5D1FFF778BB0B68904A591C527D2160A8
:10FF680001201A70FFF770BB8D4D05F1800655F81A
:10FF7800041F2046F2F772FAAE42F8D1FFF763BBCE
:10FF8800884D05F14006B5F880102046F2F77EFA54
:10FF9800236895F88220591C21601A70236895F807
:10FFA80083200435591CAE4221601A70EBD1FFF74B
:10FFB8004ABB7A4D0B682A7A591C21601A70A98BA2
:10FFC8002046F2F763FA298B2046F2F75FFA698B2D
:10FFD8002046F2F75BFA2368EA7C591C21601A7004
:10FFE800A98C2046F2F752FAE98C2046F2F74EFA2D
:08FFF8002368AA7F591C216057
:020000040801F1
:100000001A70236895F82020591C21601A70698C99
:100010002046F2F73FFA2368EA7A591C21601A70E9
:10002000E9682046F2F71EFA23682A7C591C2160F1
:100030001A70236895F82120591C216001201A703C
:10004000FFF706BB0B6801229918216010461A7051
:10005000FFF7FEBA08460021F2F704FA0120FFF785
:10006000F7BA534D534E05F1300795F90210524B34
:1000700093F906208A4203F1080336D09E42F7D155
:100080000835BD42F1D1FFF7E2BA4C4B03F15A05F6
:1000900022685979501C2060117022681978501C10
:1000A0002060117022685978501C206011702268FD
:1000B0009978501C206011702268D978501C2060FB
:1000C0001170226819790633501C9D42206011700E
:1000D000DED1FFF7BCBA0B68394A581C1178206092
:1000E0001970F7E40020FFF7B3BA23685A1C2260A6
:1000F000197029882046F2F7CDF92368EA78591C4F
:1001000021601A7023682A79591C21601A702368AB
:10011000AA79591C21601A7023686A79591C2160D8
:100120001A70ADE7DFF8A4A000254FF008080135EC
:10013000C5F1200208FA02F2A5F120032AFA05F619
:10014000164328FA03F31E43252D06F001024FF053
:1001500000030BD01343EAD0E8B209F09BFF00285C
:10016000E5D0294606A8F2F76BFBE0E7154B1B78B4
:10017000DA0700F1A9800025134E2F4602E0013571
:10018000252D25D029463046F2F76AFB0028F6D007
:10019000294606A8F2F764FB002873D10137EEE781
:1001A000F82C002010570020C0370020C437002052
:1001B000F85D0020EC560020BC5600205C36002084
:1001C000F42C00202E5A0020206E002090E33FF4F3
:1001D000644B654DB3F850102046F2F75BF90021EF
:1001E0002046F2F757F9614B19684B0103F02002E2
:1001F000C1F340031343C1F3800243EA4203C1F356
:10020000C00243EA8203C1F3401243EAC20301F091
:10021000100119432046F2F73DF904A904222046B3
:10022000F2F708F923682978514A581C20601970A0
:1002300011886429A8BF64212046F2F72BF9B9F18F
:10024000960F46D000212046F2F724F92168B7F135
:10025000190348BFA7F11203A3F3C4034A1C226089
:1002600020461A460B7005A9F2F7E4F82368414AC4
:10027000581C10212060197020461188F2F7F2F8FE
:10028000FFF7E5B9394604A8F2F7DAFA86E7F4EEA3
:10029000C87AF1EE10FA45DA4FF47A717FE50B680F
:1002A000B178354A581C2060197023681278591C9F
:1002B00021601A70DFE40827A7E523685A1C226032
:1002C00001201D70FFF7C4B9069B43F0010306939C
:1002D00051E723680322591C21601A7023686A7849
:1002E000591C21601A70B1E704278EE5F4EEC87A34
:1002F000F1EE10FA3FF570ADF4EEE87AFDEEE77A34
:10030000F1EE10FA17EE901A1ED86FF4F973303927
:1003100003FB01F140F2E73391FBF3F101F2DB5112
:1003200089B23CE5FDEEE77A40F2E73217EE903A0B
:10033000303B02FB03F388FB0312D917C1EB6221A8
:1003400001F2E93189B22AE540F2F313A1F58361A4
:1003500003FB01F140F2E73391FBF3F101F2DD51D0
:1003600089B21CE5FC000020564B0020203A0020FA
:100370002E360020EC6E0020AC2C00201B4C08B563
:1003800001210220F1F74AFC237803F00502052A37
:1003900028D003F00903092B08D000210120F1F730
:1003A0003DFC00210846F1F739FCFEE7104C94E8CB
:1003B00006000B68A0684FF6FE752B400B60138893
:1003C00023F001031B041B0C138018B12922002306
:1003D0008271C37101224E21F0F780FFA068F1F70E
:1003E00007FCDAE70FF0BEF82378D2E7B435002037
:1003F000C0230020022828BF022010B4084C094B5B
:10040000207000EB8002C0EBC20207495DF8044B8C
:10041000013003EB4203C0B20B6002F0F1BC00BF3D
:10042000564B0020764B0020684B002008B50BF09F
:100430008DFFF1F7D7FD0BF071FFFAF737FA0120C6
:10044000BDE8084002F0DCBC08B5FAF7E1FB0BF0B0
:100450007DFFF1F7C7FDBDE808400BF05FBF00BFAF
:1004600008B50BF073FFF1F7BDFDBDE808400BF0D8
:1004700055BF00BF2DE9FF4107461AF09BFD082834
:100480004AD1002501AE7C5D1BF04CFB2044437833
:1004900003F00303022B08BF203CAC550135082DA7
:1004A000F1D10025DFF87C808DF80C507C5D1BF0CD
:1004B00039FB2044437803F00303022B08BF203CA0
:1004C0007455E4B2214640461DF000FE28B10135C6
:1004D000214670191DF0FAFD20B109F0FBFB04B0B4
:1004E000BDE8F081082DE1D10D4930460BF0F8FE52
:1004F0000B4C0C4800231A5D04A90A44195C02F84D
:100500000C1C0133082BF6D1002301A906488DF8F5
:100510000C3009F0D3F9E2E70028E9D0DDE700BFAD
:10052000105700209CF90208C50703082DE9F74F72
:1005300080461AF03FFD464E04463768E8B9454804
:10054000454EDFF8388109F08EF80C25204602F080
:1005500047FB384205D005FB04634046996809F023
:1005600082F80134132CF1D117B93C4809F09AF8FC
:1005700003B0BDE8F04F09F016B902463849DFF87C
:10058000D89040461DF0B8FD054670B9354809F0D1
:1005900089F82C46344D09EB0403284699680C343D
:1005A00009F061F8FC2CF6D1E2E798F800302D2B29
:1005B00003BF08F1010804F1FF344FF0010A4FF0C6
:1005C000000A00250C2303FB05924046D2F808B030
:1005D0000193224659461DF08FFD019B70BBBAF175
:1005E000000F18D0132D0BD1204B3360204809F099
:1005F00059F81D48594603B0BDE8F04F09F05EB9FF
:10060000142D02D173683360F0E7284602F0E8FA4F
:1006100038433060EAE7132D05D1C6F800A015482D
:1006200009F040F8E5E7142D01D17760F7E7284697
:1006300002F0D6FA27EA00003060F0E70135152D08
:10064000C1D10D4803B0BDE8F04F09F03DBB00BF7C
:1006500050360020CC0703088CF40208D6070308A4
:10066000E2070308E7070308DE070308FFFF0700A8
:10067000FF07030808080308F2070308DD0703085B
:100680002DE9F84F05461AF095FC384F0446D7F887
:100690000090B0B93648374D374F09F003F80126BE
:1006A00055F8241049B106FA04F313EA090F02D0F1
:1006B000384608F0D8FF0134F2E7BDE8F84F09F0FA
:1006C00072B802462D4928461DF016FD78B92C480F
:1006D0002C4C2D4D08F0E6FF54F8041F0029ECD0F7
:1006E0000B78002BF8D0284608F0BDFFF4E72B78F4
:1006F000DFF880B02D2B03BF013504F1FF344FF03C
:10070000010A4FF0000A00265BF82680B8F1000FBE
:1007100004D11E48BDE8F84F09F0D6BA224641463A
:1007200028461DF0E9FCF8B90120B040020604D5C6
:100730001748BDE8F84F09F0C7BA8305F8D4BAF1F5
:10074000000F0AD0F1F710FC124808F0ABFF414649
:100750000D48BDE8F84F09F0B1B840EA090038602B
:100760000D4808F09FFFF2E70136CDE7E84C002086
:100770001008030810F402081A080308E207030827
:10078000E70703080CF40208DE070308F207030872
:100790001E080308FF0703080808030870B506468B
:1007A0001AF008FC124C054690B111220021204697
:1007B0001DF057FC2A460F4930461DF0C4FC38B1E5
:1007C000102D2A46314628BF102220461DF0CDFCB0
:1007D0002378074A002B08BF0121064B1CBF0021CC
:1007E00013460120044ABDE8704009F0CFB800BFAD
:1007F000942C0020BE2803082A0803082DE9F041A4
:1008000088B0804608F0D4FE054608B33B4CDFF8BC
:10081000F480002519274FF46176237917FB0363D1
:100820000493E37817FB03630393A378029363783D
:10083000019314F8053B009342462B46002101200A
:10084000013509F0A3F80A2DE7D108B0BDE8F08121
:1008500040461BF05FF90928064648DC840027184B
:1008600008F101008DF81F5008F0AAFE234D8046C4
:1008700048B11BF04FF90D2805D89DF81F30E855F9
:1008800001338DF81F30404608F09AFE804660B173
:100890001BF040F9431E042B07D8A3192B445870B2
:1008A0009DF81F3001338DF81F30404608F088FE58
:1008B000804660B11BF02EF9431E072B07D89DF828
:1008C0001F3034442C440133A0708DF81F30F91CC4
:1008D0000DF11F022944404608F07FFE9DF81F30AD
:1008E000052BB2D0EA190023EB511371ADE70922B1
:1008F0002946034808F0EFFFA7E700BF4337002071
:100900004808030832080308F7B5074608F050FE08
:10091000044630B100223649012009F049F803B0FD
:10092000F0BD38461BF0F6F80E28054659DC0626C1
:100930004643781C8DF8074008F042FE2C4C0746D1
:1009400050B11BF0E7F8032806D8A31958719DF899
:10095000073001338DF80730384608F031FE07467E
:1009600058B11BF0D7F80D2807D806236B43E05485
:100970009DF8073001338DF80730711C0DF1070227
:100980002144384608F029FE08F01AFE074660B1F7
:100990001BF0C0F8182808D8062303FB0543D870BD
:1009A0009DF8073001338DF80730384608F008FE0F
:1009B00060B11BF0AFF80D2808D8062303FB0545EE
:1009C0009DF80730287101338DF807309DF8073006
:1009D000062BA4D0A2190023A351938009F07AF921
:1009E0009DE70E222146034808F075FF97E700BFF8
:1009F0005C360020480803082DE9F047014690B016
:100A0000814D0646814808F059FF00232B70804B2A
:100A100006221978304640246C7004F0D5FC0A2078
:100A2000FAF7C6FE2B78DBB20C2B40F2E9809DF87A
:100A30000C60FE2E2BD0FF2E0BBF15240F2401259A
:100A400000259C4240F0DC80611EC9B268460DF072
:100A50004FF910AB1C4414F8413C834240F0CC8069
:100A6000012D9DF80D1014D0022D12D001F01F079A
:100A700061374C09674808F015FE022D71D0611EE0
:100A800004296AD8DFE801F00B5D61696500022581
:100A9000D7E70E469DF80E709DF80F40EAE75E48D6
:100AA00009F012F95D48DFF8C881DFF8C8A108F045
:100AB000F9FD00244FF003091DF8041040460134ED
:100AC00008F0D1FD0C2C54D108F06DFE022D5AD047
:100AD0006422B6FBF2F102FB11623B46D2B2C9B20C
:100AE0004F4808F0EBFE6B1E012B7CD84D4B4E4A55
:100AF0009DF810104D484E4E002914BF114619465E
:100B000008F0DCFE9DF811104A4B4B48002914BF39
:100B10001946314608F0D2FE022D64D19DF81240EC
:100B2000464808F0BFFDA4B3FF2C42D00A22B4FB14
:100B3000F2F102FB1142D2B2C9B2414808F0BEFE46
:100B40002AE0404809F0C0F8ACE73F4809F0BCF89B
:100B5000A8E73E4809F0B8F8A4E73D4809F0B4F822
:100B6000A0E700230DF11F008DF83F3009F0ACF82D
:100B700098E794FBF9F303EB43039C429CD1504666
:100B800008F090FD98E73A463146324808F096FE64
:100B9000A9E7304609F098F89DF813402E4808F070
:100BA00081FD54B1FF2C21D021462C4808F086FE4F
:100BB00006E02B4809F088F8EEE71D4809F084F8B4
:100BC0001B4D274E1B4F00240DEB04031A7D8AB1E9
:100BD000FF2A0CBF32463A4621462248013408F02B
:100BE0006DFE042CF0D110B0BDE8F0871C4809F070
:100BF0006BF8E5E72A46EFE71B4809F065F8F2E7EE
:100C00001A4809F061F8EEE7CC23002071080308C8
:100C10004A460020820803088D080308BB08030821
:100C2000D2080308570803084E08030809090308F7
:100C3000610803085E080308200903082709030860
:100C40003B090308940803089C080308A408030848
:100C5000B3080308EE080308430903089E260308A7
:100C600065080308530903085E0903086E090308B1
:100C7000CD080308BE28030838B50D461AF04AFF10
:100C8000041E09DB0C4B1B789C4205DA21460B48FD
:100C9000F1F7EEFC204638BD2DB1FF2C03D10848FA
:100CA000F1F7E6FCF6E7044B064819780139F1F74D
:100CB000DFFC4FF0FF34EDE74A46002077090308D8
:100CC0008A0903089F09030810B504460B4808F079
:100CD000E9FC0B4B5868F1F7D3F80A4B186801F0A0
:100CE0007DF90EF0ADFB084B084A24B108490948CC
:100CF0000860DA6010BDDA6010BD00BFC6090308E5
:100D0000CC2300204036002000ED00E00400FA056E
:100D1000FC9F0020EFBEADDE38B5084D6868F1F7E6
:100D2000AFF8074B00241C702C72C5F808410EF078
:100D30000BFD2046FFF7C8FF6C6038BDCC230020B8
:100D4000BD6E00200120BFE770B5044608460E4680
:100D50001AF030F93146024620461DF0CDF908B1AF
:100D6000002070BD1AF0DEFE054630461AF022F96A
:100D7000235C1D446A78120701D4002BF0D10130A6
:100D8000204470BD2DE9F04F82468FB091460E464B
:100D9000154600273378089373780993F3780A93FC
:100DA00096F904300B9396F9028096F905300C936E
:100DB000B3790D93B8F1000F04D10FB0BDE8F04F37
:100DC00008F0F1BCB9F1000F4ED02B78089C6A787E
:100DD00095F90210E87895F904E095F905C095F8C1
:100DE00006B09C423ED1099C94423BD1884539D102
:100DF0000A9C844236D10B9C744533D10C9C6445CB
:100E000030D10D9C5C4514BF002401240390029155
:100E100001920093CDF818B0CDF814C0CDF810E0D1
:100E20003B46124A2146504608F09AFD0D9B069318
:100E30000C9B05930B9B04930A9B0393099B0193C3
:100E4000089B0093CDF808803B46084A214650464F
:100E5000013708F09BFD102F06F1070605F1070585
:100E600098D1AAE70024D1E74C46DFE7D20903086E
:100E70002DE9F0478AB005461AF09CF8024630B9D1
:100E800087490120FFF77EFF0AB0BDE8F087052201
:100E9000844928461DF030F9044660B970220146A5
:100EA0007F481DF0DEF8804B20462246C2500C30B1
:100EB0006028FBD1E8E704227C4928461DF01CF994
:100EC000044620BB284608F07BFB06460028DBD002
:100ED0001AF070F8DFF8F881074658F824501DB969
:100EE000734808F0F1FECFE73A46294630461DF038
:100EF00003F950B920460CF035FA29466D4808F040
:100F0000DDFC6D48FFF7B4FFBEE70134E5E70722DB
:100F10006A4928461DF0F0F80446002875D12021C2
:100F200028461DF0D3F806461AF044F8054680BB63
:100F3000634808F098FB2C46624D21462846013450
:100F400008F091FB0E2CF8D108F02DFCDFF884910D
:100F5000554FDFF8848100242146484608F083FB82
:100F60000C26DFF878A1002506FB04763268564887
:100F70000123AB40134214BF41465146013508F0EE
:100F800072FB0E2DF2D1013408F00DFC082CE3D1D8
:100F90007AE7304601AA4D494C4E1AF017FE02ADD1
:100FA00000283DD0022C15D1029A072A2AD803998D
:100FB0000D2927D80378722B17D06E2B22D10C2342
:100FC00053433948012202FA01F1C25822EA0102D0
:100FD000C25013E01AF09EFD01AA45F824003146E4
:100FE00000201AF0F3FD0134DAE70C232E4C5343B2
:100FF000012000FA01F1E0580843E0502F48FFF7C4
:1010000037FF41E708F066FEF8E7284601AA2F49B6
:101010002E4E1AF0DBFD002402AD78B1082C02D16F
:1010200008F058FE30E71AF075FD01AA45F82400D3
:10103000314600201AF0CAFD0134EEE7082CEFD14A
:10104000029B0F2BECD8DDF80CC0BCF1070FE7D8E2
:10105000049F0D2FE4D8059E06F16402C82ADFD84C
:10106000069DFF2DDCD807986428D9D808996429F3
:10107000D6D88842D4DA099C032CD1D8DFF820E0F6
:10108000C3EBC3020EEB02030EF802C018715F70CF
:101090009E70DD7059719C710748FFF7E9FEF3E619
:1010A00068440020EF09030874430020F509030891
:1010B000F2070308FA090308C5090308040A03082C
:1010C000E00703080C0A0308110A0308150A0308BD
:1010D00070E902089E260308420A03085F08030815
:1010E0002DE9F04FDFF820B189B0804689461646D9
:1010F0000D4614464FF0000A002E71D06A686368EE
:101100009A426BD1AF68A368FB1A5F425F4194F9C2
:101110000B30049394F90A300393B4F90830029326
:10112000B4F906300193B4F9043000935A4653469B
:101130003946404608F014FC95F90B30049395F9B4
:101140000A300393B5F908300293B5F906300193DC
:10115000B5F9043000935A465346394640460AF1E1
:10116000010A08F013FCBAF1080F05F10C0504F1AF
:101170000C04C1D10024DFF894A0254696B30027C3
:10118000012303FA07FB325959F8043053403BEA74
:10119000030314BF0123002312EA0B0F079306D0A9
:1011A00000972B4652460799404608F0D9FB59F85C
:1011B00004301BEA030F06D000972B4652460799CE
:1011C000404608F0E3FB01370E2FD9D10135082D39
:1011D00004F10C04D2D109B0BDE8F08F002796E7E6
:1011E0003746A9E73746012359F80420BB4013428C
:1011F00006D000972B4652460121404608F0C6FB18
:1012000001370E2FEFD1E1E7170A03082F0A030871
:10121000F0B585B0054608F0CBF9002838D1044672
:101220002B78002B3BD1062C41D1BDF904309AB26A
:10123000072A3CD8BDF90610A1F2EE2292B240F284
:10124000DC54A24233D8BDF90820A2F2EE2080B2CD
:10125000A0422CD8BDF90A00814228DC824226DB5C
:10126000914224DCBDF90C5005F16404A4B2C82CF1
:101270001DD8BDF90E40112C19DC1A4E0C2707FBA6
:1012800003639980DA8018819D72DC7205B0F0BD2D
:1012900014490022012005B0BDE8F04020E72D2BC5
:1012A00003D0A3F13002092A16D8052C04DD05B0BD
:1012B000BDE8F04008F00EBD28461AF02BFC04AB48
:1012C000661C03EB440424F80C0C15F8013F303B7A
:1012D000092BFAD93446A3E7202BE8D1013526465D
:1012E000F8E700BF744300202DE9F04FDFF8E8A0D5
:1012F00085B0054688461446002706237B430393A2
:101300000026039B334408EB030292F8C0B0002C84
:101310005ED02344524693F8C0300193ABEB0300F8
:10132000D0F1000949EB000900963B4649462846A2
:1013300008F016FB8DE840083B46524649462846D1
:10134000013608F023FB062EDBD10137062FD4D15E
:10135000DFF884B008F1E40A00261AF8019B002C9B
:1013600038D0A3195A4693F8E4300193A9EB03014E
:101370004F424F41009606233946284608F0F0FABE
:101380008DE840020623144A39462846013608F003
:10139000FDFA0B2EE1D198F8F0606CB194F8F030C2
:1013A0000193F21A54425441002300930A4A07233E
:1013B0002146284608F0D4FA00230093019607231B
:1013C000054A2146284608F0E1FA05B0BDE8F08F4D
:1013D000A146AFE72746D3E7440A03087FB5054691
:1013E00008F0E6F8044630B1002218490120FFF762
:1013F0007BFF04B070BD28466A461549144E1AF0AA
:10140000E5FB01AD78B1032C02D108F063FCF0E7F5
:101410001AF080FB6A4645F82400314600201AF095
:10142000D5FB0134EEE7032CEFD101AC70CC324692
:101430002946E0B208F022F80028E6D033462A46D2
:101440002146044808F03AFAD3E700BFC437002029
:10145000150A0308440A03082DE9FF47DFF86CA0CA
:10146000814690460E4615460027B8F1000F2AD057
:101470002B8832889A4224D174886A88A21A5442EE
:101480005441EA780292AA780192009352463B4670
:101490002146484608F064FAF3780293B378019342
:1014A00036F8043B009352463B46214648460137F6
:1014B00008F06CFA102F05F10405D6D104B0BDE890
:1014C000F0870024DDE74446E6E700BF580A03083A
:1014D00070B5064608F06CF8044628B100220F49A2
:1014E0000120BDE87040B7E730461AF013FB0F2823
:1014F00005460BDC304608F063F80146284607F045
:10150000E5FF50B9BDE8704008F0E4BB21460F226A
:101510000348BDE8704008F0DEB970BD44380020D3
:10152000480803082DE9F04FDFF868808FB00746C0
:101530008A46164600240DF124095AF824300293F5
:10154000494602A815F046FF16B356F82430029D0E
:101550000393EB1A5D420DF1100B5D41594603A850
:1015600015F038FFCDF800B02346424629463846EC
:1015700008F0F6F92346CDF8009042462946384651
:10158000013408F003FA202CD7D10FB0BDE8F08F5A
:101590003546EFE76A0A030870B5064608F008F812
:1015A000044628B100220F490120BDE87040B9E788
:1015B00030461AF0AFFA1F2805460BDC304607F01C
:1015C000FFFF0146284607F083FE50B9BDE8704092
:1015D00008F080BB21461F220348BDE8704008F098
:1015E0007AB970BDC4370020480803082DE9F347D5
:1015F000DFF868A081460F46904602260024B8F125
:10160000000F28D037F8242038F824309A4238F8D0
:1016100006201ED1BD5BA91A4D424D410192009397
:10162000524623462946484608F09AF9BB5B019387
:1016300037F8243000935246234629464846013461
:1016400008F0A4F9042C06F10406D8D102B0BDE8D4
:10165000F0870025E2E74546E8E700BF740A030883
:10166000F8B5054607F0A4FF064628B10022274931
:101670000120BDE8F840B9E7254928461CF0F9FCEF
:1016800068B9224B4FF47A714FF4FA6219805A808C
:101690009980DA8019815A819981DA81F8BD2846CA
:1016A0001AF038FA0328044628D8284607F088FF9D
:1016B000064658B11AF02EFA01270546304607F0C3
:1016C0007FFF30B9BDE8F84008F004BB0546074687
:1016D000F4E71AF01FFA002FF4D0A5F2EE2240F240
:1016E000DC539A42EED8A0F2EE229A42EAD8074B97
:1016F00023F8245003EB84035880F8BD31460322BD
:101700000448BDE8F84008F0E6B800BF5C59002086
:10171000EF090308850A03082DE9F04F2DED088B2A
:10172000DFF80C9193B0804692460D461446002691
:1017300095ED008AB5EE408AF1EE10FA71D0D5ED44
:10174000019A95ED029AD5ED038ABAF1000F3FD0C8
:1017500094ED000A94ED01BAD4ED02AA94ED03AA27
:10176000B4EE408AF1EE10FA60D1F4EE4B9AF1EE4D
:1017700010FA5BD1B4EE6A9AF1EE10FA56D1F4EE9B
:101780004A8AF1EE10FA0CBF012700270FA8F0F7E4
:101790008BFDB0EE4B0A83460CA8F0F785FDB0EE4A
:1017A0006A0A059009A8F0F77FFDB0EE4A0A049096
:1017B00006A8F0F779FD049A059B03900292019325
:1017C000CDF800B033464A463946404608F0C8F8DE
:1017D000B0EE480A0FA8F0F767FDB0EE690A0746B9
:1017E0000CA8F0F761FDB0EE490A834609A8F0F7AE
:1017F0005BFDB0EE680A049006A8F0F755FD049B67
:10180000039002938DE8800833464A460021404603
:10181000013608F0BBF8082E05F1100504F110049C
:1018200086D113B0BDEC088BBDE8F08F0027ADE783
:101830008D0A03082DE9F047494E4A4FDFF83C81F5
:101840000446204607F0B4FE814628B100224649EE
:101850000120BDE8F0475FE70522314620461CF035
:101860004BFC40B9404900224318103080281A60D0
:10187000FAD1BDE8F0870422394620461CF03CFC32
:101880000546204615BB07F09BFE8146002864D024
:1018900019F090FB2C465FFA80FA58F8245025B9CD
:1018A0003248BDE8F04708F00FBA5246294648468C
:1018B0001CF022FC40B9204615F064FD29462C4856
:1018C0002C4C07F0FBFFBCE70134E6E71AF022F9E5
:1018D000072805463AD8204607F072FE064648B368
:1018E000F0F73AFC204B03EB051383ED000A0124CB
:1018F000304607F065FE064638B1F0F72DFC1A4B6E
:1019000003EB051383ED010A0134304607F058FE5E
:10191000064638B1F0F720FC134B03EB051383EDBB
:10192000020A0134304607F04BFE28B9BDE8F04703
:1019300008F0D0B90446DBE7F0F70EFC0A4B032CA5
:1019400003EB051585ED030AF0D17FE74946072231
:101950000948BDE8F04707F0BEBFBDE8F08700BF0B
:10196000EF090308F5090308D46B0020F207030808
:10197000FA090308C50903084808030870E90208C2
:10198000084B196861B130B45D68074C642202FBF2
:1019900005F2B2FBF1F2228030BC002018605860E2
:1019A000704700BFD82400202E360020704700BFAB
:1019B000F8B53422044600211CF053FB1423002206
:1019C0005220A3700E4BA272022701221E261F2551
:1019D000642184F83200C4F80330C4F80B30C4F832
:1019E0001330C4F81B30C4F82330C4F82B30A7766A
:1019F00084F8226084F82A502186A2742280F8BDDF
:101A0000050405002DE9F041334DAB6882B013B1F8
:101A10002B7B022B02D002B0BDE8F0812F4E05F1E6
:101A2000100820245527204608F034FB78B398F896
:101A3000003073BB212C4CD0222C45D10322A86846
:101A4000C0B30DF1080EAA230EF8053D4FF0010CAE
:101A500000238DF802208DF800708DF8043069465F
:101A60008DF801C055225340082213F0800F02F177
:101A7000FF324FEA430318BF83F0310312F0FF0235
:101A8000DBB2F2D171450DD011F8012FEBE788F8E8
:101A900000000134E4B2232C08F10108C3D102B0E4
:101AA000BDE8F081AA2269468DF803308DF8042044
:101AB00015F076FA0134E4B20123232C88F80030C3
:101AC00008F10108AFD1EAE73378DB07E1D401225E
:101AD000B5E70222B3E700BFD82400202E5A002029
:101AE0002DE9F04F764D81B0F9F7BCFDAC690022CD
:101AF0006A61002C00F0A180237D052B074617D9D1
:101B0000216A23690B44C31A9342B8BF05F1180137
:101B10000ADBD1E0137D052B0AD9136A126913443D
:101B2000FB1A002B80F2C88051F8042F002AF1D153
:101B30004FF0010B0023B9461E466B6198469A464A
:101B4000274620E07A6A39693B7DA9EB0204B4FBA1
:101B5000F1F40134A4B213FB04F3013301369BB258
:101B6000B6B23C83FB82984506D2BBF1000F01D18F
:101B7000012C5CD99846BA466B69013305EB8302A8
:101B80006B61976947B3BB68C3B1FC8A002CD9D19C
:101B9000396A4846A9EB01019847D0B195F86430FD
:101BA000002B52D13B7DC7F82490013601334FF012
:101BB0000102B6B23A83FB820124D4E73B6A3A6958
:101BC000A9EB0304B4FBF2F4A4B23C8334BBFB8A5C
:101BD000C9E73C83FB8AC6E72B686A683949013349
:101BE00016443C4685E848004F46C1F800A0BAF1CB
:101BF000000F27D0DAF8203095F86420AAF81640B4
